:020000040800F2
:100000000000022051F80008298B00082B8B000803
:100010002D8B00082F8B0008318B0008000000009A
:10002000000000000000000000000000338B00080A
:10003000358B000800000000378B0008398B000862
:1000400095F8000895F8000895F8000895F800085C
:1000500095F8000895F8000895F800083D8B000811
:1000600095F8000895F8000895F800083D5C000830
:1000700095F8000895F8000895F8000895F800082C
:1000800095F8000895F8000895F8000895F800081C
:1000900095F8000895F8000895F800080D8D0008FF
:1000A00095F8000895F8000895F8000895F80008FC
:1000B000618B0008718B000895F8000895F800081E
:1000C00095F8000895F8000895F8000895F80008DC
:1000D00095F8000895F80008218E000895F80008AA
:1000E00095F8000895F8000895F8000895F80008BC
:1000F00095F8000895F8000895F8000895F80008AC
:1001000095F8000895F8000895F8000895F800089B
:1001100095F8000895F8000895F8000895F800088B
:1001200095F8000895F8000895F8000895F800087B
:1001300095F8000895F8000895F8000895F800086B
:1001400095F8000895F8000895F80008658B0008F8
:1001500095F8000895F8000895F8000895F800084B
:1001600095F8000895F8000895F8000895F800083B
:1001700095F8000895F8000895F8000895F800082B
:0801800095F8000895F800084D
:100188000CAA0508000000200C0B0020100B002012
:10019800F4900020064B07481A68074B1A60074B73
:1001A80000221A70064B01221A7001F074B800BFC1
:1001B80080400020180D0020944000206C40002052
:1001C800943A002008B5034801F065F8024B002274
:1001D8001A7008BDA80F0020943A002008B5054BF6
:1001E800012200201A7004F055F80348BDE80840C1
:1001F80001F051B82C4100204C1000202DE9F041AD
:10020800144C204602F08BFB00201349134A02F0DD
:100218003DF91349134A0746002002F037F91249FD
:10022800124A0646002002F031F9D22105463A4624
:1002380023460A2002F042FAD22132462346FA2007
:1002480002F03CFA5A20D2212A462346BDE8F04162
:1002580002F034BA600E0020DA990508CD010008D2
:10026800E3990508E5010008EB9905089D010008D8
:1002780008B5054B012200201A7004F00BF803485A
:10028800BDE8084001F007B82C4100204C100020C0
:10029800044B054800221A70044B02221A7000F021
:1002A800FABF00BF6C400020600E0020943A002086
:1002B80008B5034800F0EFFF024B00221A7008BD92
:1002C800A80F0020943A00202DE9F041144C204654
:1002D80002F025FB00201349134A02F0D7F813490E
:1002E800134A0746002002F0D1F81249124A06467E
:1002F800002002F0CBF8D22105463A4623460A20D0
:1003080002F0DCF9D221324623465A2002F0D6F90F
:10031800AA20D2212A462346BDE8F04102F0CEB9F0
:10032800180D0020DA990508B9020008F4990508A3
:1003380099020008FD99050879020008002008B50F
:1003480003F0A8FF064B00221A70064B1B78022BFD
:100358000CBF05480548BDE8084000F09CBF00BF39
:100368002C410020943A0020600E0020180D002037
:1003780010B5084C204602F0D2FA00200649074A78
:1003880002F084F8D22102462346E620BDE8104058
:1003980002F094B994110020069A05084503000854
:1003A80010B5074C4FF6E071206801F0C3FB2068D8
:1003B800044901F06DFBBDE8104002F0E9BC00BF44
:1003C800100B00200F9A050810B5074C4FF6E07186
:1003D800206801F0AFFB2068044901F059FBBDE833
:1003E800104002F0D5BC00BF100B0020249A05086D
:1003F80070B5514C2DED028B20684FF6E07101F07D
:1004080099FB20684D4901F043FB02F0C1FC002034
:1004180003F040FF23790BB9FFF7C2FF6379464D1C
:1004280053B928684FF6E07101F084FB2868444905
:1004380001F02EFB02F0ACFCA3790BB9FFF7C4FF67
:100448003D4C6379002B69D02379002B66D094ED5D
:10045800038AD4ED048A78EE687A88EE288AA2683E
:10046800384B394D1A6017EE900A0EF075FB0022D2
:10047800364B0EF0C5FB02460B46002034490EF001
:10048800E9FC0EF09FFE334B0646186018EE100A82
:100498000EF062FB0022304B0EF0FEF902460B46CE
:1004A80000202B490EF0D6FC21A3D3E900230EF03F
:1004B800F3F90EF087FEA279286000232371637197
:1004C80002B1A371254A1F4C137031464FF4967040
:1004D80005F025FC29684FF4987005F020FC216888
:1004E8004FF49A7005F01BFC1A4B94ED001A124C4D
:1004F80093ED000AD5ED000A07F09EF820684FF644
:10050800E07101F017FB2068154901F0C1FA07F006
:10051800C6F802F03DFC134802F07EFC1248BDEC20
:10052800028BBDE8704000F0B6BE00BFAFF300809C
:100538000000000000805140100B0020399A050887
:100548004E9A05080C0D0020100D002000005E409A
:1005580000004940140D00200000F03F943A0020AC
:10056800639A050880969800A80F0020014800F0BB
:1005780092BE00BFA80F00202DE9F047384C394D36
:10058800A3686068AB600EF0E7FA064620680F467D
:100598000EF0E2FA0022344B0EF032FB00228046C5
:1005A800894630463946304B0EF078F942464B467C
:1005B8000EF050FC0EF006FE25A3D3E90023686177
:1005C800394630460EF06AF942464B460EF042FC78
:1005D8000EF0F8FDA8614FF6E07003F02FFE686991
:1005E800224E0EF0B9FA05F11C0402460B462046CD
:1005F800314612F07FFF224600236E203A2103F095
:100608004BFFA8690EF0A8FA02460B462046314671
:1006180012F070FF224600236E206C2103F03CFF8D
:10062800A8680EF099FA0CA3D3E900230EF0E8FAB3
:1006380002460B4620460E4912F05CFF6E209E21B2
:1006480022460023BDE8F04703F026BFAFF3008041
:100658000000000000805140000000A2941A6D4282
:10066800E48D0020100B002000005E40779A0508FA
:100678007D9A050870B506F0D9FF10EE104A06F00D
:10068800EBFF064620460EF067FA07EE106AF8EE12
:10069800C77A044617EE900A0D460EF05DFA1AA3C3
:1006A800D3E900230EF0ACFA02460B462046294651
:1006B8000EF0D0FB0EF086FD114CA0600EF04CFA47
:1006C8000DA3D3E900230EF09BFA04F11C050246A2
:1006D8000B4628460B4912F00DFF4FF6E07003F069
:1006E800ADFD00236E209E212A4603F0D5FE01238E
:1006F800A37170BDAFF30080000000A2941A6D4290
:10070800100B00207D9A05081F85EB51B81E194073
:1007180038B506F07FFF0F4C10EE100A84ED030A7F
:100728000EF01AFA04F11C0502460B4628460A493F
:1007380012F0E0FE4FF6E07003F080FD00236E201B
:100748003A212A4603F0A8FE01236371BDE8384028
:1007580026E600BF100B0020779A050838B506F08A
:1007680059FF0F4C10EE100A84ED040A0EF0F4F94C
:1007780004F11C0502460B4628460A4912F0BAFE47
:100788004FF6E07003F05AFD00236E206C212A46D4
:1007980003F082FE01232371BDE8384014E600BF50
:1007A800100B0020779A05082DE9F04F4F4D504E59
:1007B80085B000244FF6FF78284602F0B0F841468D
:1007C800224623464B480094019401F077F9042708
:1007D8007062224623464FF6E0714748009701941D
:1007E80001F06CF9414630602246234643480097A1
:1007F800019401F063F94146B0622246234640481D
:100808000097019401F05AF92346F06241462246C6
:100818003C480097019401F051F93B4930633B4A49
:10082800204601F033FE3A493A4A0746204601F08D
:100838002DFE3949394A8046204601F027FE3849BD
:10084800384A8146204601F021FE3749374A824618
:10085800204601F01BFE3649364A84462046CDF82C
:100868000CC001F013FE21468346726A2B462046CF
:1008780001F024FF214632682B467D2001F01EFF3F
:100888006E21F26A2B460A2001F018FF3C21326BD8
:100898002B460A2001F012FF69213A462B46E62032
:1008A80001F00CFF372142462B46E62001F006FFF7
:1008B8004A462B46E6209B2101F000FF52462B4674
:1008C8006E20C82101F0FAFEC8215A462B46AA20FC
:1008D80001F0F4FEDDF80CC0E620C82162462B4684
:1008E80005B0BDE8F04F01F0E9BE00BF040F0020DD
:1008F800100B0020869A05084E9A05083A9A0508B2
:100908008E9A0508A79A0508C19A05086507000880
:10091800C89A050819070008D09A05087D06000836
:10092800D89A050881050008DE9A050875050008AB
:10093800E59A0508F9030008014B93ED000A704792
:10094800140D0020014B93ED000A7047100D002094
:10095800014B93ED000A70470C0D0020AFF30080A7
:100968002A4B2B48062210B51A704FF6E07400F097
:1009780092FC0020214607F061F83120214607F05B
:100988005DF86320214607F059F89520214607F0C5
:1009980055F8C7204FF4FC6107F050F84EF29C70F0
:1009A80003F04CFC0520012100231A4A03F074FDD2
:1009B800052020210023184A03F06EFD052052214E
:1009C8000023164A03F068FD842100230520144AF9
:1009D80003F062FD4FF4F06003F030FCB621114AD9
:1009E8000023052003F058FD4FF6FF7003F026FCA6
:1009F8000D4A00238720DC2103F04EFD0B4B00221B
:100A08001A600B4B01221A7010BD00BF2C41002048
:100A1800DC120020EC9A0508239B05081B9B05089F
:100A2800F09A050830A00508F29A050884400020CD
:100A38006C40002038B53B4B3B483C4D07221A70B0
:100A48004FF6E07400F027FC0020214606F0F6FF80
:100A58003120214606F0F2FF6320214606F0EEFF22
:100A68009520214606F0EAFF2146C72006F0E6FF5A
:100A78004EF29C7003F0E2FB0520012100232C4A72
:100A880003F00AFD0520202100232A4A03F004FD73
:100A9800052052210023284A03F0FEFC052084216A
:100AA8000023264A03F0F8FC0520B6212A46002335
:100AB80003F0F2FC40F213144FF4F06003F0BEFBB5
:100AC800204601211E4A002303F0E6FC204620218F
:100AD8001C4A002303F0E0FC204652212A4600234A
:100AE80003F0DAFC20468421174A002303F0D4FCE3
:100AF800B621164A0023204603F0CEFC4FF6FF70BD
:100B080003F09CFB124A00237D20DC2103F0C4FC87
:100B1800104B00221A60104A012313700F4A1370F9
:100B280038BD00BF2C410020DC120020199F0508A9
:100B3800F79A0508FB9A0508FF9A0508029B05081D
:100B48000B9B0508079B0508069B05080A9B0508DB
:100B58000F9B0508844000206C4000208C4D00202D
:100B680038B52D4B2D4805241C704FF6E07500F064
:100B780092FB0020294606F061FF2720294606F04F
:100B88005DFF4F20294606F059FF7720294606F0D9
:100B980055FF9F20294606F051FFC720294606F039
:100BA8004DFF4EF29C7003F049FB012100232046C3
:100BB8001B4A03F071FC162100232046194A03F052
:100BC8006BFC3E2100232046174A03F065FC662192
:100BD80000232046154A03F05FFC8E21002320469F
:100BE800134A03F059FCB621124A0023204603F0A9
:100BF80053FC4FF6FF7003F021FB0F4A00237D20C2
:100C0800DC2103F049FC0D4B00221A600C4A012339
:100C180013700C4A137038BD2C410020DC120020E0
:100C2800199F05081A9B05081E9B0508229B0508A5
:100C3800269B05082A9B05082E9B05088440002052
:100C48006C4000208C4D00203B4B3C48042270B582
:100C58001A704FF6E07400F01EFB0020214606F0E3
:100C6800EDFE3120214606F0E9FE6320214606F01C
:100C7800E5FE9520214606F0E1FE314E314D214634
:100C8800C72006F0DBFE4EF29C7003F0D7FA052071
:100C980001210023324603F0FFFB05202021002319
:100CA800294A03F0F9FB052052210023274A03F0C3
:100CB800F3FB052084210023254A03F0EDFB0520E2
:100CC800B6212A46002303F0E7FB40F213144FF441
:100CD800F06003F0B3FA204601213246002303F006
:100CE800DBFB204620211B4A002303F0D5FB2046CE
:100CF80052212A46002303F0CFFB20468421164ABE
:100D0800002303F0C9FBB621144A0023204603F050
:100D1800C3FB4FF6FF7003F091FA114A00237D20C0
:100D2800DC2103F0B9FB0F4B00221A600E4A0123A5
:100D380013700E4A137070BD2C410020DC12002085
:100D48004F9B0508199F05083A9B05084A9B05080B
:100D58003F9B0508449B0508499B05084E9B0508D1
:100D6800529B0508844000206C4000208C4D0020D8
:100D7800F8B5334B3348344F344E03221A704FF6CC
:100D8800E07400F088FA0020214606F057FE632040
:100D9800214606F053FEB3204FF4F06106F04EFEF4
:100DA8002146C72006F04AFE4FF6FF7003F046FAC8
:100DB8004EF29C75DC2100237D20254A03F06CFB54
:100DC800284603F03BFA0520012100233A4603F0A8
:100DD80063FB0520522100231E4A03F05DFBB62168
:100DE80000230520324603F057FB40F213144FF45A
:100DF800F06003F023FA012120463A46002303F06D
:100E08004BFB522120460023324603F045FBB62116
:100E1800114A0023204603F03FFB284603F00EFA50
:100E28000E4A00230520A22103F036FB0C4B0022BA
:100E38001A600C4A012313700B4A1370F8BD00BFE7
:100E48002C410020DC1200206C9B0508199F050826
:100E58005D9B0508679B05086B9B05082B9B050890
:100E6800844000206C4000208C4D002008B5074BC2
:100E7800074802221A7000F00EFA06F0D9FC054B5A
:100E880000221A60044B01221A7008BD2C41002070
:100E9800DC120020844000206C400020002008B5AF
:100EA80003F0F8F9064B00221A70064B1B78022B48
:100EB8000CBF05480548BDE8084000F0ECB900BF84
:100EC8002C410020943A0020600E0020180D0020CC
:100ED8002DE9F14F2D4C204601F021FD00202C4931
:100EE8002C4A01F0D3FA2C492C4A8146002001F003
:100EF800CDFA2B492B4A0746002001F0C7FA2A49A8
:100F08002A4A0646002001F0C1FA2949294A05461D
:100F1800002001F0BBFA2849284A8046002001F049
:100F2800B5FA2749274A8246002001F0AFFAD221B4
:100F380083464A462346E62001F0C0FB28203A466D
:100F48002346014601F0BAFB4621324623462820B3
:100F580001F0B4FB64212A462346282001F0AEFBA9
:100F6800822142462346282001F0A8FB5246234608
:100F78002820A02101F0A2FB28205A46BE212346A2
:100F880001B0BDE8F04F01F099BB00BF4C10002044
:100F9800069A0508A50E0008709B0508750E00083E
:100FA8005D9B0508790D0008529B0508510C000847
:100FB8007B9B0508690B0008869B05083D0A00080D
:100FC800F29A05086909000808B5002003F062F9DB
:100FD80006F0F2FA06F06EF8064B00221A70064B7D
:100FE80001221A7006F088FD0448BDE8084000F0A8
:100FF80052B900BF2C410020943A0020180D00205F
:1010080008B5002003F046F906F0D6FA064B002290
:101018001A70064B02221A7006F06EFD0448BDE8ED
:10102800084000F038B900BF2C410020943A002055
:10103800600E002008B5002003F02CF9034B04488B
:1010480003221A70BDE8084000F025B9943A002040
:10105800040F002010B50B4C06F0AEFA04F0A8F807
:1010680006F023FB06F048FD20684FF6E07100F01B
:1010780061FD2068044900F00BFDBDE8104001F057
:1010880087BE00BF440B0020909B05080088C83825
:1010980080B2042810B505D90A480B4A0B4B7F21AA
:1010A80002F09EF80A4CC0B204F00CF920684FF622
:1010B800E07100F03FFD20680649BDE8104000F0EF
:1010C800E7BC00BFA49B0508C4D30308C49B05085C
:1010D800440B0020F59B05082DE9F04F5248534D6D
:1010E80085B0002401F01BFC4FF6FF712246234611
:1010F8004F480094019400F0E1FC042607464FF69F
:10110800E071224623464B480096019400F0D6FC35
:101118004FF6E071804622462346474800960194E0
:1011280000F0CCFC4FF6FF71814622462346434827
:101138000096019400F0C2FC234628604FF6FF7128
:1011480022463F480096019400F0B8FC3D4968608B
:101158003D4A204601F09AF93C493D4A82462046DC
:1011680001F094F93B493C4A8346204601F08EF948
:101178003A4902903A4A204601F088F93A460390E3
:101188002146294B204601F099FA21464246264B32
:10119800C82001F093FA0A214A46234BC82001F0DF
:1011A8008DFA2A68204B6421782001F087FA78208C
:1011B8006A681D4B014601F081FAC82505262827D3
:1011C800E0B203F0AFFF274A0146284601F05EF976
:1011D80094FBF6F106FB114179431E31024689B2B0
:1011E8000020114B0134013501F068FA042CADB22E
:1011F800E6D1D221524605200B4B01F05FFAD221ED
:101208005A464C20084B01F059FAD221029A064B53
:101218009C2001F053FA039A034BEC20D22105B02D
:10122800BDE8F04F01F04ABAA80F0020440B002097
:10123800059C05080F9C05081C9C0508279C0508AB
:101248003A9A05083B9C05085D100008439C050870
:101258003D1000084C9C050809100008559C05081D
:10126800D10F00089510000808B500F009FAFEF73C
:10127800C5FFFFF799FAFFF727F8FFF729FEFFF7F1
:101288002BFFFFF775F800F08FFA00F0D9F8BDE8EA
:10129800084000F0A1B910B5044628B90F48104A13
:1012A800104B452101F09CFF0F4B1868844213D066
:1012B80010B1C36900219847002002F0EBFF00201D
:1012C80002F0D2FF4FF6FF7002F0B8FFE369204644
:1012D80001219847044B1C6010BD00BF5E9C0508A7
:1012E800D3D303087A9C05084C0B00200048D2E7AA
:1012F800A80F00204FF6FF7070474FF6FF70704739
:1013080013B5002944D04FF2DE7002F0C3FF00206D
:1013180003F08AF80F2002F091FF1E4C1E4A41216B
:1013280001230A2003F0B8F8042003F07DF82368AD
:1013380028209621042B21DC0123184A03F0ACF85D
:1013480001A90DF10602206803F02EFB0F2002F020
:1013580075FFBDF80400BDF80610143828220023D4
:1013680080B202F09BFFBDF80610BDF804001439E6
:1013780089B22822012302F091FF09E0084A0123DB
:1013880003F08AF81E20A521064A012303F084F8F9
:101398001CBD00BF500B00208A9C05089D9C0508B9
:1013A800B99C0508CF9C050837B51E4C2368042B4B
:1013B80005462BDC01A80DF1060103F0F3FABDF890
:1013C8000630BDF804201849042007F0EBFE236816
:1013D800002B04DA1548164A164B592105E0042B50
:1013E80005DD1248124A144B5A2101F0F9FE04EBAC
:1013F8008302BDF8041001339180BDF80610236004
:10140800052BD18008D1201D03F04EFB00230B488B
:101418002360FFF740FF03E028460121FFF770FF34
:101428003EBD00BF500B0020E69C05082B9D05081B
:10143800E5D303084D9D0508649D0508F0100020BC
:1014480037B50B4C204601F06AFA0A4B0A4900935B
:1014580000250120094A0A4B019501F008F929469F
:1014680002462346284603B0BDE8304001F026B9BD
:10147800BC0D002009130008FD1200080313000822
:10148800B11300084FF6FF7070474FF6FF707047B2
:101498001FB54FF6E07002F0FDFE002002F0C4FF19
:1014A8000F2002F0CBFE0021294A2A4C01230A20F2
:1014B80002F0F2FF002002F0C1FE042002F0B4FFA7
:1014C8000A201921244A012302F0E6FF2521234A94
:1014D80001230A2002F0E0FF1F2002F0AFFE0123E3
:1014E8000A2037211E4A02F0D7FF237873B301235D
:1014F8001E2096211B4A02F0CFFF62881A496846CF
:1015080011F0F8FF01231E20A2216A4602F0C4FF51
:10151800A2881649684611F0EDFFAE216A460123FC
:101528001E2002F0B9FF0F2002F088FE6088A18813
:10153800143880B22822002302F0B0FEA188608807
:10154800143989B22822012302F0A8FE1FBD00BF6A
:10155800929D0508680B0020A49D0508C49D0508F8
:10156800E49D0508079E0508199E0508269E05089E
:1015780001B18DE7704713B50DF1060101A803F01D
:10158800C5F9144B01221A705988BDF80420891A2C
:101598000E311C2919460AD89C88BDF80600201A65
:1015A8000E301C2803D899680131996001E00023A6
:1015B8008B60084B9968012905DD00229A601A7032
:1015C800FFF794FE05E05A80BDF806209A80FFF7E1
:1015D8005FFF1CBD680B002037B50B4C204601F09F
:1015E8009EF90A4B0A49009300250120094A0A4B33
:1015F800019501F03CF8294602462346284603B0E7
:10160800BDE8304001F05AB8F01000207915000804
:101618008D140008931400087F15000838B50F4B87
:101628000F4D00241C700F4B1C700F4B4FF0FF32F6
:101638001A600E4B1A680E4B20461A6002F02AFEFA
:101648000C4B1B78022B0CBF0B480C48FFF723FEF2
:101658002C70BDE8384007F05BBA00BF2C41002071
:101668008C4D00206C4000208440002080400020E9
:1016780094400020943A0020600E0020180D0020AD
:1016880010B50B4C204601F04AF9002001462246CD
:1016980000F074FA00200749074A00F0F7FED2214B
:1016A800024623464FF48270BDE8104001F006B8A8
:1016B800DC120020DE9A05082516000810B5064C35
:1016C8004FF6FF71206800F035FA044B206819685E
:1016D800BDE8104000F0DCB9740B00209801002030
:1016E80008B5002002F0D6FD054B1868054B1968AF
:1016F80000F0CEF90448BDE80840FFF7CCBD00BFB4
:10170800740B002094010020A80F002008B5FFF7F3
:10171800D5FF0020014605F043FEBDE8084001F072
:1017280037BB0088A0F5C87080B2092808B505D96C
:101738000748084A084B8F2101F052FD074B1880D3
:10174800074BFF21197005F02BFEBDE80840B5E7EF
:10175800339E0508F7D30308569E0508801300201A
:10176800821300200088A0F5967080B2092808B579
:1017780005D90848084A094B832101F031FD084B77
:101788001880084B0121197005F00AFEBDE80840D1
:1017980094E700BF339E05080CD40308569E05083D
:1017A80080130020821300202DE9F34100243A48D9
:1017B8003A4D01F0B4F8224623464FF6FF713848F7
:1017C8000094019400F07AF904262246234607463D
:1017D8004FF6FF7133480096019400F06FF92346E5
:1017E800286022464FF6FF712E480096019400F0BB
:1017F80065F92D4968602D4A204600F047FE2C49BE
:101808002C4A0646204600F041FE214680463A46CC
:101818002046214B00F052FF2A681F4B2046282102
:1018280000F04CFF3246D2211B4B5A2000F046FFF5
:10183800AA20D2214246184B00F040FF0F254FF452
:10184800967440F2351620461B491C4A00F01EFECD
:1018580001340246782128460F4BA4B2233500F004
:101868002DFFB442ADB2EED10F254FF4C87440F24B
:10187800991620461249134A00F008FE0134024620
:101888009B212846044BA4B2233500F017FFB4422D
:10189800ADB2EED1BDE8FC8138120020740B0020F7
:1018A800879E05084B9A0508939E0508151700089A
:1018B8009C9E0508E9160008A59E05086D170008F6
:1018C800A79E05082B17000808B508B143682BB96F
:1018D8000348044A044B9B2101F082FC586908BD67
:1018E800A99E050820D40308CB9E050808B5FFF774
:1018F800EBFF8068123080B208BD08B5FFF7E4FF3F
:101908004068063080B208BD2DE9F84F0446884685
:10191800FFF7DAFF6689E589074606F1030905F14D
:101928000F0AB8F1000F1FD01F2002F087FC2046D5
:10193800FFF7DCFF83462046FFF7DFFF2946034613
:101948005FFA8BF2F0B202F0ADFC042002F06CFDFD
:101958000B364FF6FF70033502F070FCB0B2A9B237
:101968003A68012302F098FD3D69204641464A46FF
:101978005346A847BDE8F88F13B504460DF1060194
:1019880001A802F0C3FF2046FFF79EFF6389BDF858
:101998000410BDF80620C91AE389D21A0339C368AE
:1019A8000F3A204698471CBDF7B5044614200D464B
:1019B80016461F4611F02CFA089BC7600361064BB8
:1019C8000649074A80E8700000930190054B002003
:1019D80000F04DFEFEBD00BF1119000803190008F4
:1019E800F518000881190008704708B508B1436860
:1019F8002BB90448044A054BAD2101F0F1FB5869A5
:101A080008BD00BFEA9E050838D40308CB9E050828
:101A1800F8B505460E46FFF7E8FF836B04461BB191
:101A280028463146984700E018466F8994F83C30BC
:101A3800ED890EB9034310D0208E02F0FFFB608EB3
:101A480002F012FC94F8350002F0EEFC94F8343001
:101A580038462946224602F01FFD002384F83C3010
:101A6800F8BD08B5FFF7C1FF90F83500BDE808409C
:101A780002F0EFBC38B5FFF7B8FF044611F0C0FD1F
:101A8800054694F8350002F0DFFC684380B238BDA3
:101A980038B50D46FFF7A9FF29462E22044611F056
:101AA800DFFD50B1204629462E2211F02BFE0023DF
:101AB80084F82E30012384F83C3038BD2DE9F743F3
:101AC800074640200E461546984611F0A1F90446EF
:101AD80028B91148114A124B4E2101F081FB114BD4
:101AE800114A12498DE818000020114B00F0BFFD83
:101AF80039468146FFF7CCFF9DF82830268684F8C2
:101B080035300B9B6586A363002384F8348084F802
:101B18003C304846BDE8FE83EA9E050850D40308D9
:101B2800089F0508191A00086B1A00087D1A000892
:101B3800F119000810B50C46FFF757FF012304867A
:101B480080F83C3010BD00BF4FF4A0707047C8202B
:101B580070477047074B1B78022B07B508D1064B17
:101B68001B78022B04D001A80DF1060102F0CEFE6D
:101B78000EBD00BF8C4D00202C41002073B50A4BD0
:101B880006460D461446009300200849084A094BAA
:101B9800019000F06CFD294602462346304602B00B
:101BA800BDE8704000F08ABD5B1B0008511B0008AF
:101BB800571B00085D1B000813B502AB03E90600BC
:101BC800436843B1027C0124082A9C7004D11B6934
:101BD8002146984700E01C4620461CBD30B5002829
:101BE8002BD0058B002425E0036A1A7C012A05D135
:101BF8005B681A888A421BD1187F30BD052A06D136
:101C08005B681A888A4213D193F82C0030BD032AE6
:101C180006D15B681A888A420AD193F8250030BD3C
:101C2800062A05D15B681A888A4201D1D87A30BD64
:101C380001340430AC42D7D3002030BD08B18175DF
:101C480001207047F8B504460D46D0B1E175D0F8CB
:101C580098309847012D0DD12746002606E0F869EF
:101C680000F10802436906CA98470136238B0437F6
:101C78009E42F4D3D4F8983020462946984701204C
:101C8800F8BDF8BDF8B50546084617460E4611F0EA
:101C9800B7FC013FB84234BF04463C463CB1284635
:101CA8003146224611F02EFD00232B55F8BD2C702D
:101CB800F8BDF7B5044600200090019000296CD0CB
:101CC8000E8B68E000F1080351F823301D7C042DC9
:101CD80004D15D682D88954247D0013000F1080392
:101CE80051F823301D7C012D04D15D682D88954263
:101CF8003BD0013000F1080351F823301D7C052D3D
:101D080004D15D682D8895422FD0013000F1080379
:101D180051F823301D7C032D04D15D682D88954230
:101D280023D0013000F1080351F823301D7C022D27
:101D380004D15D682D88954217D0013000F1080361
:101D480051F823301D7C072D04D15D682D8A9542FA
:101D58000BD0013000F1080351F823301D7C062D0B
:101D680008D15D682D88954203D103F1080120460A
:101D780015E0013000F1080351F823502B7C082BA3
:101D880009D16F683F88974204D105F108012046C0
:101D98001A4605E00130B04294D32046694608222D
:101DA80011F0E6FA2046FEBDF8B505460F46164680
:101DB800002830D04388032B2FD0202011F028F89A
:101DC800044600282BD040F80C5B39460C22FFF75C
:101DD80059FF1820E66111F01BF80646B8B1022336
:101DE8000374012363760F4B446063600E4BA3605A
:101DF800002323766B8805EB830201339BB2012B0A
:101E080050606B800CD16A685268137608E02046EF
:101E180011F006F804E0064602E0002600E0064657
:101E28003046F8BDC05304085E50040837B545680D
:101E380002AB03E906003DB3037C0124042B85F8BB
:101E4800314022D1688E02F0F9F995F8300002F09D
:101E5800EBFA95F8343043B9BDF80200BDF8061026
:101E6800AA1C234602F018FB0FE0012B03D10848F7
:101E780040F2395104E0022B07D1054840F24151A4
:101E8800044A054B01F0ACF92C4620463EBD00BF84
:101E98001B9F0508101F0408199F0508F8B504467C
:101EA8000F46164610B3838A0A2B20D0202010F044
:101EB800AFFF0546E8B14460102200F1080039463A
:101EC800FFF7E0FE4FF6FF73A08A2B801F236B807D
:101ED80000232B76831D013080B20128EE6144F87F
:101EE8002350A08207D1A3691876F8BDF8BD002059
:101EF800F8BD0120F8BD0120F8BD2DE9F0411D46CF
:101F08004B1C984280460C4617460CDD95420ADC6D
:101F1800013208F101035B1A521BC8B2D2B29BB25C
:101F2800294602F0BDF9A8F10208BDF81800C4EB73
:101F3800080802F083F901261FFA88F808E0A919B1
:101F4800601C80B289B24246002302F0A7F901362C
:101F58007B1B9E42F3D3BDE8F081F8B5C7B21446A7
:101F680038461E460D4602F09FF9621E92B2384668
:101F7800294602F099F9304602F060F9022606E097
:101F8800A21B92B23846294602F08EF90136A642C3
:101F9800F6D3F8BD70B5044600F11E003C220023BC
:101FA80080B20D4602F07AF91E3DA9B220463C22C5
:101FB8000123BDE8704002F071B970B504460138DC
:101FC8000322002380B20D4602F068F9013DA9B250
:101FD800204603220123BDE8704002F05FB9F7B53F
:101FE800089D2E7BEF7A1C463604AB7A06EB072653
:101FF800F618431A687B06EB00602D180020019044
:10200800121B08462146009501F098FEFEBD30B52A
:10201800456885B004AB03E906007DB101242C7343
:102028006D68BDF80800BDF80A109DF80C209DF8F1
:102038000E300095FFF7D3FF204600E0284605B094
:1020480030BD2DE9F04385B004AB03E906004468D0
:10205800BDF80860BDF80C70002C41D0012384F84D
:10206800263094F825300BB9A26800E06268FFB208
:10207800BDF80A109DF80E30009230463A46FFF738
:10208800AEFF04F10C08022002F0CEF9404611F030
:10209800B7FA054600B1451E0F3F0024153E1FFA4A
:1020A80087F90DE002F0CAF902F0CEF904FB1061DD
:1020B80089B248462022002302F008FA0134E4B22B
:1020C800AC42EFD3002002F0B9F8B8B2B1B2424640
:1020D800012302F0FBF9002002F0A6F9012000E03C
:1020E800204605B0BDE8F0832DE9F04385B004AB88
:1020F80003E906004568BDF80860BDF80C70002DBE
:102108003CD001236B762B7EBDF80A10012B0CBF47
:102118006A68AA689DF80E300092FFB23A463046C7
:10212800FFF75DFF0C35022002F07EF9284611F01A
:1021380067FA0E3F81460024163E1FFA87F80DE025
:1021480002F07CF902F080F904FB106189B2404684
:102158002022002302F0BAF90134E4B24C45EFD949
:10216800002002F06BF8B8B2B1B22A46012302F09F
:10217800ADF9002002F058F9012000E0284605B02A
:10218800BDE8F0832DE9F04F85B00546DDF84090B5
:10219800029148469046039311F032FADDF838A0D0
:1021A800DDF83CB00646294600242F4611E024B14C
:1021B800B4420CBF5B46534600E0039B01F108059F
:1021C800ADB200932846029A4346FFF708FF013450
:1021D8002946B442EBDD002002F030F8022002F07C
:1021E80023F97D1D08F10508A8B21FFA88F14A46AF
:1021F800012305B0BDE8F04F02F04EB970B5406854
:1022080086B006AB03E9060000282ED0012380F82B
:102218002D308668164BF21A534243EB020390F8AE
:102228002C205AB1002B134D134B144A08BF1D46DE
:10223800134B00F11C0418BF13460AE0002B0D4D88
:102248000D4B0E4A18BF1D460D4B00F10C0408BF7C
:102258001346BDF81200BDF81410BDF816200096FC
:1022680001950294FFF78EFF012006B070BD00BFF4
:1022780080280408BC240408622A04089E2604084E
:10228800442C040870B5446886B006AB03E9060020
:1022980004B301236377A668104B227FF11A4B42DF
:1022A80043EB01030AB10BB904E01BB966680C4D96
:1022B8000C4B01E00C4D0D4BBDF81200BDF814108D
:1022C800BDF8162000960C3401950294FFF75AFFCA
:1022D800012000E0204606B070BD00BFCC330408E2
:1022E80008300408EA310408AE35040890370408B9
:1022F8002DE9F04385B004AB03E906004468BDF856
:102308000860BDF80A90BDF80C50BDF80E80002C8E
:1023180000F08C800123A3740220676802F084F81F
:102328004FF6FF7001F0A0FF002001F087FFEDB22B
:102338005FFA88F8A6F1160189B230462A46434664
:102348000097FFF74CFE277A002F2ED1A28A23464A
:1023580000E00137974204D29969097E04330029C5
:10236800F7D002F06BF802F06FF8A9F116091FFA1E
:1023780089F90E2101FB10914FF6FF7208F101084F
:102388005FFA88F389B2009248462A46FFF7B5FDFE
:10239800022002F049F81F2001F050FFA38A002B09
:1023A80038D0103DE8B2303E2CE0E3685C68A28A81
:1023B8002346013A002700E00137974204D2996981
:1023C800097E04330029F7D002F038F802F03CF80F
:1023D8000E2101FB10914FF6FF7208F101085FFA18
:1023E80088F389B2009248462A46FFF786FD022004
:1023F80002F01AF81F2001F021FFA38A53B1103D03
:10240800E8B21A3E0637B1B254F827200123083241
:1024180002F05CF8002002F007F84FF6FF7001F0B8
:1024280023FF1F2001F00AFF012000E0204605B02D
:10243800BDE8F0832DE9F04105463620884614466C
:102448001F4610F0E5FC0646E0B120F8025B414665
:102458002E22FFF717FCBDF8183086F83440738633
:102468001820012386F8307086F8313010F0D0FC3F
:10247800044618B104234660037404E0304610F0A3
:10248800CFFC00E004462046BDE8F081F8B50646DA
:1024980024200F46154610F0BBFC0446D8B10F4B5C
:1024A800068083600E4B39464360102200F10C0011
:1024B800FFF7E8FB012600231820256223776677BB
:1024C80010F0A6FC054610B14460067404E02046EE
:1024D80010F0A6FC00E005462846F8BDCC330408F9
:1024E800262E0408F8B506462C200F46154610F08F
:1024F8008FFC0446E8B120F80C6B39461922FFF727
:10250800C1FB0D4BA562A3600C4B6360002384F8EC
:1025180025301820012384F8263010F079FC054670
:1025280018B103234460037404E0204610F078FCDB
:1025380000E005462846F8BDFC4C04089A49040802
:1025480010B50446142010F063FC20B1002343802A
:10255800014B0480036110BDB11D000838B5054664
:10256800442010F055FC0446C0B10E4B0582436070
:102578000D4B0360012383740023037283820B4B8A
:102588000364182010F044FC054618B10723446082
:10259800037404E0204610F043FC00E0054628469A
:1025A80038BD00BF9045040886410408A51E0008F0
:1025B8002DE9F04105463420884614461F4610F0A0
:1025C80027FC064620B3144B05808360134B414615
:1025D8004360102200F10C00FFF754FB214606F17E
:1025E8001C001022FFF74EFB002386F82C30182021
:1025F8000123376386F82D3010F00AFC044618B121
:1026080005234660037404E0304610F009FC00E03E
:1026180004462046BDE8F08180280408DA22040830
:102628002DE9F041044614200D461646984610F050
:10263800EFFB0746B8B1069B048003610023C37211
:1026480001234560068180F80A800373182010F082
:10265800DFFB044618B106234760037404E03846DC
:1026680010F0DEFB00E004462046BDE8F0812DE9CD
:10267800F041044618200D461646984610F0C8FB4F
:102688000746B8B101238370069B04800361079B4A
:1026980045608660C0F80C804361182010F0B8FBD4
:1026A800044618B108234760037404E0384610F064
:1026B800B7FB00E004462046BDE8F0812DE9F34170
:1026C80098461B8B1D2B05460C4617464FF00000FD
:1026D80000F2B480B5F5A07F0090019000F2AE80C2
:1026E800F02900F2AB80127CADF80610511EADF84F
:1026F8000250072900F28A80DFE801F045595E049C
:10270800456A14767B684E4A7A611A8893F83430A1
:102718003A80013BDBB2012B7FD8ADF80240ADF81F
:1027280006507AE005F11602ADF8002004F1160211
:10273800ADF8042002AE434A16E903007A6107F1B6
:10274800080282E8030003F10802013348F8227006
:10275800A8F818307B681A8A187A3A8000286CD151
:10276800FFF7FCFE3849436859603849DF600126A5
:10277800163D196002461E72A8B2E1B24346FFF741
:102788009DFF30465AE0012A0CBF314B314B786827
:102798007B6130F80C3B3B8010F032FF431CDB00C0
:1027A8001A34ED18ADF80440ADF8005035E07B68F8
:1027B800294A1B687A6102E0284A7B687A611B888B
:1027C80014353B80ADF800501434ADF8044024E0D3
:1027D8007B68234A7A611A883A801A899B7AAD18ED
:1027E800ADF80050E418F0E77E681E4B7B61338833
:1027F80038463B8073689847013D4519ADF800504D
:10280800B36838469847013C0419DEE71648174A6A
:10281800174B40F21A3100F0E3FC02AA12E9030058
:1028280007F1080383E80300B8F8183003F1080239
:10283800013348F82270A8F818300120BDE8FC815F
:10284800351E0008F92200087C3D04087239040886
:102858008D22000805220008F12000084B200008FE
:1028680017200008C11B00081B9F0508201F04082B
:10287800199F0508F8B51646002834D01378002BA0
:102888002ED0028B002327E0046A257C042D21D159
:1028980065682F888F421DD195F8313053B16F8EFE
:1028A80001F0F2FC04F1080268866369204606CA52
:1028B80098476F86A81C31462E22FFF7E3F995F852
:1028C80031307BB104F108026369204606CA984793
:1028D8000120F8BD013304309342D5D30020F8BD60
:1028E8001846F8BD0120F8BD70B5B8B1068B04468E
:1028F800002310E0256A287C04280AD16D682888FE
:10290800884206D11046A91C2E22FFF7BBF90120E8
:1029180070BD01330434B342ECD3002070BD38B528
:10292800044620B3134BC361134BC0F89830134BC4
:10293800C0F89C30124B00257822C0F8A03085756D
:10294800C5750583294600F1200010F053FDD4F821
:1029580098302046294698470A4A1388312B07D8C9
:10296800094941F8234001331380012038BD38BD9F
:10297800284638BD4D1C0008451C0008E51B00080A
:10298800BB1C00087C0B0020841300202DE9F041BB
:102998000446002800F0B380078B02460025A8E013
:1029A800136A1E7C042E00F08780012E23D15868FC
:1029B80003888B4240F09B8005F1080710F030FA3D
:1029C80054F827004FF00008C0F8048010F028FAE7
:1029D800228B531E9D4208D00732238354F82210BD
:1029E80044F8271044F8228002E044F82780258321
:1029F8003046BDE8F081052E5ED0032E5CD0022E55
:102A080013D15B68186803888B4270D14388013BF7
:102A18009BB243800BB910F003FA05F1080654F88D
:102A28002630586810F0FCF94EE0072E21D15E6878
:102A3800338A8B425BD1002706E0BB1D013756F86D
:102A4800230010F0EDF9FFB2B38ABB42F5D8002796
:102A5800B78205F1080654F82630586810F0E0F9F6
:102A680054F8260033E044F8267025830120BDE899
:102A7800F081062E1ED1586803888B4237D105F1A4
:102A8800080610F0CDF954F826000027476010F02A
:102A9800C7F9228B531E9D4209D00833013A54F8D6
:102AA8002310228344F8261044F82370DEE744F804
:102AB80026701AE0082E1AD1586803888B4216D15E
:102AC80010F0AEF905F1080654F826000027476013
:102AD80010F0A6F9228B531E9D42C4D0073254F839
:102AE800221044F8261044F822702383BEE70135EB
:102AF8000432BD42FFF454AF0020BDE8F081BDE8C8
:102B0800F08170B5044600282AD0068B751E083659
:102B180000EB86061EE056F8043D1A7C042A13D002
:102B2800012A11D0052A0FD0032A0DD0022A02D17A
:102B38005B681B6809E0072A02D15B68198A05E00F
:102B4800062A01D0082A04D15B6819882046FFF7B5
:102B58001DFF013D681CDED100232383012070BDC9
:102B680070BDF0B528B30023068B1A461EE0046A30
:102B7800257C072D18D16468258A8D4214D1A78A2F
:102B8800002504EB83040DE004EB050C0435DCF8A8
:102B980018C09CF818C0BCF1010F03F1010301D162
:102BA800D8B2F0BDBB42EFD301320430B242DED31B
:102BB8000020F0BD70B508B3048B00231BE0026A47
:102BC800157C072D15D15268158A8D4211D1002325
:102BD800958A11461C46012007E013B9966930769C
:102BE80001E08E69347601330431AB42F5D301201C
:102BF80070BD01330430A342E1D3002070BD2DE93C
:102C0800F04128B30023078B1A461EE0046A257C8E
:102C1800072D18D16468258A8D4214D1B4F814C0E0
:102C2800002504EB83040CE066190435B66996F8B0
:102C38001880B8F1010F03D106F10800BDE8F08152
:102C480001336345F0D301320430BA42DED30020A9
:102C5800BDE8F0812DE9F04700282FD00023B0F817
:102C680018C01D4627E0046A267C072E21D1646817
:102C7800268A8E421DD1B4F81480002604EB8309FD
:102C880015E009EB0604A7693C7E012C0DD192F8EA
:102C980000A0BAF1000F08D007F108001146102271
:102CA800FEF7F0FF2046BDE8F087013304364345C0
:102CB800E7D3013504306545D5D30020BDE8F0875A
:102CC800F0B5B0B1068B002510E0046A277C062F0A
:102CD8000AD1646827888F4206D123819DF8143071
:102CE8006260A3720120F0BD01350430B542ECD317
:102CF8000020F0BD10B500210446FEF7A3FF2046D2
:102D08000121BDE81040FEF79DBF38B598B1048B8E
:102D1800024600230CE0106A058804328D4206D171
:102D280000F10802436906CA9847012038BD0133FB
:102D3800A342F0D3002038BD10B50C460021FEF7A1
:102D480081FF20460121BDE81040FEF77BBF13B587
:102D580002AC04E90C00BDF80230834206D8BDF885
:102D68000030834234BF0020012000E00020BDF87D
:102D780006308B4206D8BDF804308B4234BF0021A0
:102D8800012100E00021002818BF0846C0B21CBD80
:102D980038B5114B114A1988002319E052F8045F1D
:102DA800A87D012812D100240CE004F1080355F88D
:102DB8002300037C082B03D1436800211B69984733
:102DC8000134A4B22B8BA342EFD838BD01339BB298
:102DD8008B42E3D138BD00BF7C0B0020801300205C
:102DE800704770B5094CA5787DB9094B1E78012E3E
:102DF8000BD16368013363606268064B9A4204D959
:102E0800284601F0D3FAA670656070BD7C0B0020DF
:102E18003000002040420F00054A9060134602E04F
:102E280099680139996091680029F9D1704700BF04
:102E38007C0B0020F0B585B001F066FD002800F09D
:102E48004981002502A80DF10A01ADF80850ADF836
:102E58000A5001F05BFD03A80DF10E01ADF80C500E
:102E6800ADF80E5001F09EFDBDF80C10BDF808201D
:102E78000091BDF80E10BDF80A3001912C46964D10
:102E88009649082006F08EF9A878012803D101F0A8
:102E98008DFAAC7019E1924B5B78012B40F01581EB
:102EA800AB78002B40F011816B6029888D4A09E1CD
:102EB80052F8046FB07D012840F002810025FAE045
:102EC80005F10803BDF8080056F82340BDF80A10BC
:102ED80004F108030CCBFFF73AFF002800F0E98063
:102EE800237C013B062B00F29F80DFE803F00429D6
:102EF800159D1F9D4C006668012304F10805337772
:102F080095E80600636920469847002333772046F2
:102F1800636995E8060086E0636893F8252012F156
:102F2800FF3218BF012283F8252077E0636893F801
:102F38002C2012F1FF3218BF012283F82C206DE0FB
:102F48006268137E1568002B6ED16E882F4629465D
:102F5800184606E051F804EFDEF804E001338EF875
:102F68001800B342F6D301231376002607E057F87A
:102F7800040F00F10802436906CA984701366B88B6
:102F88009E42F4D350E0656820892E68A37B227B9B
:102F98000096A0F1160189B2FFF721F81420FFF777
:102FA8003BFF2B7AC3B9AF8A29461A461E4609E069
:102FB800886990F818E00676BEF1010F08BF13463D
:102FC80004310132BA42F3D301220BB9AB6924E0D0
:102FD800053355F8233020E06368DB685A6800231E
:102FE800908A154619461F4609E0AE6996F818E01A
:102FF8003776BEF1010F08BF0B4604350131814217
:10300800F3D3411E8B4203D1053052F8203003E040
:1030180004D2073352F8233001221A7604F1080249
:1030280006CA636920469847237C013B072B4CD886
:10303800DFE803F00410074B0A0D123A63681B6AB5
:1030480034E063689B6A2DE063681B6B2AE0636861
:103058001B6927E0636824E063681A7A7AB9988A5A
:103068001946013800E00132824204D28C69247E7C
:103078000431002CF7D0063253F8223011E0DB6817
:103088005A68908A11460138002300E001338342D0
:1030980004D28C69247E0431002CF7D0063352F810
:1030A8002330DB69984710E06368DB68204698475F
:1030B8000BE00135ADB2338BAB423FF601AF04E014
:1030C80001339BB28B427FF4F3AE01F063FC0F2017
:1030D800FFF7A2FE05B0F0BD7C0B0020419F05085C
:1030E8003000002080130020034B9A6812B19A68C0
:1030F800013A9A60704700BF7C0B00202DE9F34726
:103108000120DFF8D080DFF8D09001460AF072F98C
:103118000025012403234FF48076022740466946A0
:103128008DF8053000968DF804708DF806508DF8EE
:10313800074009F0B7FD40460821224609F032FE53
:10314800234BDFF898801A6844F2A243B2FBF3FAE3
:103158000AF1FF3A204621461FFA8AFA0AF07AF95C
:10316800C8F804A048464146A8F80050A8F80250FC
:10317800A8F8085088F80A500AF008FD7023A8F843
:103188000C300423A8F810300AF1FF3A63236422B4
:1031980003FB0AF3B3FBF2F39BB2C8F8143008F14F
:1031A8000C014846A8F80E40A8F81870A8F81A505C
:1031B800A8F81C60A8F81E500AF006FE48462146EA
:1031C8000AF079FD484621460BF07FF8BDE8FC87F8
:1031D800A401002000000240000001408C0B0020E8
:1031E80083B50E460746154910201C46154605F0BE
:1031F800D9FF1020124905F0D5FF1020114905F01C
:10320800D1FF10200E4905F0CDFF002310200E49F4
:10321800019305F0C7FF334610200C493A4605F0E4
:10322800C1FF10200A492A4605F0BCFF10200949B1
:10323800224605F0B7FF019B0133E7E77B9F0508AE
:10324800809F0508A09F0508B09F0508C09F050836
:10325800D59F0508E69F050808B5164B1A6A01327E
:103268001A621A6A012A1A4603D013484FF4A07149
:103278000FE05862194602E04B6A013B4B62506A04
:103288000C4B0028F8D11A6A012A06D00A4840F2E5
:103298004B110A4A0A4BFFF7A3FF1A6A013A1A624E
:1032A8001B6A2BB10448054A064B40F24D11F2E760
:1032B80008BD00BF8C0B0020F79F050822570408A3
:1032C80021A0050832A005080C4B0D491A6844F2E4
:1032D800A2436428B2FBF3F3D4BF20EAE070642071
:1032E800013B9BB24B60013B58436422B0FBF2F0B8
:1032F80080B2486103480C310AF0E9BCA4010020FF
:103308008C0B00200000014010B5134B93F82820C7
:103318002AB11248124A134B4FF40A710EE00122E7
:1033280083F8282066234FF0C042013BDBB21080AF
:1033380033B90A480A4A0C4B40F23221FFF750FFD2
:103348001488A4B28442F0D1084B1980024B0022A1
:1033580083F8282010BD00BF8C0B0020F79F0508BC
:103368002C57040843A00508199F050800000260AF
:1033780010B5FFF7C3FE6420FFF7A6FFE5204FF462
:103388000041FFF7C1FF00200121FFF7BDFF012029
:103398004FF48071FFF7B8FF02204FF4E061FFF7A8
:1033A800B3FF032041F23001FFF7AEFF04200021F4
:1033B800FFF7AAFF082040F20221FFF7A5FF092026
:1033C8000021FFF7A1FF0A200021FFF79DFF0C2035
:1033D8000021FFF799FF0D200021FFF795FF0F202F
:1033E8000021FFF791FF10200021FFF78DFF11202A
:1033F8000021FFF789FF12200021FFF785FF132026
:103408000021FFF781FF102041F2B071FFF77CFF28
:1034180037211120FFF778FF3220FFF71DFF122018
:1034280040F23B11FFF770FF3220FFF715FF132022
:103438004FF4C051FFF768FF0F212920FFF764FF01
:103448003220FFF709FF20200021FFF75DFF212030
:103458000021FFF759FF30200021FFF755FF3120E9
:103468000721FFF751FF322040F20311FFF74CFF0D
:10347800352040F20741FFF747FF40F20444362069
:1034880040F60F11FFF740FF37202146FFF73CFFBA
:1034980038204FF48061FFF737FF39202146FFF7C6
:1034A80033FF3C200021FFF72FFF3D204FF48061C0
:1034B800FFF72AFF50200021FFF726FFEF215120B8
:1034C800FFF722FF52200021FFF71EFF532040F292
:1034D8003F11FFF719FF60204FF41C51FFF714FF4D
:1034E80061200121FFF710FF6A200021FFF70CFF80
:1034F80080200021FFF708FF81200021FFF704FF4B
:1035080082200021FFF700FF83200021FFF7FCFE47
:1035180084200021FFF7F8FE85200021FFF7F4FE44
:1035280090201021FFF7F0FE92200021FFF7ECFE1B
:1035380093200321FFF7E8FE95204FF48871FFF7E9
:10354800E3FE97200021FFF7DFFE98200021FFF718
:10355800DBFE072040F27311BDE81040D4E610B539
:10356800FFF7CCFD6420FFF7AFFE21210720FFF70E
:10357800CBFE3220FFF770FE01210020FFF7C4FECA
:103588003220FFF769FE23210720FFF7BDFE322016
:10359800FFF762FE00211020FFF7B6FE41F28830E7
:1035A800FFF75AFE33210720FFF7AEFE3220FFF760
:1035B80053FE112046F63001FFF7A6FE3220FFF732
:1035C8004BFE4FF4C0610220FFF79EFE3220FFF74A
:1035D80043FE122046F6EB41FFF796FE3220FFF736
:1035E8003BFE03204AF6A401FFF78EFE3220FFF7C8
:1035F80033FE00210C20FFF787FE3220FFF72CFE58
:103608000D2040F60C01FFF77FFE3220FFF724FE65
:103618000E204FF42C51FFF777FE3220FFF71CFEE7
:10362800B0211E20FFF770FE3220FFF715FE0120A3
:1036380042F63F31FFF768FE3220FFF70DFE052006
:103648000021FFF761FE3220FFF706FE0021062069
:10365800FFF75AFE3220FFF7FFFD16204EF61C71C9
:10366800FFF752FE3220FFF7F7FD172040F2031153
:10367800FFF74AFE3220FFF7EFFD00210B20FFF78E
:1036880043FE3220FFF7E8FD00210F20FFF73CFE44
:103698003220FFF7E1FD41200021FFF735FE3220FF
:1036A800FFF7DAFD42200021FFF72EFE3220FFF758
:1036B800D3FD00214820FFF727FE40F23F143220B7
:1036C800FFF7CAFD21464920FFF71EFE3220FFF70B
:1036D800C3FD00214A20FFF717FE3220FFF7BCFD8B
:1036E80000214B20FFF710FE3220FFF7B5FD4420E4
:1036F8004FF46F41FFF708FE3220FFF7ADFD0021C0
:103708004520FFF701FE3220FFF7A6FD214646209F
:10371800FFF7FAFD3220FFF79FFD302040F20771D6
:10372800FFF7F2FD3220FFF797FD31204FF40171CA
:10373800FFF7EAFD3220FFF78FFD32204FF40171C9
:10374800FFF7E2FD40F202543220FFF785FD2146E3
:103758003320FFF7D9FD3220FFF77EFD342040F2F9
:103768000751FFF7D1FD3220FFF776FD35204FF4E2
:103778000171FFF7C9FD3220FFF76EFD36204FF4C7
:103788000171FFF7C1FD3220FFF766FD21463720A2
:10379800FFF7BAFDA4F500743220FFF75DFD21465E
:1037A8003A20FFF7B1FD3220FFF756FD2F2041F2F6
:1037B800BE21FFF7A9FD3220FFF74EFD21463B2031
:1037C800FFF7A2FD3220FFF747FD00212320FFF776
:1037D8009BFD3220FFF740FD00212420FFF794FDD8
:1037E8003220FFF739FD25204FF40041FFF78CFD0B
:1037F8003220FFF731FD00214F20FFF785FD3220F1
:10380800FFF72AFD4E200021FFF77EFD3220BDE89C
:10381800104021E508B5124B93F829202AB1114828
:10382800114A124B40F242210FE0012283F829206D
:10383800222166234FF0C042013BDBB2118033B92D
:103848000848094A0A4B40F25B21FFF7C9FC108877
:1038580080B22228F0D1024B002283F8292008BD2B
:103868008C0B0020F79F05083957040843A005086A
:10387800199F050810B5224B49F22032032823D896
:10388800DFE800F0021A0B111C8846F6280041F206
:103898002801944218BF01461AE01C8841F208002A
:1038A80046F6080104E01C8841F2300046F6300173
:1038B800944208BF01460BE0188846F62001904262
:1038C80008BF4FF4815103E00E4840F2792113E01C
:1038D8001B8848F68912934205D049F22032934258
:1038E80007D1032000E01120FFF70EFDBDE81040CE
:1038F80090E7044840F28521034A044BFFF770FC27
:1039080032000020F79F05084E570408199F050844
:10391800014B18800A209FE4000002604FF0C0436A
:10392800188003F500331A881A88188880B27047FF
:103938002DE9F041022098B00121002409F05AFD38
:10394800012502268C48169616A98DF85C508DF82C
:103958005D608DF85E408DF85F4009F0A3F918208E
:10396800294609F047FD2846294609F05BFD21460E
:103978000C22824809F016FA29460C227F4809F0E1
:1039880011FA04210C227D4809F00CFA05210C22B9
:103998007A4809F007FA07210C22784809F002FA58
:1039A80008210C22754809F0FDF909210C227348F9
:1039B80009F0F8F90A2171480C2209F0F3F90B21F2
:1039C8006E480C2209F0EEF90E210C226B4809F022
:1039D800E9F90F210C22694809F0E4F907210C22C2
:1039E800674809F0DFF908210C22654809F0DAF97F
:1039F80009210C22624809F0D5F90A210C226048F5
:103A080009F0D0F90B210C225D4809F0CBF90C2103
:103A18000A465B4809F0C6F90D210C22584809F0FE
:103A2800C1F90E210C22564809F0BCF90C22544861
:103A38000F2109F0B7F903274CF6B3734F481693D3
:103A480016A98DF85C608DF85E408DF85F408DF8A2
:103A58005D7009F027F94FF6807316A94848169348
:103A68008DF85C608DF85E408DF85F408DF85D7074
:103A780009F018F940F6B830FFF7EEFB3146224658
:103A88003D4809F084F944F6FF70FFF7E5FB2A4644
:103A98003146394809F07BF940F6B830FFF7DCFBCE
:103AA8004FF480530F961196099310264FF4002374
:103AB8000DF13C0868460C931094129413951494D5
:103AC800159400940194029404940694079408941D
:103AD8000A9405940B940396CDF8348008F05BFEA5
:103AE8006846109412941395149415940F9711978F
:103AF800CDF8388008F04FFE2946204608F0CBFE66
:103B080040F6B830FFF7A8FB2046FFF707FF04464A
:103B18001C491D4D3046224605F044FB48F68913E2
:103B28009C421AD049F220339C420DD041F289239D
:103B38009C4212D03046154905F034FB1448154A0A
:103B4800154BA621FFF74CFB30461449224605F0D9
:103B580029FB2C80FFF70CFC0AE0FFF700FD48F674
:103B680089122A8010200E4941F2892305F01AFB98
:103B780018B0BDE8F08100BF00040240000C02400C
:103B88000010024058A00508320000206FA0050868
:103B9800F79F050866570408199F0508A6A0050899
:103BA800DBA005084FF0C04322221A8003F500333A
:103BB80082B01A8892B2ADF806201B889BB2ADF885
:103BC8000630BDF8060080B202B07047134B1B8860
:103BD80048F68912934210B504460BD049F22032B8
:103BE800934213D1C1F1EF01202089B2FFF78CFB7A
:103BF800212006E0C1F1EF014E2089B2FFF784FBD6
:103C08004F202146BDE81040FFF77EBB0448054A17
:103C1800054B40F2F321FFF7E3FA00BF3200002022
:103C2800F79F05086F570408199F05082DE9F0410B
:103C38000D46C5F1F008411E5E18C2EB0802C5F139
:103C4800EF039BB292B2B6B29A422CBF9046984606
:103C58009A4234BF11461946864234BF3746074652
:103C680040F23F13864238BF06469E4228BF1E4692
:103C78001B4B1B8848F68912B8F1EF0F28BF4FF08D
:103C8800EF089342044610D049F2203293421FD1E4
:103C98005020FFF739FB51204146FFF735FB5220F2
:103CA8003946FFF731FB53200AE041EA082189B27F
:103CB8004420FFF729FB45203946FFF725FB46201E
:103CC8003146FFF721FB20462946BDE8F0417DE754
:103CD8000448054A054B40F2DD21FFF781FA00BF91
:103CE80032000020F79F05087D570408199F050832
:103CF80000200146F0224FF4A07397E7072040F216
:103D08007311FFF701BB07200021FFF7FDBA10B5BB
:103D18001446FFF75BFFFFF77DFD2046BDE8104026
:103D2800F6E508B5FFF752FF4FF0C04322221A808C
:103D380003F500331A88188880B208BDF8B580B238
:103D480002FB03F589B292B29BB2069C9DF81C60F7
:103D5800FFF76CFF0020FFF78DFD002709E034F81E
:103D6800020B1EB1030A43EA002080B2FFF7D0FD20
:103D78000137AF42F3DBBDE8F840B9E72DE9F74F6B
:103D880016469DF834200C9F01920546B2B280B2C7
:103D98000C46984689B29BB2FFF748FF4FF0000BDC
:103DA8000020FFF767FDDA463DE0002D30DB09EB28
:103DB800050340F23F1293422ADC002C28DB0BEB70
:103DC8000403EF2B24DC19F00F0F04D1B9F1000F15
:103DD800C8BF0AF1010A174B09EA0303002B03DAEB
:103DE800013B63F00F030133019A0AB1C3F10F03DA
:103DF800012202FA03F337F81A2013401BB213B159
:103E08000D4B588D01E00D4A508880B2FFF780FDB8
:103E180009F1010901E04FF00009C145C5DB0AF1CC
:103E2800010A0BF1010BB345F5DB03B0BDE8F04F18
:103E38005EE700BF0F0000808C0B002032000020DE
:103E48002DE9F04F85B004469DF83C00029200270A
:103E58008A46039088463E4640F23F1C9B463AE01D
:103E6800002C2FDBE1452DDCBAF1000F2ADBB8F17D
:103E7800EF0F27DC2A0702D1002DC8BF01361B49E6
:103E88002940002903DA013961F00F010131039A51
:103E98000AB1C1F10F010E9830F8162003FA01F1AA
:103EA8000A4012B272B112494A8D019392B21FFAB6
:103EB80089F01FFA88F1CDF800C0FFF728FFDDF878
:103EC80000C0019B013509F101095D45C8DB0136D8
:103ED800013708F10108029A974203DAA146002542
:103EE8000123F2E705B0BDE8F08F00BF0F000080A6
:103EF8008C0B002082B0044BADF80600BDF80620FC
:103F080092B25A8502B070478C0B002082B0044BE5
:103F1800ADF80600BDF8062092B25A8002B070478C
:103F28003200002070B50646FFF7E2FE0020FFF7DA
:103F3800A1FCF02409E0013D3046ADB2FFF7E8FCF2
:103F4800002DF8D1013CA4B214B14FF4A075F2E7EA
:103F580070BD70B51D461446FFF738FE2846FFF7BA
:103F680089FC0025054E05E0708D80B2FFF7D0FC76
:103F78000135ADB2A542F7D170BD00BF8C0B002052
:103F88002DE9F0410C4616461F461A460023054601
:103F9800FFF7DFFF611E711828463A46002389B2F1
:103FA800FFF7D7FF2846214632460123FFF7D1FF06
:103FB800013D7F19B8B2214632460123BDE8F041E0
:103FC800C7E770B580B202FB03F489B292B29BB224
:103FD800FFF72CFE0020FFF74DFC0025054E04E0FE
:103FE800708D80B2FFF794FC0135A542F8DBBDE87F
:103FF80070407DE68C0B0020F8B5561A0C4601314E
:1040080089B21F460546FFF7E1FD0120FFF732FCA4
:104018004FF0C04322221A800E4A0F491388B6B2C5
:10402800002304E01088013321F8020B9BB2B3424D
:10403800F8D121462846FFF7C9FD0120FFF71AFCF1
:10404800002404E03846FFF763FC0134A4B2B4420C
:10405800F8D1F8BD000002608E4D002070B5194BF4
:10406800194AD98D92F9004064180025A4B2AC42CF
:1040780008BF0124C62C28BFC6240F2615704FF68A
:10408800FF7288B09E85DC855A8519200A222B4646
:104098002146FFF75EFF21463046FFF742FE2246E3
:1040A80003460A4968460FF025FA6A4604A80849F3
:1040B8000FF020FA3220D22104AA2B4600F0ECF9A6
:1040C80008B070BD8C0B0020302A00201AA105080A
:1040D80022A105082DE9F0431F2093B0FFF722FF26
:1040E8004FF47840FFF71EFF4FF6E0754FF4FC6081
:1040F800FFF718FF2846FFF715FF0020494CFFF788
:1041080011FF00200146642203464FF6FF79A4F808
:104118002A90FFF71EFF00200A2164220346FFF7BA
:1041280018FF00200146642201234FF47847658573
:10413800FFF70FFF7720EF21C82200234FF4FC661A
:104148006785FFF706FFBD213222012340F23F10A9
:104158006685FFF7FEFEA0203222002378216785BE
:10416800FFF7F7FEA0207821322201234FF01F0825
:104178006685FFF7EEFEA020782132220223A4F8FC
:104188002A80FFF7E6FEA0207821322203236585E6
:10419800FFF7DFFE244B2549A3F8028002AD3C223D
:1041A80028460FF0E5F8EB20C321052230230095BF
:1041B8000025A4F82A900195FFF7E0FD32210A2096
:1041C80096220B466785FFF7DBFE32213C209622BC
:1041D8000B466685FFF7D4FE32210B4696226E20E9
:1041E800A4F82A80FFF7CCFEFFF78DFDFFF786FDC8
:1041F8003220FFF769F82846FFF766F86420FFF7D2
:1042080063F80B4B03F110028DE8240028465A6826
:104218001B682946FFF792FD1195119B01331193F5
:10422800FBE700BF8C0B00203200002092570408E7
:10423800B07B0108004870475014002082B0064B3C
:10424800ADF80600BDF8062092B21A80188880B230
:1042580002B0FFF74FBE00BF4C140020014B188876
:1042680080B270474C14002082B0064BADF80600AF
:10427800BDF8062092B21A80188880B202B0FFF703
:1042880045BE00BF4E140020014B188880B270470D
:104298004E140020FFF746BEFFF7C8BCFFF759BE13
:1042A800FFF76EBEFFF78DBE2DE9F04F4FEA4208CB
:1042B80000253D4C85B082468B46C8F10308174659
:1042C8002E461FFA87F909EB0B0C228805EB0A0327
:1042D8001FFA8CFC9BB26146184692B2CDF804C016
:1042E8000293FFF714FDC9EB0B0292B20392029BF3
:1042F80022880399184692B2FFF709FDDDF804C039
:104308002288C5EB0A039BB26146184692B2029313
:10431800FFF7FDFC029B22880399184692B2FFF72B
:10432800F6FC05EB0B0292B2039209EB0A03228812
:1043380003999BB2184692B20293FFF7E8FC029BDE
:104348002288C5EB0B0C1FFA8CFC1846614692B20A
:10435800CDF804C0C9EB0A09FFF7D9FC22880399F4
:104368001FFA89F992B24846FFF7D1FC2288DDF896
:1043780004C092B248466146FFF7C9FCB8F1000F85
:1043880004DA08EB860808F1060805E0F31B08F1D3
:104398000A0808EB8308013F01360135BE42ADB279
:1043A8008FD905B0BDE8F08F4C14002008B9FFF78D
:1043B800AABC012801D1FFF7A1BC704770470020B3
:1043C8000146F0224FF4A073FFF730BC704708B5E0
:1043D80005280CD8DFE800F012140305070909487E
:1043E80008BD094808BD094808BD094808BD09486D
:1043F800094A0A4B40F24111FEF7F2FE084808BD8F
:10440800084808BD200000201000002008000020F7
:104418000000002027A10508CE570408199F0508A9
:10442800280000201800002010B50446FFF7CFFF31
:10443800014B18601C7110BD38000020014B187921
:10444800704700BF3800002008B5FFF7C0FF80881C
:1044580008BD08B5FFF7BBFFC08808BDF7B51F4604
:104468000B4B0C4E1D681446EA882B68203C5443BD
:10447800A4B2AE1B03EB440418BF0126AB888DE839
:10448800500017B1FFF7DCFC01E0FFF777FCFEBD39
:1044980038000020280000202DE9F0410F469846FA
:1044A80015460446084E08E0204643463946FFF7BD
:1044B800D5FF33689B88E418A4B215F8012B002AAD
:1044C800F2D1BDE8F08100BF3800002010B50446E5
:1044D80008462146BDE81040DEE7094B70B50446A2
:1044E80018790E461546FFF7B4FFC6F1F001091A10
:1044F80089B220462A460023BDE87040CCE700BFB9
:1045080038000020704700BF044B1A680AB9044AF3
:104518001A601A681018186010467047BC0B002003
:10452800F49000204FF0FF30704708B50248034A66
:10453800034B3721FEF754FE46A10508E45704084B
:10454800199F05080120704710B504460A48022142
:1045580009F0D6F90028F9D00748214609F099F959
:104568000548012109F0CCF90028F9D00248BDE836
:10457800104009F08BB900BF0038004010B5194849
:10458800022109F0BDF90028F9D01648002109F0E8
:1045980080F91448012109F0B3F90028F9D011482D
:1045A80009F074F90402A4B2002301E001339BB2BC
:1045B800002BFBD00B48022109F0A2F90028F9D002
:1045C8000848002109F065F90648012109F098F921
:1045D8000028F9D0034809F059F92043C0F3CB006B
:1045E80010BD00BF003800402DE9F0478AB00AAF7F
:1045F8000A20012108F0FEFE4FF4604347F8143DFD
:10460800474EDFF824A1012400254FF00208304668
:1046180039468DF81A508DF818808DF819808DF864
:104628001B4008F03FFB30460D21052208F0BAFB7D
:1046380030460E21052208F0B5FB052230460F2131
:1046480008F0B0FB21464FF4804008F0F7FE5046D2
:1046580008F0D2FF4FF48273ADF802304FF40073C4
:10466800ADF80A303823ADF80C30504607236946B8
:10467800ADF81030ADF80050ADF80450ADF8065064
:10468800ADF80850ADF80E5008F0E8FF5046214646
:1046980009F07FF8A9468DF81A5030464FF4805536
:1046A800394605958DF818408DF819808DF81B400E
:1046B80008F0F8FA3046294608F065FB40253946E7
:1046C80018488DF818908DF819808DF81A908DF883
:1046D8001B40059508F0E6FA21464FF4804008F0A3
:1046E800B9FE0621032009F043F90C2307A88DF829
:1046F800213007958DF820908DF8224007F0C6FFED
:1047080017238DF8243009A80F238DF825308DF84C
:1047180026308DF8274004F0D3FE0AB0BDE8F087B4
:1047280000040240000C024000380040014B187899
:10473800704700BFC00B0020024B5A889B8802803C
:104748000B807047C00B0020014B00221A70704785
:10475800C00B0020F0B593B06846002148220EF047
:1047680049FE6D46002464484FF4805108F00DFB63
:10477800002301E001339BB2002BFBD09020FFF710
:10478800E3FE002301E001339BB2002BFBD0FFF7CF
:10479800F5FE4FF480510746574808F0F4FA002315
:1047A80001E001339BB2002BFBD053484FF48051FA
:1047B80008F0EBFA002301E001339BB2002BFBD099
:1047C800D020FFF7C1FE002301E001339BB2002B8C
:1047D800FBD0FFF7D3FE4FF480510646464808F059
:1047E800D2FA45F8047B01342E6244484021E4B2F1
:1047F80008F0B7FA10B9092CB5D101E0092C78D125
:104808009DE80C00D218029B03980699D218049BC5
:10481800C018059BC018079BCB180899032490FB68
:10482800F4F092FBF4F25B1893FBF4F3151AC11A37
:104838009C1A002DB8BF6D420029B8BF4942002C10
:10484800B8BF6442502D03DD502909DD502C50DCDF
:104858008D4205DAAC424FF0020405DB111806E080
:104868008C424FF0020401DAD11800E0C1180A9B0B
:10487800099A0C980F9DD2180B9BD2180D9BC01843
:104888000E9BC018109BEB18119D91FBF4F10324AB
:1048980092FBF4F290FBF4F05B1993FBF4F3161A15
:1048A800C41A9D1A002EB8BF7642002CB8BF6442C5
:1048B800002DB8BF6D42502E89B203DD502C09DDA2
:1048C800502D16DCA64205DAB5424FF0020405DB8E
:1048D800131806E0A5424FF0020401DAD31800E0ED
:1048E800C318074A93FBF4F39BB2938001235180CA
:1048F800137013B0F0BD00BF00040240000C02406A
:10490800C00B002000000000FFF710BFF7B50546F8
:104918000C4601A80DF10601FFF70EFF1B4BBDF871
:104928000660BDF8040093E80600724301FB00220C
:1049380099685218164992FBF1F207EE102AF8EE20
:10494800C77A40F23F17FCEEE77A17EE902A92B248
:10495800B2F5207F28BF3A462A801D69DA685B696C
:104968006E4302FB0060C01890FBF1F107EE101ACD
:10497800F8EEC77AFCEEE77A17EE903A9BB2B3F5F9
:10498800F07F28BFEF232380FEBD00BFC80B0020A7
:1049980040420F00FFF7D8BE014B187E704700BF9A
:1049A800C80B0020FFF7C8BE042808B505D907487A
:1049B800074A084B7D21FEF713FC054B03EB8000EB
:1049C800038B0B80438B138008BD00BF67A10508CC
:1049D800EA57040885A1050808B5082001F090F9F0
:1049E80042F69643C31A584240EB030008BD10B57F
:1049F8000A2001F0ADF90C4C20600E2001F0A8F956
:104A08006060122001F0A4F9A060162001F0A0F95E
:104A1800E0601A2001F09CF920611E2001F098F94D
:104A280001236061237610BDC80B002010B5FFF785
:104A3800DBFD01F02FFA044601F038FA0749034676
:104A48002246202004F0AEFBFFF7C6FF28B101F094
:104A58003BFA10B9BDE81040C9E710BDC1A105086F
:104A680010B5104C0A20216801F059F961680E2030
:104A780001F055F9A168122001F051F9E1681620FA
:104A880001F04DF921691A2001F049F961691E20E8
:104A980001F045F9082042F69641BDE8104001F0C2
:104AA80021B900BFC80B00202DE9F04F0346A7B07D
:104AB800B0F800C01C898688DF885D89CDF810C0F1
:104AC800B249B0F802C0B3F80C90B3F80E80CDF834
:104AD80024C00FFA84FB30B201220FFA87FE0BEBD9
:104AE800000C0A7629B20FFA89FACDF888C001EBD2
:104AF8000E0C0FFA88F2CDF890C00AEB0B0CCDF82B
:104B080030C002EB010CCDF858C0B3F810C05B8A76
:104B1800CDF800C00FFA8CFC06910CEB00010A914D
:104B280002930CEB0A011BB2239103EB0E010E91C9
:104B380099182591049900FA81F05844504460442A
:104B4800DDF824C006990EFA8CFEDDF810C01FFAB5
:104B580080FB1CFB0CF08E4416FB0600964414FBED
:104B68000400009A19FB09009E4412FB02001FFA78
:104B78008EFA09F0CFFFDDF824C0029ACDE91201C0
:104B88001CFB0CF017FB070015FB050018FB0800C1
:104B980012FB020009F0BEFFDDF824C0029ACDE93D
:104BA800140104991CFB01F317FB063615FB046678
:104BB800009B18FB096612FB036009F0ABFFDDE9F7
:104BC8001423CDE90001DDE912010AF019F80446C1
:104BD8000D46DDE9000102460B460AF011F80246CF
:104BE8000B462046294609F057FECDE918015846DC
:104BF80009F0A0FFCDE91001DDE91023DDE900018E
:104C080009F0FEFFCDE90601504609F093FF804602
:104C180089464246DDE912014B4609F0F1FFDDE91C
:104C28001023CDE91C01DDE9140109F0E9FF002298
:104C380006460F46564BDDE9180109F0E1FF4246EA
:104C480004460D464B46DDE9060109F0D9FF024648
:104C58000B4609F023FE02460B462046294609F07A
:104C68001DFE424604460D464B46DDE91C0109F08F
:104C7800C7FF02460B462046294609F00DFEDDE92E
:104C8800102304460D463046394609F0B9FF02465E
:104C98000B462046294609F0FFFDDDF828C0CDE97E
:104CA80002014FEA8C10DDF830C000EB0C20DDF873
:104CB80010C0A0241CFB040009F02CFFDDF838C04C
:104CC800CDE90A014FEA8C10DDF858C000EB0C2042
:104CD800DDF824C01CFB040009F01CFFCDE90C0121
:104CE800504609F017FFDDE91023CDE91601DDE98B
:104CF8000C0109F085FF4246CDE91E014B46DDE96E
:104D08000A0109F07DFF4246CDE920014B46DDE965
:104D1800000109F075FF32463B4609F0BDFDCDE9BB
:104D28000E01584609F0F6FEDDE91C23CDE91A010B
:104D3800DDE9060109F0B0FDDDF88CC0C024CDE93D
:104D4800060104FB0CF0DDF888C0302505FB0C00DB
:104D5800DDF810C078261CFB060009F0DBFEDDF844
:104D680094C0824604FB0CF0DDF890C005FB0C00F3
:104D7800DDF824C01CFB06008B4609F0CBFEDDE9FC
:104D8800102306460F4609F03BFF03E0C80B00203E
:104D9800000014404246CDE904014B4650465946AE
:104DA80009F02EFFDDE9142380468946DDE90A0172
:104DB80009F026FFDDE9002304460D46DDE90C0174
:104DC80009F01EFF02460B462046294609F064FDFD
:104DD8000022A14B09F014FFDDE9202304460D460B
:104DE800DDE91E0109F058FD02460B46DDE9160112
:104DF80009F006FF02460B462046294609F04EFDFB
:104E0800002204460D46954BDDE90E0109F0F8FE37
:104E180002460B462046294609F040FDDDE90223FB
:104E28000AF018F888A3D3E9002309F0E9FE0AF08C
:104E380081F98B490860DDE91223DDE90C0109F0ED
:104E4800DFFEDDE9002304460D46DDE90A0109F02D
:104E5800D7FE02460B462046294609F01DFD0022D2
:104E68007D4B09F0CDFEDDE91E2304460D46DDE944
:104E7800200109F011FD02460B46DDE91A0109F08F
:104E8800BFFE02460B462046294609F007FD0022D0
:104E980004460D46714BDDE9060109F0B1FE0246F4
:104EA8000B462046294609F0F9FCDDE9022309F002
:104EB800D1FF65A3D3E9002309F0A2FE0AF03AF96D
:104EC800674A5060DDE90E23DDE90A0109F098FE22
:104ED800DDE9062304460D46DDE90C0109F090FEE4
:104EE80002460B462046294609F0D8FC0022044613
:104EF8000D465A4BDDE9180109F082FE02460B46C1
:104F08002046294609F0CAFCDDE9022309F0A2FF80
:104F18004DA3D3E9002309F073FE0AF00BF9504BB7
:104F280059469860DDE91423504609F069FEDDE929
:104F3800002304460D463046394609F061FE024614
:104F48000B462046294609F0A7FC0022424B09F0EF
:104F580057FE424604460D464B46DDE9040109F07A
:104F68009BFC02460B46DDE9160109F049FE0246A4
:104F78000B462046294609F091FC35A3D3E90023C6
:104F880004460D46DDE90E0109F03AFE02460B46DD
:104F98002046294609F082FCDDE9022309F05AFF80
:104FA80029A3D3E9002309F02BFE0AF0C3F8DFF8A0
:104FB800B0C0DDE91223CCF80C003946304609F0C0
:104FC8001FFEDDE9002304460D465046594609F008
:104FD80017FE02460B462046294609F05DFC0022D2
:104FE8001D4B09F00DFEDDE9042304460D4640463D
:104FF800494609F051FC02460B46DDE91A0109F061
:10500800FFFD02460B462046294609F047FC10A33F
:10501800D3E9002304460D46DDE9060109F0F0FD59
:1050280002460B462046294609F038FCDDE90223F2
:1050380009F010FF04A3D3E9002309F0E1FD0AF009
:1050480079F8074908610DE00000000080842E41CE
:105058000000000000C082400000144000008940A9
:10506800C80B0020DDE90E235046594609F0C8FD5B
:10507800DDE9062304460D463046394609F0C0FDF1
:1050880002460B462046294609F008FC11A3D3E93D
:10509800002304460D46DDE9180109F0B1FD02467A
:1050A8000B462046294609F0F9FBDDE9022309F001
:1050B800D1FE0AA3D3E9002309F0A2FD0AF03AF8C9
:1050C800034A506127B0BDE8F04FC9E4AFF3008050
:1050D800C80B00200000000000C082400000000053
:1050E80080842E41AFF30080064B074A596811604F
:1050F8001969064A1160D969054A11609A6A054B0F
:105108001A60704740000020884000203841002085
:105118008C4000204C400020014B1878704700BF9D
:10512800E40B0020032808B505D90548054A064BB5
:105138007121FEF755F80C235843044B185808BD45
:10514800FCA105081658040816A20508400000200E
:10515800032808B505D90648064A074B7621FEF705
:105168003FF8064B0C2202FB0030406808BD00BF28
:10517800FCA105082658040816A2050840000020CE
:10518800034B044A1B780C2101FB032398687047E2
:10519800E40B002040000020034B044A1B780C203D
:1051A80000FB032399607047E40B002040000020B7
:1051B800144B1B78012B10B5134B144C0ED11968E6
:1051C800C82000F0ACFD2168CC2000F0A8FD104BF1
:1051D800D020196800F0A3FDD4200DE01968D8206C
:1051E80000F09DFD2168DC2000F099FD084BE020CF
:1051F800196800F094FDE420064B1968BDE81040DA
:1052080000F08DBD080D00208840002038410020A6
:105218008C4000204C400020144B1B78012B10B50B
:10522800134C0FD1C82000F093FD2060CC2000F073
:105238008FFD104B1860D02000F08AFD0E4B1860CF
:10524800D4200EE0D82000F083FD2060DC2000F0A0
:105258007FFD084B1860E02000F07AFD064B1860CF
:10526800E42000F075FD054B186010BD080D002006
:1052780088400020384100208C4000204C4000200D
:1052880008B502F001FA10B1BDE80840C4E7BDE86E
:10529800084029E70148FBF7FEBF00BF381200208D
:1052A8000148FBF7F8BF00BF381200200148FBF7A0
:1052B800F2BF00BF381200200148FBF7ECBF00BF67
:1052C80038120020032808B505D91448144A154B8C
:1052D8004E21FDF785FF144B1870144B02281870E7
:1052E800134B0FD0032813D0012805D0114A126898
:1052F8001A60BDE80840CDE70F4A12681A60BDE899
:105308000840CDE70D4A12681A60BDE80840CDE7AD
:105318000B4A12681A60BDE80840CDE7FCA10508F1
:105328003758040840A20508E40B00207E400020FE
:1053380098010020900100208C01002088010020A5
:1053480084010020064B07495960C02100221972C8
:105358001E211A70D9601A745A611A76DA61704778
:105368007814002040787D0110B50321FF22C02069
:1053780001F076F81F4C102120608022C02001F037
:105388006FF8112120608022C02001F069F81221F5
:1053980020608022C02001F063F813212060802261
:1053A800C02001F05DF8142120608022C02001F0A7
:1053B80057F8152120608022C02001F051F8802282
:1053C80020601621C02001F04BF82060C020172172
:1053D800802201F045F82060074CC020227AB721CE
:1053E80001F03EF80023237463612376E36101230F
:1053F800237010BD684000207814002038B5C02004
:105408000321FF2201F02CF80B4D00242B19615DBC
:105418005A78C020023401F023F8C82CF6D1B12103
:10542800AC22C02001F01CF8C0200321002201F0AA
:1054380017F8002038BD00BF4B5804082DE9F34782
:1054480006460F4692461D461AB90C1FE4019146BE
:1054580035E005EE902A06EE903AB8EE657AF8EE59
:10546800667AFC01C7EE277AA4F500749FED5C7A92
:1054780067EE877A17EE900A09F06EFB41EC100B85
:105488000BF05AFB59EC108B4946404609F07AFE5E
:1054980024184FEACA1009F03DFBCDE9000128465F
:1054A80009F038FB4B46424609F0AAFB02460B4678
:1054B800DDE9000109F0F0F909F064FE8146002EEB
:1054C80014BF4FF022084FF01A08C5F307224146CF
:1054D800C02000F0C5FF08F10101EAB2C02000F0C9
:1054E800BFFFC4F3014208F10201C02000F0B8FF79
:1054F800C4F3072208F10301C02000F0B1FFE2B2B3
:1055080008F10401C02000F0ABFFC9F3034305F420
:10551800702243EA123208F10501C02000F0A0FF12
:1055280008F10601C9F30722C02000F099FF08F12D
:1055380007015FFA89F2C02000F092FFC020B12174
:10554800A02200F08DFF07EE107A264CF8EEC77AFD
:105558000EBBD4ED015A06EE90AAB8EE657A05EEB8
:10556800905AB8EE666AF8EE656A0123C6EE266AB6
:10557800237477EEA67A67EE277A17EE900A09F079
:10558800EBFA41EC100B0BF0D7FA51EC100B09F0C9
:10559800F9FD606120E005EE90AAD4ED016AB8EE4D
:1055A800656A05EE905AB8EE667AF8EE656A0123E8
:1055B800C6EE266A237677EEA67A67EE277A17EE86
:1055C800900A09F0C9FA41EC100B0BF0B5FA51EC4E
:1055D800100B09F0D7FDE0610020BDE8FC8700BF93
:1055E80000000043781400200022012326E7012848
:1055F80038B50D4604D002280CBF3C242C2400E00A
:1056080034242146C02001F027F805F0070200F0F5
:105618000F0040EA02122146C020BDE8384000F0E1
:105628001FBF2DE9F3470A9C1D4607468A461646C2
:10563800524B01E06D0864089C42FBD82DB906F175
:105648000076043EF601A94634E006EE905AB8EE1C
:10565800667A06EE904AF8EE667AF601C7EE277A81
:10566800A6F500769FED467A67EE877A17EE900AE0
:1056780009F072FA41EC100B0BF05EFA59EC108B42
:105688004946404609F07EFD3618E80109F042FA1D
:10569800CDE90001204609F03DFA4B46424609F0A3
:1056A800AFFA02460B46DDE9000109F0F5F809F00A
:1056B80069FD8146022F9BBF324BDB194FF0000872
:1056C80093F8C880C4F307224146C02000F0C8FE02
:1056D80008F10101E2B2C9B2C02000F0C1FE08F130
:1056E8000201C9B2C6F30142C02000F0B9FE08F1B8
:1056F8000301C9B2C6F30722C02000F0B1FE08F1C9
:105708000401C9B2F2B2C02000F0AAFE04F4702469
:10571800C9F3034308F1050143EA1432C9B2C020B2
:1057280000F09EFE08F10601C9B2C9F30722C020A5
:1057380008F1070800F094FE5FFA89F25FFA88F131
:10574800C02000F08DFEBAF1010F0CBF2F220F22EE
:105758000DB942F04002012F06D002D3022F0AD120
:1057680005E0C020102104E0C020112101E0C02084
:10577800122100F075FE0020BDE8FC87FFFF0F0036
:10578800000000434B58040807B501230093002389
:10579800FFF747FF0EBD00280CBFFF22002208B507
:1057A800C020032100F05CFE002008BD08B5C02021
:1057B800B121AC2200F054FE002008BD704708B5A6
:1057C80000F050F900F050F9014B00221A7008BDA2
:1057D800E80B0020024B187880F00100704700BFEA
:1057E800E80B0020014B1878704700BFE80B002039
:1057F80008B54FF400710F4807F0B3FA0E4BD0F11B
:1058080001005A7838BF0020824201460ED05A68FB
:105818001D2A0DDC01321E2A5A6009D1587007482A
:1058280000225A60BDE8084003F0C6BD00225A6055
:1058380008BD00BF00080240E80B00209CA2050834
:10584800014B5878704700BFE80B002010B50021C5
:1058580004460122302000F003FEC0B9012001F007
:10586800A1F8002CB8BF4034E4B210212246302001
:1058780000F0F6FD012001F095F8302011212246B4
:1058880000F0EEFD0120BDE8104001F08BB810BD1E
:1058980010B5002104460122302000F0E1FDC0B916
:1058A800012001F07FF8002CB8BF4034E4B2122187
:1058B8002246302000F0D4FD012001F073F830209A
:1058C8001321224600F0CCFD0120BDE8104001F074
:1058D80069B810BD002810B5044603DB5F2CA8BFCB
:1058E8005F2400E0002430200021012200F0B8FDF0
:1058F800A8B90120E4B201F055F83B212246302036
:1059080000F0AEFD012001F04DF830203C21224688
:1059180000F0A6FD0120BDE8104001F043B810BD1D
:10592800302810B504460ADC10F17F0F02DB00288E
:1059380002DB05E06FF07E0404F5807400E030249B
:10594800002130200A4600F08BFDA8B90120E4B2FE
:1059580001F028F841212246302000F081FD012085
:1059680001F020F830204221224600F079FD012084
:10597800BDE8104001F016B810BD282810B504463F
:1059880009DC10F1180F02DB002802DB04E06FF0DD
:1059980017047F3400E02824002130200A4600F054
:1059A8005FFDA8B90120E4B200F0FCFF53212246B4
:1059B800302000F055FD012000F0F4FF3020542184
:1059C800224600F04DFD0120BDE8104000F0EABF7E
:1059D80010BD08B530200021012200F041FD60B95A
:1059E800012000F0DFFF30203321402200F038FD95
:1059F8000120BDE8084000F0D5BF08BD10B5302033
:105A08000021012200F02CFD044660B9012000F0BD
:105A1800C9FF30203321224600F022FD0120BDE8D5
:105A2800104000F0BFBF10BD10B53020002101228A
:105A380000F016FD0446A0B9012000F0B3FF3421A0
:105A48002246302000F00CFD012000F0ABFF302092
:105A58003721224600F004FD0120BDE8104000F087
:105A6800A1BF10BD4020F1E6402011E708B5002194
:105A78000122302000F0F4FC012000F093FF3020D8
:105A88003421024600F0ECFC012000F08BFF3020AE
:105A98003721024600F0E4FC0120BDE8084000F090
:105AA80081BF08B500210122302000F0D9FC012077
:105AB80000F078FF302034210C2200F0D1FC0120C6
:105AC800BDE8084000F06EBF704770477047194B3B
:105AD8001949D3ED006A93ED017A00231A469FED28
:105AE800176A03E0F0EE476AB0EE677A505E05EE9B
:105AF800900AF8EEE57A0133C7EE867A9BB218B2BF
:105B080004327F2877EEE67AECDD27EE077A07EE97
:105B1800A77A0B49074A0B80BDEEC77A00231360AA
:105B28005360C2ED027A17EE102A064B92001A60F3
:105B3800704700BFF00B0020302600200000FA4517
:105B4800603A0020041700202DE9F84F2E4B2F4A09
:105B580019682F4B19B92F4911602F4A02E02F49B4
:105B680011602F4A1A602F4BDFF8BCA0DFF8BC90F9
:105B7800DFF8BCB000221A80244A9846176830E043
:105B880007EB84036500B3F9023007EE103AF8EE2C
:105B9800C77A013617EE900A08F0DEFF18A3D3E99A
:105BA800002309F02DF809F0C5FA29F815002AF89C
:105BB800140037F9243007EE103AF8EEC77A0135A9
:105BC80017EE900A08F0C8FF0DA3D3E9002309F0E7
:105BD80017F809F0AFFA2BF8140029F81500A8F8FF
:105BE8000060B8F8006034B2FF2CC9DD00F05EF840
:105BF80000F06AF801F0C0F8BDE8F84F67E700BFA9
:105C08009A9999999999E93FF8160020EC1600207D
:105C180028150020322E0020322A0020323600209B
:105C280032320020603A0020302200203026002046
:105C38003024002010B50B4C204606F080FC0A4B9F
:105C480018600A4806F07BFC094B1860FFF77CFFD8
:105C5800084B0949012220469A81BDE8104006F008
:105C6800EFBC00BF10600240F816002088600240B8
:105C78000C170020F00B002020800010014B186842
:105C8800704700BF0417002008B5054B0548198860
:105C98000022012309F042FF034B187008BD00BF22
:105CA8007000002018220020341D002003480449F9
:105CB800044A4FF4807309F0A9BF00BF74000020A4
:105CC800302200201620002003480449044A4FF4DB
:105CD800807309F09BBF00BF8000002030240020A3
:105CE8005018002038B505460C460135C1F3072188
:105CF80000F066FEA8B2E1B200F062FE00B238BD64
:105D080038B5044600F070FD01340546A0B200F035
:105D18006BFDEDB2C0B240EA052000B238BD37B520
:105D28000B0E8DF804300B0C8DF805300B0A8DF82E
:105D380006308DF80710002400E0284601AB451C0A
:105D4800E15C013400F03CFE042CADB2F5D13EBD5F
:105D580037B5002400E02846451C00F045FD01AB9E
:105D6800ADB2E0540134042CF5D19DF805009DF83E
:105D78000430000440EA03609DF8073018439DF89A
:105D8800063040EA03203EBD38B50446642000F0E2
:105D980009FE25786068AD00EDB2257006F0E7FFD2
:105DA800237A40FA03F000F003000543104B2570F6
:105DB80005F00F055A5D6378D218D2B2D3B201321A
:105DC800D2B2022A637001D80022A2705BB2012B02
:105DD80003DD0123A3700023637094F901300133BC
:105DE80003DAFF23A3700023637094F9020038BD1F
:105DF8001C590408F7B504200121234F07F0FAFACB
:105E080002AD01214FF48040012407F023FB002656
:105E18004FF4B0733846694645F8083D8DF804607C
:105E28008DF8074006F03EFF1020214607F0E2FA01
:105E380078236946154800938DF804608DF807406B
:105E480006F030FF0420214607F0D4FA21464FF42B
:105E5800804007F0FFFA1E233846694600938DF804
:105E680004608DF8074006F01DFF0220214607F068
:105E7800C1FAB02306488DF8046069468DF80740DA
:105E8800009306F00FFFFEBD00080240001002401C
:105E980000040240802108B5034806F062FFD0F1F3
:105EA800010038BF002008BD0004024008B54FF4C7
:105EB8008071044806F055FFD0F1010038BF00207A
:105EC80008BD00BF0008024008B5FFF7E3FF08B1AE
:105ED800FFF7ECFFC0B208BD10B5642000F062FD0A
:105EE8000F48FFF751FF044610B90E4B187009E030
:105EF800FFF7DCFF30B9002C0A4B01DD012200E07E
:105F0800FF221A700848FFF73FFF0028074B01D10E
:105F1800187010BD01DD012200E0FF221A7010BDCB
:105F2800C000002090400020CC000020302A002033
:105F380007B50220012107F05DFA012300938DF8CF
:105F4800043002238DF805300448002369468DF893
:105F580006308DF8073006F0A5FE0EBD000402409D
:105F680010B5084C01210022204606F010FF40F22F
:105F7800FF4000F017FD012120460A46BDE8104009
:105F880006F005BF0004024008B5FFF7E9FF00214D
:105F98000A46302000F064FA012000F003FD0121D8
:105FA8000A46302000F05CFA012000F0FBFC0021DA
:105FB8000122302000F054FA012000F0F3FC012106
:105FC8000822302000F04CFA012000F0EBFC0221FE
:105FD8000122302000F044FA012000F0E3FC002107
:105FE8000A46302000F03CFA012000F0DBFC1B21BF
:105FF800CD22302000F034FA012000F0D3FC042137
:106008000322302000F02CFA012000F0CBFC0621FE
:106018000822302000F024FA012000F0C3FC0721F8
:106028000A46302000F01CFA012000F0BBFC0821D1
:106038008022302000F014FA012000F0B3FC1E2169
:10604800B022302000F00CFA012000F0ABFC052152
:106058009122302000F004FA012000F0A3FC0D2169
:106068000322302000F0FCF9012000F09BFC0E21F7
:106078000022302000F0F4F9012000F093FC1421F4
:106088008022302000F0ECF9012000F08BFC0B217D
:106098008822302000F0E4F9012000F083FC302051
:1060A8000C21822200F0DCF9012000F07BFC122197
:1060B8008822302000F0D4F9012000F073FC13216D
:1060C8008C22302000F0CCF9012000F06BFC00217C
:1060D8000122302000F0C4F9012000F063FC0C21FB
:1060E8000822302000F0BCF9012000F05BFC0D21F3
:1060F8000822302000F0B4F9012000F053FC0E21F2
:106108000822302000F0ACF9012000F04BFC0F21F0
:106118000822302000F0A4F9012000F043FC0021FF
:106128000A46302000F09CF9012000F03BFC402199
:106138000222302000F094F9012000F033FC002204
:106148004121302000F08CF9012000F02BFC302098
:106158003F21D42200F084F9012000F023FC002123
:106168000122302000F07CF9012000F01BFC1021F6
:106178000F22302000F074F9012000F013FC1121E7
:106188000F22302000F06CF9012000F00BFC1221E6
:106198000022302000F064F9012000F003FC1321F4
:1061A8000022302000F05CF9012000F0FBFB0921FF
:1061B8003C22302000F054F9012000F0F3FB0021CC
:1061C8000122302000F04CF9012000F0EBFB3020D8
:1061D8003421024600F044F9012000F0E3FB3020AE
:1061E8003721024600F03CF9012000F0DBFB3621A4
:1061F8000322302000F034F9012000F0D3FB3921CC
:106208000322302000F02CF9012000F0CBFB3B21C9
:106218003C22302000F024F9012000F0C3FB3C218F
:106228000A46302000F01CF9012000F0BBFB0021D9
:106238000A46302000F014F9012000F0B3FB512188
:10624800C022302000F00CF9012000F0ABFB302018
:106258005221002200F004F90120BDE8084000F0B6
:10626800A1BB00BF2DE9F04F454E464D93B001212B
:106278004FF4001007F0BEF8304606F061F84FF012
:10628800C0630293404B0393404B002404934FF4A4
:1062980000794FF400334FF480684FF400674FF4EF
:1062A800005A4FF4807B304602A90C93019309975A
:1062B800CDF8189005940794CDF82080CDF828A043
:1062C800CDF82CB00D9406F0C7F822463046304978
:1062D80006F01DF93046012106F023F901210A468E
:1062E8004FF0402007F0F4FA284606F029F8294A2A
:1062F800019B0392284A0C9304922846402202A943
:10630800059209970294CDF818900794CDF820804B
:10631800CDF828A0CDF82CB00D9406F09DF82246B3
:1063280028461E4906F0F3F82846012106F0F9F838
:1063380042F2107701220221194807F0C9FA3846BB
:1063480000F030FB3046012106F0C1F80121284653
:1063580006F0BDF8384600F025FB0B238DF84430D5
:1063680011A801238DF845408DF846408DF8473037
:1063780003F0A6F8384600F015FB13B0BDE8F08F1F
:1063880010600240886002400C4000403236002015
:10639800322E00200C3C004032320020322A0020ED
:1063A800003C004002481021012206F007B900BF56
:1063B8001060024013B50220012107F01BF84FF4CA
:1063C80010730E4C009302238DF804308DF80530BD
:1063D80001238DF806302046002369468DF80730E2
:1063E80006F060FC20460621042206F0DBFC20466D
:1063F8000921042206F0D6FC1CBD00BF000402409F
:1064080030B5154D85B001214FF4001007F016F88E
:10641800284606F0DDFC0023ADF804304BF6FF7388
:10642800ADF806303323ADF808304FF48063ADF88B
:106438000A304FF48043ADF80C3004AC074B2846C3
:10644800012144F8103D06F065FD2846694606F02E
:10645800EDFC05B030BD00BF00540040801A0600B6
:1064680073B54FF4961306460D461446019304E09F
:10647800019B5A1E0192002B57D031484FF400312E
:1064880006F060FE0028F3D12D48012106F04EFDEC
:106498004FF48053019304E0019B5A1E0192002B94
:1064A80045D02748274906F038FE0028F4D024486C
:1064B8003146002206F052FD4FF48053019304E068
:1064C800019B5A1E0192002B33D01D481E4906F02D
:1064D80024FE0028F4D01A48294606F0C2FD4FF4DD
:1064E8008053019303E0019B5A1E01921BB3144889
:1064F800164906F012FE0028F5D01148214606F08C
:10650800B0FD4FF49613019303E0019B5A1E0192CC
:106518009BB10B480E4906F015FE0028F5D0084837
:10652800012106F00FFD002008E0012006E002200E
:1065380004E0032002E0042000E005207CBD00BF49
:10654800005400400100030082000700800007009B
:1065580004000010F7B51F464FF4961306460D4683
:106568001446019304E0019B5A1E0192002B5ED051
:1065780034484FF4003106F0E5FD0028F3D13148E6
:10658800012106F0D3FC4FF48053019304E0019BF2
:106598005A1E0192002B4CD02A482B4906F0BDFD0B
:1065A8000028F4D027483146002206F0D7FC4FF4E3
:1065B8008053019304E0019B5A1E0192002B3AD0AC
:1065C8002048224906F0A9FD0028F4D01D48294694
:1065D80006F047FD4FF48053019304E0019B5A1ED7
:1065E8000192002B29D01748194906F096FD00287A
:1065F800F4D000254FF4961610E0615D114806F0BE
:1066080030FD019603E0019B5A1E0192BBB10D4873
:10661800104906F097FD0028F5D00135EBB2BB42D2
:10662800EBD30848012106F08DFC002008E001208A
:1066380006E0022004E0032002E0042000E0052038
:10664800FEBD00BF005400400100030082000700A7
:10665800800007000400001037B54FF49613044675
:106668000D46019305E0019B5A1E0192002B00F094
:106678009B8056484FF4003106F064FD0028F2D1A3
:106688005248012106F052FC4FF48053019305E073
:10669800019B5A1E0192002B00F088804B484C4900
:1066A80006F03BFD0028F3D048482146002206F0BA
:1066B80055FC4FF48053019304E0019B5A1E01924C
:1066C800002B75D04148434906F027FD0028F4D037
:1066D8003E48294606F0C5FC4FF48053019304E078
:1066E800019B5A1E0192002B64D038483A4906F0A3
:1066F80029FD0028F4D03548012106F017FC4FF495
:106708008053019304E0019B5A1E0192002B53D041
:106718002E482F4906F001FD0028F4D02B482146C9
:10672800012206F01BFC4FF48053019304E0019B07
:106738005A1E0192002B41D0244C2849204606F0CD
:1067480001FD0028F3D02046002106F00FFC20466A
:106758000121238B06F0F6FB4FF48053019304E0EC
:10676800019B5A1E0192002B2AD018481C4906F09A
:10677800E9FC0028F4D0154806F075FC4FF4805366
:106788000193124A03E0019B591E0191D3B113886A
:106798009B05F8D4012104460C4806F0E7FB0B489A
:1067A800104906F0E9FC0EE001240CE002240AE09E
:1067B800032408E0042406E0052404E0062402E09B
:1067C800072400E0082420463EBD00BF00540040D6
:1067D80001000300820007000400001002000010FE
:1067E800400000100004001013B54FF4961304463F
:1067F800019305E0019B5A1E0192002B00F0B08026
:1068080061484FF4003106F09DFC0028F2D15E4843
:10681800012106F08BFB4FF48053019305E0019BA7
:106828005A1E0192002B00F09D805748574906F0E8
:1068380074FC0028F3D05448A021002206F08EFBF7
:106848004FF48053019305E0019B5A1E0192002BDF
:1068580000F08A804C484E4906F05FFC0028F3D0CF
:10686800C4F30521484806F0FCFB4FF4805301931C
:1068780004E0019B5A1E0192002B77D042484549FB
:1068880006F060FC0028F4D0E1B23F4806F0E9FBCE
:106898004FF48053019304E0019B5A1E0192002B90
:1068A80066D039483B4906F04DFC0028F4D03648FC
:1068B800012106F03BFB4FF48053019304E0019B58
:1068C8005A1E0192002B55D02F48304906F025FC5E
:1068D8000028F4D02C48A121012206F03FFB4FF4F8
:1068E8008053019304E0019B5A1E0192002B43D070
:1068F800254C2949204606F025FC0028F3D02046DF
:10690800002106F033FB20460121238B06F01AFBF9
:106918004FF48053019304E0019B5A1E0192002B0F
:106928002CD019481D4906F00DFC0028F4D0164853
:1069380006F099FB4FF480530193134A03E0019B3F
:10694800591E0191E3B113889905F8D40121044631
:106958000D4806F00BFB0C48114906F00DFC10E041
:1069680001240EE002240CE003240AE0042408E0D9
:10697800052406E0062404E0072402E0082400E0D9
:10698800092420461CBD00BF00540040010003003C
:1069980082000700040000100200001040000010F0
:1069A8000004001082B0002304E0019B013301932E
:1069B800009B01330093009B8342F6D302B07047DB
:1069C80037B54FF4805304460D46019304E0019B0C
:1069D8005A1E0192002B6ED03D484FF4003106F04C
:1069E800B1FB0028F3D13A48012106F09FFA4FF491
:1069F8008053019304E0019B5A1E0192002B5CD046
:106A08003348344906F089FB0028F4D03048A021E7
:106A1800002206F0A3FA4FF48053019304E0019B8F
:106A28005A1E0192002B4AD029482B4906F075FBC3
:106A38000028F4D0C4F30521254806F012FB4FF4D2
:106A48008053019304E0019B5A1E0192002B38D019
:106A58001F48224906F061FB0028F4D0E1B21C4827
:106A680006F0FFFA4FF48053019303E0019B5A1E8E
:106A7800019243B31648194906F04FFB0028F5D098
:106A88001348294606F0EDFA4FF49613019303E0F4
:106A9800019B5A1E0192C3B10D48114906F052FBE1
:106AA8000028F5D00A48012106F04CFA0D48FFF7F6
:106AB80079FF00200AE0012008E0022006E0032018
:106AC80004E0042002E0052000E006203EBD00BFEF
:106AD8000054004001000300820007008000070006
:106AE80004000010A086010013B50520012106F05E
:106AF80081FC184C4FF4E053009302238DF80430C6
:106B08008DF805302046002369468DF806308DF84B
:106B1800073006F0C7F820460A21062206F042F997
:106B280020460C21062206F03DF9062220460B21BC
:106B3800A4F5006406F036F94FF400432046694690
:106B4800009306F0AFF820460F21062206F02AF936
:106B58001CBD00BF000802401FB50446FFF7E8F956
:106B6800FFF74EFCFFF710FAFFF7BEFF01214FF4C5
:106B7800004006F063FC02940F4C1023ADF802307D
:106B8800204600236946ADF80430ADF80C30ADF866
:106B98000030ADF8063006F080FD69464FF0402021
:106BA80006F04FFE2046012106F0FFFD4FF0402081
:106BB800012106F0FAFD1FBD003C0040014B1860A2
:106BC800704700BF0C0C0020704710B50A4A1379B3
:106BD800262B04D80949C8540133137110BD074A3C
:106BE8000123591ED45C0133272B5454F9D1034B8C
:106BF80083F8260010BD00BF0C0C0020343A00209A
:106C0800704710B504462078FFF7DFFF14F8013FFE
:106C1800002BF8D110BD38B504460D46013D14F8D7
:106C2800010BEDB2FFF7D1FF002DF7D138BD00BF42
:106C3800014B1878704700BF140C0020014B58789E
:106C4800704700BF140C0020024B187880F0010038
:106C5800704700BF140C0020024B00221A705A70B3
:106C6800704700BF140C0020014B01221A707047B6
:106C7800140C0020014B01225A707047140C00209C
:106C880082B0002304E0019B01330193009B013390
:106C98000093009B8342F6D302B070470148024933
:106CA80004F028BC983A00209840002007B504203A
:106CB800012106F09FFB01214FF4804006F0CAFB3A
:106CC8004FF40073009300238DF804300348012328
:106CD80069468DF8073005F0E5FF0EBD0008024053
:106CE800034A044B1A60044A044B1A60704700BFF9
:106CF8000000FA45B84A0020DB0FC93F904A00203F
:106D0800034B00221A60034A034B1A60E8E700BFEE
:106D1800444100200000FA450816002007EE100A3A
:106D2800024BF8EEC77AC3ED007A704708160020C8
:106D380038B510EE100A07F00FFF0DA3D3E90023B2
:106D480007F05EFF084B044618680D4607F004FF7D
:106D58000B4602462946204608F07CF808F032FA2D
:106D6800024B186038BD00BFB84A0020904A002086
:106D7800182D4454FB2119402DE9F04F2DED068BB9
:106D8800734CDFF800A289B00027A34637F80A50F1
:106D9800704B2580FE5A704B6680186807F0DCFE41
:106DA80069A3D3E9002307F02BFF08F0C3F9636850
:106DB8006A4AC018011101F580610905090D606072
:106DC800C0F30B100DF1200C32F8203032F82120DE
:106DD800616A238115FB02F0628115FB03F516FB3E
:106DE80002F216FB03F60CEB4103E0602561C0F3E9
:106DF800CF30C5F3CF356261A661C2F3CF32C6F397
:106E0800CF3623F8200C23F8105C23F8182C23F82D
:106E1800086C534BA08301310B40002BE58322847F
:106E2800668403DA013B63F003030133CBF82430B3
:106E3800002B7CD14B484C4A6946042309F0A6F93B
:106E48004A484B4A04A9042309F0A0F949484A4A88
:106E580002A9042309F09AF9484A494806A90423D3
:106E680009F094F9B4F9283007EE903AB4F92A30C9
:106E7800B8EEE79A07EE903AB4F92C30B8EEE78A04
:106E880007EE903AB4F92E30F8EEE79A07EE903A0A
:106E9800F8EEE78A68EE087A49EE097A17EE900A62
:106EA80007F05AFE41EC100B09F0D2FF51EC100B21
:106EB80008F088F968EEA87A49EEA97A0AEE100A6D
:106EC800206317EE900A07F047FE41EC100B09F01B
:106ED800BFFF51EC100B08F075F968EE897A58EE8F
:106EE800297A28EE288A0AEE900A606309EE298A30
:106EF80017EE900A07F030FE804618EE100A894611
:106F080007F02AFE49EC108B41EC110B09F018FF31
:106F180051EC100B08F056F98AEE2A0AA06384EDAA
:106F28000F0A01F07DFD94ED0E0A01F089FD02378C
:106F3800B7F5007F7FF42AAF09B0BDEC068BBDE83A
:106F4800F08F00BFAFF3008039D6C56D305FC44005
:106F5800180C002050180020904A002038590408C6
:106F680003000080B4000020400C0020A80000208E
:106F7800420C00209C000020440C0020460C0020FD
:106F88009000002016200020014B93ED0F0A704757
:106F9800180C0020014B93ED0E0A7047180C0020C6
:106FA800014B93ED0C0A7047180C0020014B93ED30
:106FB8000D0A7047180C002010B5FEF7D5F900200F
:106FC800012324210246FEF739FA114B1C780020D0
:106FD800012C05D10146FEF70AFB2046002104E0FA
:106FE8000721FEF704FB01200721FEF700FB6322BF
:106FF8001221C020FFF734FA02200121FEF7F7FA28
:10700800FEF7D4FB0120BDE81040FEF7C4BB00BF6B
:10701800080D00200D4B1B78012B05D10C4B0D4A98
:10702800196812688A181A600B4B1B78012B084BD9
:10703800196805D1094A914207DD01321A60704783
:10704800074A914201DD01321A607047943A0020E4
:1070580094400020903A0020080D00207FD1F008CD
:10706800FF1FA1070E4B1B78012B05D10D4B0E4AB4
:10707800196812688A1A1A600C4B1B78012B094B85
:1070880005D10B4A1968914208DC1A6070471A68E2
:10709800B2F57A2FDCBF4FF47A221A60704700BF2E
:1070A800943A002094400020903A0020080D0020D7
:1070B80040420F00024B1A68024B1A60704700BF2B
:1070C80080400020944000202DE9F04F8246584827
:1070D8008BB0B0FBF1F00C4607F01CFD41EC100B37
:1070E80009F02AFD51EC100B08F04CF8C3070746CD
:1070F80048BF471E04FB07F007F00CFD46A3D3E981
:10710800002307F0A7FE04460D4645EC104B09F096
:1071180013FD59EC108B204642464B46294607F092
:10712800BBFBCDE904014946404608F02BF83CA3D7
:10713800D3E900230990DDE9040107F0DDFF002809
:107148003DD1002401234FF01509224698462046D8
:10715800DFF8E4B003E0234642462C46B04600FB85
:1071680004355D452ED800FB0826DDE904012EA371
:10717800D3E9002307F0C0FF30BBDDE9042300207A
:107188002C4907F067FE41EC100B0390029109F0BF
:10719800D3FC0398029953EC102B8DED060B07F0E6
:1071A8007BFB09F1FF39CDE904015FFA89F9DDE9D3
:1071B800060107F0E7FFB9F1000FCCD104E0012583
:1071C800002601E025464646099BD9B2BAF1000FD0
:1071D8000BD132462B465046FEF730F90123009377
:1071E800504651463A46534609E032462B4601205E
:1071F800FEF724F90120009001463A460023FEF7E5
:1072080010FAFEF7D3FA01200BB0BDE8F04FFEF7F5
:10721800C2BA00BFAFF300800000000084D77741F6
:10722800956479E17FFDA53DBBBDD7D9DF7CDB3D0A
:1072380000E9A4350000F03FFFFF0F001F4B1B784B
:10724800022B10B539D01E4B1E4A19681E4B1F4C15
:107258001B68CB189342236018DC0020FFF734FF2B
:1072680001202168FFF730FF194B1C780020012C02
:1072780005D10146FEF7BBF92046002104E00721AD
:10728800FEF7B5F901200721FEF7B1F9114B1B787C
:10729800022B12D10A4C104B22681B689A420CDA56
:1072A8000E4B1B78012B08D10D4B186800F070F8B5
:1072B8000C4B22681B68D318236010BD8C4D00202E
:1072C8009440002080D1F008304100203441002053
:1072D800080D0020943A0020704000206C400020E7
:1072E8004C400020903A002008B5FEF7D3FD094B2A
:1072F8005A78187002435A701AB19A7801329A7003
:1073080030B99B78034A012B02D90023537093703C
:1073180008BD00BF580C002007B50420012106F065
:1073280069F84FF46043009301238DF80430022379
:107338008DF805300448002369468DF806308DF82D
:10734800073005F0AFFC0EBD00080240084B1A6874
:107358004FF47A73B2FBF3F2064B013A5A60064ACD
:10736800F02182F8231000229A6007221A607047E1
:10737800A401002010E000E000ED00E0034B5A6893
:1073880012B15A68013A5A60704700BF580C002081
:10739800024B58605A68002AFCD17047580C0020EC
:1073A80030B585B004460D4601A85C490A220BF0A9
:1073B800DFFF5B4B1B78032B10D8DFE803F00205D7
:1073C800080B01A8574907E001A8574904E001A89C
:1073D800564901E0564901A80CF0B4F804AA13195B
:1073E80013F80C3C5D19EDB22F2D01D80A3502E0D7
:1073F800392D01D90A3DEDB204AB1C194FF6FF70C7
:1074080004F80C5CFCF71AFF0020FDF70DF80DF1ED
:1074180003050F24204623345A21002315F8012F91
:10742800A4B2FDF71BF8B4F5A57FF3D164205A2167
:107438002C220023FDF712F80023CD205A212C22FC
:10744800FDF70CF80020FCF7F9FE354B1B78032BF1
:1074580062D8DFE803F002284B5601A931480CF046
:1074680071F80A2200212F480CF010FA314A324BE9
:1074780012781860012A06D1304A904201DC0132A4
:107488001A602F4A06E0B0F5FA5FBCBF4FF4FA5213
:107498001A602C4A1B689342C4BF274B1A602A4BB8
:1074A8001A682A4B20E001A91F480CF04BF80A2261
:1074B80000211D480CF0EAF91E4A254B1278186085
:1074C800012A06D11D4A904201DC01321A601C4A89
:1074D80006E0B0F5FA5FBCBF4FF4FA521A60194AD9
:1074E8001B68934218DD1A4B1A6015E001A90F4872
:1074F8000CF028F80D4800210A220CF0C7F9154BAA
:1075080009E001A90A480CF01DF8094800210A22DF
:107518000CF0BCF9104B186005B030BD51A305083C
:107528007E4000205A400020744000201C4100206A
:1075380050400020080D0020884000203F420F00E6
:1075480080D1F00840420F00804000209440002085
:10755800384100208C4000204C40002010B50D4BD5
:107568000D4C1A680D4821460BF0C4FF0C4B0D4812
:107578001A6821460BF0BEFF0B4B0C481A682146CF
:107588000BF0B8FF0A4B0B481A682146BDE81040BB
:107598000BF0B0BF884000205BA305085A400020CC
:1075A80038410020744000208C4000201C410020FD
:1075B8004C4000205040002008B500210A220D4808
:1075C8000CF064F90C4B002118600A220B480CF0EF
:1075D8005DF90B4B002118600A220A480CF056F995
:1075E800094B002118600A2208480CF04FF9084B93
:1075F800186008BD5A4000208840002074400020D0
:10760800384100201C4100208C40002050400020C0
:107618004C400020014B93ED020A7047580C0020A3
:10762800014B93ED030A7047580C0020014B93ED72
:10763800040A7047580C0020034B83ED000AC3ED81
:10764800010A83ED021A7047E48D0020014B18608F
:10765800704700BF94400020014B1868704700BF76
:1076680088400020014B1868704700BF384100204F
:1076780008B54FF49570FEF743FB40F26523C31A33
:10768800584240EB030008BD08B5C620FEF738FB9A
:1076980040F28D13C21A504240EB020008BD4FF46D
:1076A800957040F26521FEF71DBBC62040F28D1192
:1076B800FEF718BB08B5F9F73FF9BCEEC00A4FF45E
:1076C800967010EE101AFEF72AFBF9F73BF90146FF
:1076D8004FF49870FEF723FBF9F73AF9BCEEC00AAD
:1076E8004FF49A7010EE101ABDE80840FEF717BB69
:1076F80038B5FFF7BDFFC0B14FF49670FEF728FB11
:10770800124D134C28604FF49870FEF721FB20604F
:107718004FF49A70FEF71CFB0E4B2A6818600E4B4C
:107728005A612268D8619A6106E00B4B0B4A5A618C
:107738000B4A9A610B4ADA61074A0B4B9069D16987
:10774800526958601A60996038BD00BF140D002056
:10775800100D00200C0D0020580C0020E17A843F09
:1077680014AE3740CCBC8C2CE48D002060EEA00A0F
:10777800B7EE007AF0EE606A70EE077A40EE006AC3
:1077880047EEA70A36EEC77A08B5C7EE200A10EE0C
:10779800900A07F0E1F90022084B07F031FA0022BD
:1077A800074B07F07BF807F00DFD07EE900AFDEE9A
:1077B800E77A17EE900A9F3008BD00BF00005940D5
:1077C8000000E03F38B52DED028BF7EE008AB0EEF1
:1077D800608A70EE288A10EE900A28EE088A07F070
:1077E800BBF908EEA88A00220F4B07F009FA0446F5
:1077F80018EE100A0D4607F0AFF902460B46204670
:10780800294607F027FB0022084B07F047F807F046
:10781800D9FC07EE900AFDEEE77A17EE900A77306A
:10782800BDEC028B38BD00BF000069400000E03F9E
:10783800F0B5694D2DED068B95E80F008DB008AEBB
:10784800103586E80F000FCD01AC0FC495E807008E
:107858004FF6FF7384E807009F2077216422FAF728
:107868007CFBA020772164224FF6FF73FAF775FBA3
:107878009E20772164224FF6FF73FAF76EFB9F2054
:10788800762164224FF6FF73FAF767FB4FF6FF7312
:10789800782164229F20FAF760FB0020FCF72AFB7E
:1078A8009F2077216522FCF7FFFC9F207721642227
:1078B800FCF7FAFC07AD0C36F7EE009A0435F7EE44
:1078C800008A95ED009A4FF49674B0EE68AA18EE07
:1078D800900A07F041F93EA3D3E9002307F090F995
:1078E80007F070FC08EE900A38EEE98AB0EE490A13
:1078F800F0EE480AFFF73AFFB0EE490AF0EE480A00
:107908000746FFF75FFFBFB281B20F223846FCF788
:10791800FEF9013CDBD14FF49674F7EE008A18EEBD
:10792800900A07F019F92AA3D3E9002307F068F9A8
:1079380007F048FC08EE900A39EEE88AB0EE490AEA
:10794800F0EE480AFFF712FFB0EE490AF0EE480AD7
:107958000746FFF737FFBFB281B20F223846FCF760
:10796800D6F9013CDBD1B542A8D16C4607AE043448
:1079780094ED009A4FF4C875F7EE008A18EE900A55
:1079880007F0EAF812A3D3E9002307F039F907F062
:1079980019FC08EE900A38EECA8AF0EE490AB0EEF1
:1079A800480AFFF7E3FEB0EE480AF0EE490A074638
:1079B800FFF708FFBFB281B200223846FCF7A7F9EB
:1079C800013DDBD1B442D2D10DB0BDEC068BF0BD88
:1079D800295C8FC2F528F03F38990408121A06EE80
:1079E800902A081AB8EEE67A06EE900AF8EEE67AD9
:1079F800C7EE277A9FED047A67EE877AFDEEE77A7D
:107A080017EE900A704700BF0000A0438A1A06EEDE
:107A1800902A081AB8EEE67A06EE900AF8EEE67AA8
:107A2800C7EE277A9FED047A67EE877AFDEEE77A4C
:107A380017EE900A704700BF0000484370B506462D
:107A48000D460024610704D5A0B231462A46FCF74A
:107A58005EF90134B4F5A07FF4D170BD70B5064667
:107A68000D460024600704D5A1B230462A46FCF72B
:107A78004EF90134C82CF5D170BD114B11481B7853
:107A88001149124A0068012B114B09D1126808608C
:107A98001A60104B1A68104B1A60104B1A680CE0E9
:107AA8001268D2011A600B4B1A680B4BD2011A608C
:107AB8000A4B1A68C0010860D201094B1A60704766
:107AC800080D002088400020804000203841002018
:107AD800704000208C400020903A00206440002034
:107AE80030410020024B1A68024B1A60704700BFF1
:107AF800804000209440002008B5FFF7BEFFBDE895
:107B08000840EFE70022F0B51346202603254FF082
:107B18002C0C00E02646303EF6B217460132092EFC
:107B280010F8014B0AD897FBF5F605FB16772FB925
:107B3800CE1801F803C07470023301E0CC5401334D
:107B4800092AE7D12022CA54CB1848225A707A222F
:107B58009A700022DA70F0BD70B58CB005460C46FC
:107B680008A80E491E460BF0C5FC08A86946FFF791
:107B7800C9FF6A460A4904A80BF0BCFCBDF84000DE
:107B8800FCF75CFB3046FCF76FFB2846214604AA4D
:107B98000023FCF781FC0CB070BD00BF61A3050891
:107BA80022A105082DE9F047084B2DED0A8B1B781B
:107BB800022BC4B000F01485054B1A78054B5AB94E
:107BC8001A68802392FBF3FA08E000BF8C4D00206E
:107BD800080D002094400020D3F800A0FFF7D4F946
:107BE800CD4C84ED080AFFF7D5F994ED0A8AD4ED57
:107BF800088A38EE088AF0EE087A38EE288A84ED8A
:107C0800090A88EE278AE06A10EE105A84ED028A83
:107C180084ED0A8A06F0A0FF02460B4606F03EFEF7
:107C2800064628460F4606F097FF02460B463046A2
:107C3800394606F033FE0022B84B07F00BF907F07F
:107C4800C1FAB74BB74A9D68E060D3ED007A67EE9A
:107C5800A88AC2ED007AD3ED017AB34BE062C4ED95
:107C6800088A1B78DFEDB18AC2ED017A77EEA88A1F
:107C780013B984ED088A6062206A06F06DFF064633
:107C8800606A0F4606F068FF41EC100B41EC190BD7
:107C980008F0FAFE59EC108BB0EE490AF0EE690ACA
:107CA80008F0F2FF304653EC102B394606F0A8FFD7
:107CB80007F088FA42464B4608EE100A3946304625
:107CC80006F09EFF07F07EFA9FED997AC8EE878A44
:107CD80009EE900A79EEE89A68EE087A49EEA97AF0
:107CE800B1EE488A67EE877A9FED92BA88EE278AC6
:107CF800C9EEA79A84ED048A18EE100A06F02CFF44
:107D0800CDE90601504606F015FF7FA3D3E900230D
:107D180006F076FF064628460F4606F01DFF024687
:107D28000B463046394606F06BFF02460B46DDE946
:107D3800060106F0B1FD07F045FA0AEE100A29EE31
:107D4800A98A6AEE0ACAB1EE4A9A78EE2C7ADFED71
:107D58007ABA89EE279A794BC9EEA7AAB4EE4B9A5C
:107D6800F1EE10FAC8BFB0EE4B9AB4EE6B9AF1EE92
:107D780010FA48BFB0EE6B9AC3ED00AA83ED019AE2
:107D88001AEE900A06F0E8FE00226D4BCDE90201DA
:107D980006F082FD69EE097A044617EE900A0D4650
:107DA80006F0DAFE224606460F462B4620462946AE
:107DB80006F026FF32463B4606F070FD41EC100BFC
:107DC80009F046F80022DDE902015D4B59EC108B01
:107DD80006F064FD02460B4606F012FF32463B46AB
:107DE80006F05CFD41EC100B09F032F840464946BC
:107DF80055EC104B07F0E6F9294608EE900A2046A4
:107E080007F0E0F907EE900AC8EEA78A4D4D4E4CF0
:107E1800B7EE00CA18EE900A06F09EFE3CA3D3E91E
:107E2800002307F05FF9DFED497A002818BFF0EE6C
:107E3800678AF4EE4C8ADFED467AF1EE10FAC8BF95
:107E4800F0EE678ADFED437A6AEE277AC5ED008A9D
:107E580017EE900A06F080FEDFED3F7A37EEC88A0B
:107E6800064678EE6CCA0F46C4E902671CEE900A13
:107E780006F072FE47EC106B41EC110BC4E90001EF
:107E880008F05EFF38EE8C8A3CEE68CA51EC100BA5
:107E980088EE0C8A07F096F9304B1B7880F0004882
:107EA800B4EE4B8AF1EE10FAC8BFB0EE4B8AB4EECE
:107EB8006B8AF1EE10FA48BFB0EE6B8A022BC5F858
:107EC80004806AD1264F3E68002E66DB254B264D7E
:107ED800C3F800A0B400621C5B6845F824A018EE43
:107EE800900A45F8223006F037FE00221F4B06F0B4
:107EF80087FE07F047F904F1020980B245F8290026
:107F0800404635E0AFF300801F85EB51B81E19409D
:107F18002D431CEBE2361A3F580C002000000840A5
:107F2800E48D00209C0100202C41002000008C42A0
:107F38000000F042003C1C46003C1CC6844D00205A
:107F480000004940684C0020404F002017B7D13846
:107F580072F97F3F0AD7233D17B7D139943A0020E9
:107F680084400020784D0020544F00200000F0404D
:107F780006F0F2FD9AA3D3E9002306F041FE07F0CC
:107F8800D9F803340136B6F57A7FC8BF4FF0FF330E
:107F980045F824003E60C8BF3B60FFF701F87E4CFF
:107FA80084ED0C0AFFF702F884ED0D0AFDF766FE72
:107FB8005246A063794934A80BF09CFA206B06F06E
:107FC800CBFD02460B4624A875490BF093FA606B6B
:107FD80006F0C2FD02460B4628A872490BF08AFA41
:107FE80019EE900A06F0B8FDCDE90401DDE9042395
:107FF8006D492CA80BF07EFA6C49DDE9062330A800
:108008000BF078FADDE90223694910A80BF072FA3F
:1080180019EE100A06F0A0FDCDE90A01DDE90A23F0
:10802800644914A80BF066FA18EE900A06F094FD5D
:10803800CDE90801DDE908235F4918A80BF05AFAD1
:10804800404606F089FD06460F4632463B465B49E8
:108058001CA80BF04FFA18EE100A06F07DFD8046BA
:1080680089464B465649424620A80BF043FA0CA8CD
:108078005449A26B0BF03EFA534B1B78013BDBB221
:10808800012B00F29F82514B1B78072B00F29A823A
:10809800DFE813F008009802AA0031017401D0014A
:1080A80068022E020220FCF7BFF94FF6FF70FCF7BA
:1080B800DBF81F20FCF7C2F819210023444A2D20C1
:1080C800FCF7EAF94FF6FF70FCF7CEF80020002421
:1080D800FCF7B4F80F20B42152464FF6FF73009412
:1080E800FFF73AFD0F20772124AA2346FCF7D4F99D
:1080F800A0200DEB000277212346FCF7CDF90F20D5
:10810800412118AA2346FCF7C7F9A02041211CAA3F
:108118002346FCF7C1F90F2065212CAA2346FCF75A
:10812800BBF930AA2346A0206521FCF7B5F90F203A
:10813800532110AA2346FCF7AFF9A020532114AA13
:108148002346FCF7A9F90F209B2120AA2346FCF718
:10815800A3F9114B9B6BB3F57A7FCCBF4FF4FC604E
:108168004FF47840FCF780F80CAAA0209B2100234C
:10817800FCF792F9174B1B780221012B0CBF164A0A
:10818800164A4FF48C700023FCF786F91F20FCF781
:108198006BF817E2AFF30080580C002066A30508BF
:1081A80070A305087BA3050886A3050890A3050806
:1081B8009AA30508A5A30508B0A30508BBA305084D
:1081C800C6A30508D2A30508943A00202C41002034
:1081D800DFA30508080D0020FEA3050802A4050872
:1081E800CDCCCCCC0C5FC440DDE904233EA8B24919
:1081F8000BF080F9DDE9062341A8B0490BF07AF9C4
:10820800DDE9022338A8AE490BF074F9DDE90A2349
:108218003BA8AC490BF06EF9E62002213EAA0023E8
:10822800FCF73AF9E620162141AA0023FCF734F9B5
:108238000220C82138AA0023FCF72EF93BAA002304
:108248000220DC21FCF728F9DFED9F7A68EEA78A87
:108258004FF6E07518EE900A06F07EFC47EC106BBE
:10826800CDE9020108F010FC59EC108B47EC106BBB
:1082780008F00AFD002057EC106BFBF7F5FF0A2108
:108288005246002305200095FFF766FC4FF478401E
:10829800FBF7D4FFDDE9020142464B4606F0B0FC8D
:1082A80077A3D3E9002306F0F9FA06F043FF324634
:1082B80084B23B46DDE9020106F0A2FC02460B4609
:1082C80071A1D1E9000106F0E7FA06F033FF81B2A7
:1082D8002046F9F772FE9D20772105220023FBF73F
:1082E800DDFF9F20752105220123FBF7D7FF2846D4
:1082F800FBF7A4FF66E1754B1868754B5246196881
:10830800FFF76CFBB0F59F7F044602DD714B02223C
:108318001A709FED718AF4EEC8AAF1EE10FA14D51E
:10832800F5EEC0AAF1EE10FA0FDDFDEEEAAA4FF461
:10833800FA711AEE902A0020FFF768FBA3B281B207
:108348004FF6FF721846FBF7E2FCB4EEC89AF1EE5E
:1083580010FA40F13781DFED617AB4EEE79AF1EE79
:1083680010FA40F32F81BDEEC99A5D4819EE102A24
:108378004FF4FA71FFF74AFBA4B2EEE0534B1868CA
:10838800534B52461968FFF729FBB0F59F7F064605
:1083980002DD504B02221A70F5EEC09AF1EE10FA87
:1083A8001DDDDDE904013AA3D3E9002306F09AFEB6
:1083B800A8B139A3D3E90023DDE9040106F020FCC4
:1083C80002460B460020474906F066FA06F0B2FE60
:1083D800B4B281B24FF6FF722046FBF798FC1AEE52
:1083E800100A06F0B9FB2EA3D3E9002304460D4674
:1083F80006F096FE002800F0E5802046294624A3D2
:10840800D3E9002306F06EFE002800F0DB8026A3E7
:10841800D3E900232046294606F0F2FB02460B4624
:108428000020314906F038FA06F084FEB6B281B26F
:10843800304694E0DDE908011DA3D3E9002306F0E6
:108448006FFE002800F0BE80204B1868204B524673
:108458001968FFF7C3FAB0F59F7F044602DD1D4B8C
:1084680002221A709DED080B08F06CFC53EC102BDF
:108478001046194600221D4BA4B206F0C1FB99E034
:108488000000000000E063400000000000C05D4004
:108498009A9999999999B93F0000000000409F4026
:1084A8009A9999999999B9BF0000000000408F40A6
:1084B80076711B0DE02DA03F06A4050810A4050841
:1084C8001AA4050824A405080000C8428840002012
:1084D800384100208C4D00200000FA430000FAC308
:1084E8000CFEFFFF0000694000005940000054C026
:1084F80047A3D3E900233046394606F081FB46A35B
:10850800D3E9002306F0A6FC06F05CFE384B08EE23
:10851800100A1868374B52461968FFF75FFAB0F52A
:108528009F7F02DD344B02221A70DFED347A48EE69
:10853800E77A84B2FDEEE77A204617EE901A4FF6F6
:10854800FF7289B2FBF7E3FBBDEEC88A6FF0B30098
:1085580018EE102AB421FFF759FA81B220464FF4D9
:10856800FC622DE0DFED267AB4EEE78AF1EE10FA30
:1085780028D51F4B18681F4B52461968FFF72EFA6B
:10858800B0F59F7F044602DD1B4B02221A7049ECAE
:10859800108B08F0D7FB53EC102B1046194600221D
:1085A800184B06F02DFB02460B4600201649A4B2D4
:1085B80006F072F906F0BEFD4FF6FF7281B2204652
:1085C800FBF7A5FB114B1B78022B09D043B14FF6E3
:1085D800FF7300930520DC2152460023FFF7BCFA05
:1085E80044B0BDEC0A8BBDE8F08700BFAFF3008054
:1085F80088400020384100208C4D0020000048436E
:108608000000C84200005940000069402C41002089
:1086180000000000008076401F85EB51B81E19400D
:108628002DE9F04F764B2DED048B93ED008A78EE13
:10863800087A83B017EE900A06F08EFA714B064658
:1086480018680F4606F088FA68EE088A82468B4654
:10865800F7EE009A4BEC10AB08F016FA78EEA97A10
:1086680055EC104B17EE900A06F076FA22462B4688
:10867800804689463046394606F0C2FA02460B461D
:108688004046494606F008F906F09CFD79EEE88A6E
:1086980009EE100AC8EE898ADFED5B7A4BEC10AB65
:1086A80068EEA78A08F0F0FA304653EC102B3946EA
:1086B80006F0A6FA044619EE100A0D4606F04CFA22
:1086C80002460B462046294606F0C4FB4F4B0022C3
:1086D80006F096FA06F076FD4D4B1B78033B09EE43
:1086E800100A042B78D8DFE803F003122F5846004D
:1086F80018EE900A06F030FA044619EE100A0D46F4
:1087080006F02AFACDE900014248434917E029EE6C
:10871800098A08EEA88AB1EE499AC8EE888A89EED5
:10872800088A18EE900A06F017FA044618EE100A9E
:108738000D4606F011FACDE90001364837492246C0
:108748002B460AF0D7FE47E018EE100A06F004FAA6
:1087580041EC100B08F0F6FA0022314B51EC100BEB
:1087680006F04EFA06F02EFD06F0F6F902460B4624
:1087780028482C492EE018EE100A06F0EDF91CA343
:10878800D3E9002304460D465046594606F038FA08
:10879800CDE900011F482449D1E718EE100A06F078
:1087A800DBF915A3D3E9002306F0BAFCDFED1F7A45
:1087B800002818BFB0EE678A78EE297A79EEC89A51
:1087C800C7EEA99A19EE900A06F0C6F902460B46BA
:1087D800104817490AF08EFE0E4A0220CA210023CB
:1087E80003B0BDEC048BBDE8F04FFBF755BE00BFEE
:1087F800F6285C8FC2A54C40AE47E17A14AEEF3F35
:10880800704C0020744C0020000048420000494091
:108818002C410020424C00202EA405083EA4050847
:10882800000034C04EA4050860A40508A4707D3F6C
:108838007CA4050873B50546002800F09E80524BBD
:1088480018884519ADB22AB2002A05DB40F23F1359
:108858009A42C8BF1D4600E000250121FBF7B6F982
:108868000120FBF707F8494E0024A05B0234FBF710
:108878004FF8B4F5C67FF8D1A8B2C72201214EF24D
:108888009C73FBF7B9FB404B1D80414B1C68414B67
:108898002DB21B6806EE905A1B1BB8EEE67A06EE60
:1088A800903AF8EEE67A67EE277A17EE900A06F025
:1088B80053F90022384B06F0CDFA06F03BFC4FF690
:1088C800FF73241800930520DC2100232246FFF7BC
:1088D80043F9002131480B4600E0114690E8240096
:1088E800A24203DB2E4880E8240008E00133103060
:1088F800B3F57A7FF1D12A4981E824001146022094
:10890800521892FBF0F294420BDA013B03FA00F0A2
:108918002249234A51F820400130146051F82010B0
:1089280051609B001D4A1F4C1F4D991C033352F880
:10893800211052F8233007EE901AB8EE677ADFED6F
:108948001B7A06EE903A67EE277AC4ED007AF8EEC5
:10895800E67A17EE900A06F0FFF809A3D3E9002398
:1089680006F078FA06F02EFC114B28601A7820469B
:10897800294602B0BDE8704052E602B070BD00BFA3
:10898800CDCCCCCC0C5FC440404C00208E4D002098
:10899800884000203841002000007440544F0020D7
:1089A800784D0020704C0020744C00200000803767
:1089B8002C41002013B50F4CA38FADF80630BDF83D
:1089C80006309BB253B1BDF806004EF29C7380B2DC
:1089D8000121C722FBF710FB0023A387064B1B7856
:1089E800022B06D1054C94F90000FFF723FF002362
:1089F80023701CBD580C00208C4D0020302A00200C
:108A080038B54FF47A7441F288352046FDF7ECFE0C
:108A18000134C0B2A4B200F083F9AC42F5D138BD3C
:108A2800054B06491A6801EB8201013202F01F0268
:108A380081ED000A1A607047644C0020F84C002051
:108A4800054B06491A6801EB8201013202F01F0248
:108A580081ED000A1A607047F08D00207C4C0020E0
:108A6800094A0A4913680968994209D0084901EB7B
:108A78008301013303F01F0391ED000A136070476F
:108A88009FED040A704700BF784C0020644C00201A
:108A9800F84C002000000000094A0A4913680968D8
:108AA800994209D0084901EB8301013303F01F0300
:108AB80091ED000A136070479FED040A704700BFEC
:108AC800344F0020F08D00207C4C00200000000076
:108AD800024A00231360024A13607047784C002052
:108AE800644C0020024A00231360024A1360704756
:108AF800344F0020F08D002008B50021C620FDF776
:108B0800F1F84FF495700021BDE80840FDF7EAB888
:108B1800024B4FF6FF721A80704700BF404C00208E
:108B280070477047FEE7FEE7FEE7704770477047FB
:108B3800FEF724BC08B5022003F002FE48B1054B3D
:108B4800D3F880305B6998470220BDE8084003F0FD
:108B580005BE08BD9840002000F062BA014802F046
:108B6800DBBA00BF983A0020704700BF414BD3F8EA
:108B7800882042F47002C3F888203F4B1A6842F0FC
:108B880001021A6000229A60196821F0847121F4A8
:108B98008031196039495960196882B021F48021FF
:108BA8001960DA60009201921A6842F480321A6001
:108BB8001A6802F400320192009A01320092019A76
:108BC8001AB9009AB2F5A06FF2D12B4B1B6813F4B7
:108BD800003318BF01230193019B012B2ED1264B93
:108BE8001A6C42F080521A64254A116841F4804197
:108BF80011609A689A609A6842F400429A609A688A
:108C080042F4A0529A601F4A5A601A6842F0807271
:108C18001A601968184A8901FBD51B4B40F2056197
:108C28001960936823F003039360936843F0020389
:108C38009360936803F00C03082BFAD10E4B9A68E3
:108C480022F400029A60114AC3F884201A6842F09C
:108C580080621A601A681201FCD5064B4FF0006258
:108C68009A60D3F8882042F47002C3F8882002B0D2
:108C7800704700BF00ED00E00038024010300024CB
:108C88000070004008544007003C0240804000301B
:108C9800184B194A996801F00C01042903D00829D6
:108CA80003D0164B19E0164B17E059685A6811F4AF
:108CB800800F596814BF124B104B02F03F02B3FBF0
:108CC800F2F30C4A5268C2F30142C1F3881101322F
:108CD80052004B43B3FBF2F3074A1360054B9A6803
:108CE800054BC2F303129A181968127921FA02F295
:108CF8001A60704700380240A40100200024F400E4
:108D080000127A0008B5402003F01AFD30B1FBF7D5
:108D180021FD4020BDE8084003F020BD08BD00004B
:108D2800014608B5044805F0D5FC0348402105F084
:108D38007EFD0028F9D008BD00440040F0B589B098
:108D48004FF4E1330120019300232B4CADF8083098
:108D58001E460146ADF80A30ADF80C30ADF81030BB
:108D68000C23ADF80E3004F045FB4FF40030012120
:108D780004F064FB20680221072204F013F807229C
:108D88006068032104F00EF80125022704232068F7
:108D9800059305A98DF81A608DF81B508DF8187089
:108DA8008DF8197003F07EFF08236068059305A904
:108DB8008DF8187003F076FFA06801A905F0E0FBB4
:108DC8002A4640F225510D4805F018FD262307A82C
:108DD8008DF81C308DF81D608DF81E608DF81F50C1
:108DE80000F06EFBA068294605F047FC044A054BD5
:108DF8001A6009B0F0BD00BFB8010020004400406F
:108E0800298D00083C8E0020024B9868002105F04F
:108E180034BC00BFB801002010B5094C40F2255100
:108E2800204605F00EFD50B1A288D2B2112A02D117
:108E3800044B01211970044B19884A401A8010BD4F
:108E480000440040160C0020980C00201FB5214B50
:108E58000C46186000214FF0804004F02CFF0121DF
:108E680000224FF0804005F056FA022C01D10B2366
:108E780003E0012C02D142F6DF6302930523ADF82B
:108E880004304FF08040002301A9ADF80C30ADF854
:108E9800063004F07BFE4FF08040012105F05BFABC
:108EA8004FF08040012104F0E4FE01210A464FF012
:108EB800804005F030FA4FF08040012104F0FBFEBD
:108EC800044B19680029FCD14FF0804004F0F3FEF0
:108ED8001FBD00BF9C0C00207047F0B5012085B075
:108EE8002D4D014604F086FA4FF4D0530026019325
:108EF80003270223284601A98DF808308DF8097048
:108F08008DF80A608DF80B6003F0CCFE2846092125
:108F18000A2203F047FF28460B210A2203F042FFEA
:108F28000A2228460C2103F03DFF01244FF48063F8
:108F3800284601A901938DF80A408DF80B408DF859
:108F4800097003F0AFFE0A210A46284603F02AFFFB
:108F580021464FF4804004F07DFA8020214604F039
:108F680055FA31464FF0006000F0DEFA4FF4A06089
:108F780000F09CFA1C2303A88DF80C308DF80D60C6
:108F88008DF80E408DF80F4000F09AFA20462146E1
:108F980004F054FA05B0F0BD0000024007B54FF4E4
:108FA800C06000F083FA43238DF8043001A8012340
:108FB8008DF805308DF806308DF8073000F080FA0E
:108FC8000EBD044811B9012103F0DDBE012103F0F3
:108FD800DCBE00BF00080240022137E7012135E767
:108FE80037B5042001210D4D04F004FA02230124B1
:108FF8008DF805302846002369468DF806308DF82F
:10900800073000948DF8044003F04CFE28462146B2
:1090180003F0B9FEC820FFF7E1FF3EBD000802409B
:1090280008B54FF08040012105F08AF988B1012187
:109038004FF0804005F08FF9064B196819B11A688E
:10904800013A1A6008BD4FF08040BDE8084004F0BE
:1090580032BE08BD9C0C00207047012070470349B0
:10906800034A02204FF4B77300F09CB887A40508A0
:109078007C9904080349044A022040F2371300F09F
:1090880091B800BF87A405088C9904080349044ACD
:10909800022040F2011300F085B800BF87A405083C
:1090A800A99904080249034A0220F52300F07AB876
:1090B80087A40508C29904080249034A0220EA2342
:1090C80000F070B887A40508DC9904080249034A2F
:1090D8000220DF2300F066B887A40508F499040885
:1090E8000249034A0220C82300F05CB887A4050897
:1090F800119A04080249034A0220BC2300F052B81E
:1091080087A40508369A04080249034A0220A623C0
:1091180000F048B887A40508559A04080249034A8C
:1091280002208B2300F03EB887A40508739A040830
:109138000249034A0220802300F034B887A40508B6
:10914800909A04080249034A0220682300F02AB8CA
:1091580087A40508A59A04080249034A0220522355
:1091680000F020B887A40508BF9A0408FDF774BD6D
:10917800FDF77ABD04490A6801320A6003490346CB
:10918800022000F00FB800BFA00C0020A8A405081A
:10919800FDF770BD80F08000092801D8FDF730BDCB
:1091A800704700BF0EB403B070470A2810B50446D4
:1091B80002D10D20FFF7F9FF064A13681BB103F827
:1091C800014B136010BD044B1B680BB12046984738
:1091D80010BD00BFA40C00203C8E002010B5044632
:1091E80001E0FFF7E2FF14F8010B0028F9D110BDE8
:1091F8002DE9F04F044685B00D464FF00A0A00E00D
:1092080035462078002800F0C480252801D0013494
:1092180067E06078302803D1A0780123033407E0A1
:109228002D2802D00234002302E0A0780223033460
:109238004FF0000805E00AFB080814F8010BA8F134
:109248003008A0F13002D2B2092AF4D96C2801D032
:109258004C2803D114F8010B43F00403002800F054
:109268009880602886BFA0F12002D2B202464F2A19
:109278003DD006D8432A2DD0442A09D0422A30D1DD
:1092880033E0552A04D0582A29D0532A29D101E09D
:109298000A272DE02E1D2F68002500E001357A5D94
:1092A800002AFBD104E02020FFF77FFF4D4601E0B4
:1092B800980704D4454505F10109F4D34D463846CD
:1092C800FFF78CFF03E02020FFF76FFF01354545CE
:1092D800F9D395E728782E1DFFF767FF90E7102749
:1092E80006E0FFF762FF2E468AE7022700E008271C
:1092F8002E1D442A296804D1002902DA494243F084
:109308000803002200E02A46B1FBF7FE07FB1E1106
:10931800CDB2092D714607D9782814BF4FF0070C34
:109328004FF0270C6544EDB230350DF80250551C4E
:10933800BEF1000F02D0102DE5D10F22190705D577
:1093480004A94D192D2105F8101C951C13F0010FC7
:109358000CBF4FF0200B4FF0300B9B072F4604D566
:1093680008E05846FFF721FF4F46474507F1010936
:10937800F7D34F46013D1DF80500FFF716FF002DF6
:10938800F8D103E02020FFF710FF01374745F9D354
:1093980036E705B0BDE8F08F70B5064D0C462E686F
:1093A800286001E0FFF701FF14F8010B0028F9D14C
:1093B8002E6070BD3C8E00200FB407B504A951F88B
:1093C800040B0191FFF714FFBDE80E4004B070478D
:1093D8000EB417B505A9084C51F8043B206018468F
:1093E8000191FFF705FF2268002313702360BDE891
:1093F8001E4003B0704700BFA40C00200EB433B564
:1094080005A9074C51F8043B2568206018460191CE
:10941800FFF7EEFE2560BDE83C4003B0704700BF93
:109428003C8E002070B51E4604461C481546FFF7C2
:10943800C3FF022E1FD0042E25D0012E2AD105E00D
:10944800A15D1748FFF7B8FF013600E00026AE42DD
:10945800F6DB2020FFF7A9FE002609E0A05DA0F1B9
:109468002003DBB25E2B88BF2E20FFF79EFE01365D
:10947800AE42F3DB0EE034F8021B0A48FFF79CFF0C
:10948800013DF8D106E054F8041B0748FFF794FFA4
:10949800013DF8D10A20BDE8704086E6CBA4050856
:1094A800D2A40508D8A40508DEA4050840F0BE60CB
:1094B800024B40F42020D860704700BF00ED00E068
:1094C800C37810B503B3164B4278DB688478DB4366
:1094D800C3F30223C3F10401C9B202FA01F10F2256
:1094E80042FA03F2C9B222400A430E4B0178120134
:1094F800CB18D2B283F8002303780122590903F06C
:109508001F0302FA03F307E003780122590903F065
:109518001F0302FA03F32031024A42F8213010BD3A
:1095280000ED00E000E100E021F0604121F07F0162
:10953800014B08439860704700ED00E0044B1A693E
:1095480009B1104301E022EA00001861704700BF2A
:1095580000ED00E0044B1A6804280CBF42F0040236
:1095680022F004021A60704710E000E037B50023CB
:10957800104C019305460320FFF72EFDEB681A698E
:10958800013C019213D0019A002AF4DA019A42F0C0
:1095980001020192019A1A61064A1969013A019178
:1095A80002D00199C907F8D40320FFF715FD002060
:1095B8003EBD00BF410D030010B5C47874B900EB7F
:1095C800820003339B10D0F8D000224603E051F804
:1095D800044C0132046004319A42F8D1002010BDD5
:1095E800033230B59210D0F8D0400B46002003E08B
:1095F8002568013043F8045C04339042F8D101EB4C
:10960800800030BD0122F0B500238270402201297C
:10961800C37082800CD108230370042343704FF475
:10962800A073C38002230372C1724FF0A04309E004
:1096380041B90C230370062343704FF4A063C38021
:109648001F4BC17203F500620261C360467804468D
:1096580001461A46002508E002F5106C02F5306252
:109668000A65C1F814C001353A460431B54202F121
:109678002007F1D303F58062426103F58862C0F8E0
:10968800CC20067803F5A0650146002203E0C1F866
:109698008C50013220350431B242F8D319460022E9
:1096A80002E0C4F8CC1001320434B24201F5805112
:1096B800F7D303F56063C0F80C310020F0BD00BF9C
:1096C8000000044038B5037AC2680025012B04461F
:1096D8001FD1936B417A65F3104309B143F48013AA
:1096E8009363D3686FF386136FF396536FF3514305
:1096F8006FF3D343D3602046FFF738FFE378012B9D
:1097080019D1052363F34405E36845F020059D60FE
:1097180011E0D36843F04003D360FFF727FF637A73
:10972800E268002B0CBF4FF404134FF44413936307
:109738001420FFF753FCE378012B07D1E3689D68F9
:10974800052262F3440545F020059D60002038BDE0
:10975800C3689A6842F001029A6000207047C368A3
:109768009A6822F001029A600020704707B500232A
:109778000193019B43F020030193019B61F38A133A
:109788000193019BC2681361064B1169013B01916A
:1097980002D001998806F8D40320FFF71DFC0020A9
:1097A8000EBD00BF410D030007B500230193019BC7
:1097B80043F010030193019BC2681361064B1169C2
:1097C800013B019102D00199C906F8D40320FFF7A3
:1097D80003FC00200EBD00BF410D030008B5C268A0
:1097E800D36801296FF35D736FF39E7302D143F061
:1097F800005302E009B943F080433220D360FFF7F9
:10980800EDFB002008BDC368586900F001007047EF
:10981800C3685B6913F0010F14BF00200120704773
:10982800C368586900F001007047C3685A699869AD
:1098380010407047C3685868704743699B6813F0C5
:10984800010F14BF002001207047C36800229A61ED
:109858004FF0FF325A615A606FF080425A610B4AEA
:109868009A61C2789969002A0CBF1022002242F03E
:10987800487221EA02010A439A619A6922F0005269
:1098880022F008029A610020704700BF000800809B
:1098980043691A6861F301021A607047D0F8CC3046
:1098A80018686FF382006FF341006FF3C3006FF322
:1098B8004510704738B504460D46FFF782FB204631
:1098C800FFF7ECFFC0F3072303F01003DBB233B953
:1098D800012D04D1D4F8CC3040F480501860C0F386
:1098E800072303F01003DBB22BB125B9D4F8CC3031
:1098F80065F30C301860C820BDE83840FFF76EBB30
:1099080043695869704738B50546FFF7C7FFD5F86A
:10991800CC3040F480741C606420FFF75FFBD5F8FE
:10992800CC306FF3082414201C60FFF757FB01208C
:1099380038BD70B50446FFF753FBD4F80C31002549
:109948001D60237A012B08BF2946204618BF012134
:10995800FFF79EFF2046FFF7D6FF63691A686FF38B
:1099680082021A60E37A012B2E460ED1E368802228
:109978005A6262F30F05E02262F30F06C0F2600537
:10998800C0F260069D62C3F8006110212046FFF70F
:10999800EDFE2046FFF708FF002322464FF0FF3573
:1099A800184604E0D2F88C1001338D60C860217825
:1099B80004328B42F6D320460121FFF77BFF204675
:1099C800FFF743FF002070BD70B500EB810301F184
:1099D8001504D3F8902000EB44154FF0FF33936043
:1099E800C37895F81551012B0CBF04230023032DD0
:1099F8002BD8DFE805F0021F021300EB411404F531
:109A08006C7443F08903A57843F482637DB92479A3
:109A180043F04003CCB143F0200316E000EB4114BF
:109A280043F0990394F8B24343F4C0636CB143F430
:109A380080730AE000EB441443F0010394F81241E8
:109A480043F408730CB143F4C073D3604369012431
:109A58009D6904FA01F42C439C61C3689C69153123
:109A680000EB411044F000749C6190F81011002341
:109A780061F39C5390F8111161F3CE2390F8121101
:109A880061F3CF3390F81311A1F1020CDCF100015E
:109A980041EB0C0161F3514390F8151100F58874FE
:109AA800B0F8160161F3934360F30A03032908BF72
:109AB80043F000531360002070BD70B501F11E041F
:109AC800640186B003590A46002583B100EB4111B1
:109AD800013BB1F8B6135B18B3FBF1F39BB2B3F5D6
:109AE800807F05D9090201514FF4807300E00123FA
:109AF80000EB421191F8B24301F56C712CB1C988A1
:109B080000EB42145943C4F8C01300EB4211D1F8DA
:109B1800C01361F3120563F3DC4500EB421393F8BD
:109B2800B84364F35E7500EB8204D4F89040256175
:109B3800C578012D08BFD3F8BC33456908BF6361F8
:109B48002368AE6816F0010F14BF0026012666F3DD
:109B58005D7343F000436FF39E732360C378002B5B
:109B680031D102F1150300EB431393F8124154BBB2
:109B780049B393F81531032B1DD8DFE803F0020F22
:109B8800020FC368DC6A03310194C1F38F01A4B2E8
:109B98008C4210D2996941F020010BE02B69033106
:109BA8000493C1F38F019BB28B4204D2C3689969B5
:109BB80041F08061996100EB4211B1F8C033D1F8EE
:109BC800BC13FFF7F9FC002006B070BD00EB810163
:109BD80086B0D1F89020136843F04043C3F307419F
:109BE80011F00C0101D0082902D1C168C96A01E04D
:109BF80041690969C1F3074109B961F3DF7313606A
:109C0800002006B07047034610B503EB810301241A
:109C1800D3F890304FF0004264F3DC421A611A68BE
:109C2800002042F0004260F39E721A6010BD436942
:109C38004FF0FF31002210B59A6104465961014680
:109C48000AE0D1F88C0003686FF3DF7343F08043B8
:109C58006FF3CF3303600132237804319A42F0D393
:109C68002046FFF7A1FD20461021BDE810407DE504
:109C7800002310B51A460446C0F8103303F1C60095
:109C880044F8202003F1D40004EB80004260E0187F
:109C980001330F2B80F89023F0D10823A4F8B633B2
:109CA8002046FFF7AFFC2046FFF759FD2046FFF797
:109CB80009FD01212046FFF791FD2046FFF739FEF7
:109CC8002046FFF745FD002010BDD0F8CC301868BD
:109CD800C0F34140704708B5FFF715FE002008BDE6
:109CE800D0F810037047D0F8140370474369986898
:109CF80080B27047401890F89F037047D43100EB4A
:109D0800810040687047401890F89003704708B584
:109D1800FFF75AFE08BD421808B5002382F89F33A2
:109D280001F11E0200EB42125360FFF7C6FE08BDA8
:109D380080B584B000AF78604FF00003FB6040F25C
:109D48000C23C2F200031B681B6878689847FB68FD
:109D580043F00803FB607B68DB68FA685A614FF0E0
:109D68000103184607F11007BD4680BD80B584B0D1
:109D780000AF78604FF00003FB6040F20C23C2F2A2
:109D880000031B689B6878689847FB6843F000539A
:109D9800FB607B68DB68FA685A614FF0010318467C
:109DA80007F11007BD4680BD80B485B000AF78606C
:109DB8007B68D3F890301B68BB60BB6843F00043F6
:109DC800BB60BB6843F08043BB607B68D3F89030CE
:109DD800BA681A604FF00003FB60FB6843F4001395
:109DE800FB607B68DB68FA685A614FF0010318462C
:109DF80007F11407BD4680BC704700BF80B588B026
:109E080000AF78604FF00003FB724FF000037B61F6
:109E18007B6943F010037B617B68DB687A68D268F2
:109E2800926911467A696FEA02020A409A617B6870
:109E3800DB681B6ABB61BB69C3F30303DBB2FB725C
:109E4800FB7ADBB27A6803F122034FEA8303D31863
:109E58009B681B68FB60BB69C3F34343DBB2022BFF
:109E680040F09A80BB69C3F30A139BB2002B40F3FE
:109E78009480FB7ADBB27A684FEA4313D31803F570
:109E88006F731B68002B00F08880FB7ADBB27A685E
:109E98004FEA4313D31803F56F731A68BB69C3F30A
:109EA8000A139BB2786811461A46FFF799FBBB69FB
:109EB800C3F30303DBB2BA69C2F30302D2B279680F
:109EC8004FEA42128A1802F56F721168BA69C2F332
:109ED8000A1292B28A1879684FEA4313CB1803F52D
:109EE8006F731A60BB69C3F30303DBB2BA69C2F3C9
:109EF8000302D2B2796802F11E024FEA42128A18AE
:109F080002F104021168BA69C2F30A1292B28A18FD
:109F1800796803F11E034FEA4313CB1803F10403D6
:109F28001A60FB7ADBB27A6803F11E034FEA431327
:109F3800D31803F104031B68FB61FB7ADBB27A6870
:109F480003F1D4034FEA8303D318FA695A60FB7A02
:109F5800DBB27A6803F122034FEA8303D3189B68C4
:109F68001B693B613B69C3F3C9439BB2002B14DDFA
:109F7800FB6843F00043FB60FB686FF39E73FB6074
:109F8800FB7ADBB27A6803F122034FEA8303D31822
:109F98009B68FA681A6000E000E000BF7B6943F044
:109FA80010037B617B68DB687A68D2689269114626
:109FB8007A690A439A614FF00103184607F12007AE
:109FC800BD4680BD80B59CB000AF786039607A68C6
:109FD8003B6803F122034FEA8303D3189B68FB66AF
:109FE800FB6E9B68BB66FB6EDB687B66BA6E7B6E3E
:109FF8001340BB667A683B6803F122034FEA830388
:10A00800D3189B681B683B664FF000037B6697F884
:10A01800683003F00403DBB2002B22D04FF00003BA
:10A02800BB65BB6D43F00403BB65BA6DFB6E9A60FC
:10A038007A683B6803F122034FEA8303D3189B68CD
:10A04800DB687B657B6D43F002037B657A683B6860
:10A0580003F122034FEA8303D3189B687A6DDA6011
:10A0680098E097F8683003F02003DBB2002B0AD0A1
:10A078004FF000033B653B6D43F020033B653A6DB1
:10A08800FB6E9A6086E097F8683003F00803DBB24D
:10A09800002B3ED07A683B6803F122034FEA830322
:10A0A800D3189B68DB68FB64FB6C43F00203FB641A
:10A0B8007A683B6803F122034FEA8303D3189B684D
:10A0C800FA6CDA607A683B68D31803F564734FF06A
:10A0D80005021A704FF00003BB64BB6C43F0100319
:10A0E800BB64BA6CFB6E9A604FF000037B647B6CB8
:10A0F80043F008037B647A6CFB6E9A60BB6E6FF367
:10A108000413BB663B68DBB278681946FFF75EFD4F
:10A1180040E097F8693003F00403DBB2002B39D034
:10A128007A683B6803F122034FEA8303D3189B68DC
:10A13800DB683B643B6C43F002033B647A683B6832
:10A1480003F122034FEA8303D3189B683A6CDA6061
:10A158003B68DBB278681946FFF738FD4FF000031B
:10A16800FB63FB6B43F01003FB63FA6BFB6E9A60B7
:10A178007A683B68D31803F564734FF008021A70C5
:10A188004FF00003BB63BB6B43F48063BB63BA6BE4
:10A19800FB6E9A6097F8693003F00203DBB2002B7C
:10A1A80028D07A683B6803F122034FEA8303D31867
:10A1B8009B68DB687B637B6B43F002037B637A6895
:10A1C8003B6803F122034FEA8303D3189B687A6B39
:10A1D800DA603B68DBB278681946FFF7F7FC4FF0A6
:10A1E80000033B633B6B43F400733B633A6BFB6ECA
:10A1F8009A60DEE197F8683003F00103DBB2002BC8
:10A2080000F0A5807B68DB78012B1DD17A683B685C
:10A2180003F122034FEA8303D3189B681B69FB658C
:10A228007A683B6803F11E034FEA4313D3181A6890
:10A23800FB6DC3F31203D21A79683B6803F1D403A8
:10A248004FEA8303CB185A607A683B68D31803F542
:10A2580064734FF001021A707B683A6802F1C60213
:10A268004FF0000143F822104FF00003FB62FB6A35
:10A2780043F00103FB62FA6AFB6E9A6097F862305A
:10A2880003F00C03DBB2002B06D097F8623003F022
:10A298000C03DBB2082B3BD17A683B6803F122033D
:10A2A8004FEA8303D3189B68DB68BB62BB6A43F041
:10A2B8000203BB627A683B6803F122034FEA830317
:10A2C800D3189B68BA6ADA603B68DBB278681946CB
:10A2D800FFF77CFC4FF000037B627B6A43F01003BE
:10A2E8007B627A6AFB6E9A607A683B684FEA43132E
:10A2F800D31803F572731B7883F00103DAB2796817
:10A308003B684FEA4313CB1803F572731A7050E198
:10A3180097F8623003F00C03DBB20C2B40F0488155
:10A328003B6E43F000533B667A683B6803F12203B7
:10A338004FEA8303D3189B683A6E1A607A683B68C1
:10A34800D31803F566734FF00102DA7130E197F81C
:10A35800683003F00203DBB2002B00F084807A68D7
:10A368003B6803F122034FEA8303D3189B68DB6839
:10A378003B623B6A6FF341033B627A683B6803F1D7
:10A3880022034FEA8303D3189B683A6ADA607A6833
:10A398003B68D31803F564731B78DBB2012B08D133
:10A3A8007A683B68D31803F566734FF00102DA71D7
:10A3B8004EE07A683B68D31803F564731B78DBB208
:10A3C800052B08D17A683B68D31803F566734FF0FC
:10A3D8000402DA713CE07A683B68D31803F56473C9
:10A3E8001B78DBB2062B08D07A683B68D31803F5D4
:10A3F80064731B78DBB2082B10D17B683A6802F1D2
:10A40800C6024FF0000143F822107A683B68D3185F
:10A4180003F566734FF00302DA7119E097F86230BA
:10A4280003F00C03DBB20C2B12D17A683B684FEABD
:10A438004313D31803F572731B7883F00103DAB260
:10A4480079683B684FEA4313CB1803F572731A70A7
:10A458004FF00003FB61FB6943F00203FB61FA69FB
:10A46800FB6E9A60A5E097F8683023F07F03DBB2B3
:10A47800002B3ED07A683B6803F122034FEA83033E
:10A48800D3189B68DB68BB61BB6943F00203BB61FF
:10A498007A683B6803F122034FEA8303D3189B6869
:10A4A800BA69DA607B683A6802F1C60253F822306A
:10A4B80003F101017B683A6802F1C60243F82210F1
:10A4C8007A683B68D31803F564734FF006021A7074
:10A4D8003B68DBB278681946FFF778FB4FF000035A
:10A4E8007B617B6943F080037B617A69FB6E9A60CC
:10A4F8005FE097F8683003F01003DBB2002B58D008
:10A5080097F8623003F00C03DBB20C2B1DD17A688C
:10A518003B6803F122034FEA8303D3189B68DB6887
:10A528003B613B6943F002033B617A683B6803F196
:10A5380022034FEA8303D3189B683A69DA603B68C1
:10A54800DBB278681946FFF741FB7A683B68D31895
:10A5580003F564734FF003021A704FF00003FB60B9
:10A56800FB6843F01003FB60FA68FB6E9A6097F88B
:10A57800623003F00C03DBB2002B06D097F8623090
:10A5880003F00C03DBB2082B13D13B6E43F00043FE
:10A598003B663B6E6FF39E733B667A683B6803F1DC
:10A5A80022034FEA8303D3189B683A6E1A6000E0CF
:10A5B80000BF4FF00103184607F17007BD4680BD84
:10A5C80080B59AB000AF786039607A683B6803F16B
:10A5D80022034FEA8303D3189B687B667B6E9B68D4
:10A5E8003B667B6EDB68FB653A6EFB6D13403B6632
:10A5F8007A683B6803F122034FEA8303D3189B6808
:10A608001B68BB6597F8603003F00403DBB2002BCE
:10A6180022D04FF000037B657B6D43F004037B651C
:10A628007A6D7B6E9A607A683B6803F122034FEA81
:10A638008303D3189B68DB683B653B6D43F00203DB
:10A648003B657A683B6803F122034FEA8303D3181A
:10A658009B683A6DDA6080E297F8603003F0200377
:10A66800DBB2002B0AD04FF00003FB64FB6C43F015
:10A678002003FB64FA6C7B6E9A606EE297F8613097
:10A6880003F00203DBB2002B28D07A683B6803F1A1
:10A6980022034FEA8303D3189B68DB68BB64BB6C57
:10A6A80043F00203BB647A683B6803F122034FEA74
:10A6B8008303D3189B68BA6CDA603B68DBB27868AE
:10A6C8001946FFF783FA4FF000037B647B6C43F471
:10A6D80000737B647A6C7B6E9A603EE297F8603018
:10A6E80003F00103DBB2002B38D07B683A6802F133
:10A6F800C6024FF0000143F822107A683B6803F164
:10A7080022034FEA8303D3189B68DB683B643B6CE6
:10A7180043F002033B647A683B6803F122034FEA83
:10A728008303D3189B683A6CDA603B68DBB27868BD
:10A738001946FFF74BFA4FF00003FB63FB6B43F03E
:10A748000103FB63FA6B7B6E9A607A683B68D318E7
:10A7580003F564734FF001021A70FEE197F8603058
:10A7680003F00803DBB2002B30D04FF00003BB63CB
:10A77800BB6B43F00803BB63BA6B7B6E9A607A6865
:10A788003B6803F122034FEA8303D3189B68DB6815
:10A798007B637B6B43F002037B637A683B6803F15E
:10A7A80022034FEA8303D3189B687A6BDA603B680D
:10A7B800DBB278681946FFF709FA7A683B68D3185C
:10A7C80003F564734FF005021A70C6E197F860301C
:10A7D80003F01003DBB2002B38D07B683A6802F133
:10A7E800C6024FF0000143F822107A683B6803F173
:10A7F80022034FEA8303D3189B68DB683B633B6BF8
:10A8080043F002033B637A683B6803F122034FEA93
:10A818008303D3189B683A6BDA603B68DBB27868CD
:10A828001946FFF7D3F94FF00003FB62FB6A43F0C8
:10A838001003FB62FA6A7B6E9A607A683B68D318E9
:10A8480003F564734FF003021A7086E197F86030DD
:10A8580023F07F03DBB2002B3ED07A683B6803F11C
:10A8680022034FEA8303D3189B68DB68BB62BB6A89
:10A8780043F00203BB627A683B6803F122034FEAA4
:10A888008303D3189B68BA6ADA603B68DBB27868DE
:10A898001946FFF79BF97B683A6802F1C60253F83C
:10A8A800223003F101017B683A6802F1C60243F8DD
:10A8B80022107A683B68D31803F564734FF00602D8
:10A8C8001A704FF000037B627B6A43F080037B625F
:10A8D8007A6A7B6E9A6040E197F8603003F0400333
:10A8E800DBB2002B38D07B683A6802F1C6024FF021
:10A8F800000143F822107A683B6803F122034FEA0B
:10A908008303D3189B68DB683B623B6A43F002030E
:10A918003B627A683B6803F122034FEA8303D3184A
:10A928009B683A6ADA603B68DBB278681946FFF7D9
:10A938004DF94FF00003FB61FB6943F04003FB61F5
:10A94800FA697B6E9A607A683B68D31803F564737A
:10A958004FF004021A7000E197F8613003F0040325
:10A96800DBB2002B3AD07A683B6803F122034FEA46
:10A978008303D3189B68DB68BB61BB6943F00203A0
:10A98800BB617A683B6803F122034FEA8303D3185B
:10A998009B68BA69DA603B68DBB278681946FFF7EA
:10A9A80015F94FF000037B617B6943F010037B616D
:10A9B8007A697B6E9A607A683B68D31803F564738A
:10A9C8004FF008021A704FF000033B613B6943F4F3
:10A9D80080633B613A697B6E9A60BEE097F86030AD
:10A9E80003F00203DBB2002B00F0B7807A683B6803
:10A9F80003F122034FEA8303D3189B68DB68FB60EB
:10AA0800FB686FF34103FB607A683B6803F122033C
:10AA18004FEA8303D3189B68FA68DA607A683B6860
:10AA2800D31803F564731B78DBB2012B22D17A6843
:10AA38003B68D31803F566734FF00102DA7197F893
:10AA48005A3003F00C03DBB2082B7CD17A683B68E0
:10AA58004FEA4313D31803F572735B7883F001034D
:10AA6800DAB279683B684FEA4313CB1803F572737F
:10AA78005A7068E07A683B68D31803F564731B78EA
:10AA8800DBB2032B08D17A683B68D31803F56673E9
:10AA98004FF00202DA7156E07A683B68D31803F582
:10AAA80064731B78DBB2042B1AD17A683B6803F114
:10AAB80015034FEA4313D31803F588731B79012B49
:10AAC80005D13B68DBB278681946FFF79CF87A68CD
:10AAD8003B68D31803F566734FF00202DA7132E06F
:10AAE8007A683B68D31803F564731B78DBB2052BCF
:10AAF80008D17A683B68D31803F566734FF00402EF
:10AB0800DA7120E07A683B68D31803F564731B7820
:10AB1800DBB2062B17D17B683A6802F1C60253F8FC
:10AB28002230032B0FD17A683B68D31803F566737C
:10AB38004FF00302DA717B683A6802F1C6024FF0FF
:10AB4800000143F822104FF00003BB60BB6843F0DC
:10AB58000203BB60BA687B6E9A604FF00103184627
:10AB680007F16807BD4680BD80B588B000AF786042
:10AB78004FF00003FB614FF00003FB604FF0000350
:10AB88003B614FF00003BB614FF000037B617B68C2
:10AB9800D3F8CC301B68BB617B68D3F8CC301B681A
:10ABA8007B617B696FF382037B617B696FF3410390
:10ABB8007B617B696FF3C3037B617B696FF345132B
:10ABC8007B613B7E03F00203DBB2002B0FD07B6975
:10ABD80043F002037B6140F20C23C2F200031B68BE
:10ABE8005B6878689847FB6943F00103FB613B7E2B
:10ABF80003F00803DBB2002B75D07B6943F0080330
:10AC08007B613B7E03F00403DBB2002B63D0BB7E89
:10AC180003F00603DBB2042B05D0BB7E03F006036A
:10AC2800DBB2022B35D17B685B691B683B61BB7E5D
:10AC380003F00603DBB2042B17D17B685B6941F292
:10AC480070725A603B7C03F00303DBB2022B24D002
:10AC58007B681B7A022B04D178684FF00201FEF75B
:10AC680017FE7868FEF74FFE17E07B685B694BF6C6
:10AC780080325A603B7C03F00303DBB2012B0CD01B
:10AC880078684FF00101FEF703FE7868FEF73BFE97
:10AC980003E07868FEF737FE00E000BF40F20C23BF
:10ACA800C2F200031B68DB68786898474FF000031E
:10ACB800FB60FB6843F00053FB607B68DB687A68E5
:10ACC800D26892691146FA686FEA02021140FA687E
:10ACD8000A439A6107E040F20C23C2F200031B68A2
:10ACE8001B69786898473B7E03F02003DBB2002B92
:10ACF80007D07B6943F020037B61FB6943F00103C4
:10AD0800FB617B68D3F8CC307A691A60FB69184616
:10AD180007F12007BD4680BD80B586B000AF7860DA
:10AD28007B685B691B69BB603B7BC3F3C303DBB216
:10AD38007A6803F11E034FEA4313D3181B6803F123
:10AD480003034FEA9303FB82A3E03B894FEA8303A3
:10AD5800BB82BA8A3B7BC3F3C303DBB2796803F1D6
:10AD68001E034FEA4313CB181B689A421DD93B7B3D
:10AD7800C3F3C303DBB27A6803F11E034FEA43133C
:10AD8800D3181B68BB824FF000033B613B6943F05B
:10AD980080633B617B68DB687A68D2689269114698
:10ADA8003A696FEA02020A409A613B7BC3F3C30324
:10ADB800DBB27A6803F11E034FEA4313D3181B680A
:10ADC80003F103034FEA9303FB823B7BC3F3C30303
:10ADD800DBB27A684FEA4313D31803F56F73196827
:10ADE8003B7BC3F3C303DBB21A46BB8A7868FEF722
:10ADF800E3FB3B7BC3F3C303DBB23A7BC2F3C3027F
:10AE0800D2B279684FEA42128A1802F56F72116855
:10AE1800BA8A8A1879684FEA4313CB1803F56F7317
:10AE28001A603B7BC3F3C303DBB23A7BC2F3C302B2
:10AE3800D2B2796802F11E024FEA42128A181168EA
:10AE4800BA8A8A1A796803F11E034FEA4313CB18AA
:10AE58001A603B7BC3F3C303DBB23A7BC2F3C30282
:10AE6800D2B2796802F11E024FEA42128A1802F140
:10AE780004021168BA8A8A18796803F11E034FEA36
:10AE88004313CB1803F104031A607B685B691B69E1
:10AE9800BB603B89FA8A9A420DD23B7BC3F3C3035A
:10AEA800DBB27A6803F11E034FEA4313D3181B6819
:10AEB800002B7FF44AAF4FF00103184607F118073B
:10AEC800BD4680BD80B588B000AF78607B68DB6820
:10AED800DB6AFB603B7CC3F3C303DBB27A6803F134
:10AEE8001E034FEA4313D3181B6803F103034FEA09
:10AEF8009303FB83A3E0BB894FEA8303BB83BA8B2D
:10AF08003B7CC3F3C303DBB2796803F11E034FEA4A
:10AF18004313CB181B689A421DD93B7CC3F3C30368
:10AF2800DBB27A6803F11E034FEA4313D3181B6898
:10AF3800BB834FF00003BB61BB6943F02003BB61D7
:10AF48007B68DB687A68D26892691146BA696FEAE9
:10AF580002020A409A613B7CC3F3C303DBB27A68FE
:10AF680003F11E034FEA4313D3181B6803F10303CD
:10AF78004FEA9303FB833B7CC3F3C303DBB27A68DA
:10AF88004FEA4313D31803F56F7319683B7CC3F377
:10AF9800C303DBB21A46BB8B7868FEF70DFB3B7C1C
:10AFA800C3F3C303DBB23A7CC2F3C302D2B27968FB
:10AFB8004FEA42128A1802F56F721168BA8B8A1822
:10AFC80079684FEA4313CB1803F56F731A603B7C1B
:10AFD800C3F3C303DBB23A7CC2F3C302D2B27968CB
:10AFE80002F11E024FEA42128A181168BA8B8A1AB5
:10AFF800796803F11E034FEA4313CB181A603B7CB0
:10B00800C3F3C303DBB23A7CC2F3C302D2B279689A
:10B0180002F11E024FEA42128A1802F10402116874
:10B02800BA8B8A18796803F11E034FEA4313CB18C9
:10B0380003F104031A607B68DB68DB6AFB60BB8989
:10B04800FA8B9A420DD23B7CC3F3C303DBB27A6816
:10B0580003F11E034FEA4313D3181B68002B7FF438
:10B068004AAF4FF00103184607F12007BD4680BDDF
:10B0780080B586B000AF78604FF000037B614FF079
:10B0880000033B617868FEF73BFC0346FB604FF02A
:10B0980000037B6134E0BB891A467B6942FA03F3FB
:10B0A80003F00103DBB2002B26D07A687B6903F139
:10B0B80022034FEA8303D3189B681B68BB607B7A23
:10B0C80023F07F03DBB2002B0BD049F6CD73C0F61B
:10B0D800000378687969984703463A6913433B61E6
:10B0E8000AE04AF2C953C0F60003786879699847BC
:10B0F80003463A6913433B617B6903F101037B61B2
:10B108007B681B781A467B699A42C4D83B69184603
:10B1180007F11807BD4680BD80B584B000AF7860E0
:10B128004FF00003FB604FF00003BB607868FEF748
:10B1380077FB0346002B00F08B807868FEF775FBE1
:10B148000346BB60BB68002B02D14FF0000380E0D0
:10B158003B7A03F00803DBB2002B09D049F63953D8
:10B16800C0F60003786898470346FA681343FB6003
:10B178003B7A03F01003DBB2002B09D049F60563D4
:10B18800C0F60003786898470346FA681343FB60E3
:10B198003B7A03F02003DBB2002B09D04AF6CD63DB
:10B1A800C0F60003786898470346FA681343FB60C3
:10B1B800FB7A03F00403DBB2002B09D04AF62153D3
:10B1C800C0F60003786898470346FA681343FB60A3
:10B1D800FB7A03F00203DBB2002B09D04BF27903B0
:10B1E800C0F60003786898470346FA681343FB6083
:10B1F800FB7A03F00103DBB2002B09D04AF6713366
:10B20800C0F60003786898470346FA681343FB6062
:10B21800FB7A03F02003DBB2002B09D049F6755303
:10B22800C0F60003786898470346FA681343FB6042
:10B23800BB7A03F02003DBB2002B09D049F6B153E7
:10B24800C0F60003786898470346FA681343FB6022
:10B25800FB68184607F11007BD4680BD0123C0F8FA
:10B268001033002070470123C0F8143300207047C2
:10B278000023C0F81433184670470020704738B5CB
:10B2880004460021FDF79DFEE36800254FF0FF32DC
:10B298009D6120465A61FEF762FAC4F810532846A9
:10B2A80038BD70B50123002540220C46CB700B77C2
:10B2B8008A7181F8213006460D704D708D7081F8C5
:10B2C8002050097900F02BFB6179304600F027FB0C
:10B2D800284670BD2DE9F041069F1646984604465B
:10B2E8000D46FDF7FAFD0020FDF77AFE31462046AF
:10B2F800FFF7D7FF2946C6F87C80C6F8807020463D
:10B30800FEF7B6FCD6F880301B6898472046BDE8A3
:10B31800F041FDF743BE0B1FDBB2012B10B504460D
:10B3280006D8D0F880305B6C98470B23237010BD8B
:10B33800062905D10B230370D0F880301B68984785
:10B3480010BD002370B58B740B7F013B05460C467E
:10B358000A2B00F2C980DFE813F00B001200390055
:10B36800400058006500790080009900A900B900E4
:10B3780001F11401627900F03BFD022343E04979B1
:10B38800FEF7B8FC012819D1237D618B584A03F0D8
:10B39800800339B141F2883111800BB1032307E0F2
:10B3A800052305E0322111800BB1092300E00723B2
:10B3B80023772846FEF79AFC208295E0032840F080
:10B3C80093800B2323770523A3748DE00B798A8957
:10B3D800896800F044FD042315E00979FEF78AFC2A
:10B3E800012802D10923237703E0042823D0032866
:10B3F80008D02846FEF77AFC238AC01A3C4B1B88E3
:10B40800984271D90B2323776EE04B7900EB4313F5
:10B41800012283F8C9234B798A89896800F0FDFCE9
:10B428000623F0E74979FEF765FC012801D10723D7
:10B43800E9E7042803D1637823700C23E3E70228A3
:10B4480001D10523DFE703284ED1DBE70B79002183
:10B458000A4600F004FD0823D5E70979FEF74AFCFF
:10B468000128064627D00328CCD02846FEF73EFC04
:10B47800238AC01A1E4B1B889842C3D8042E33D186
:10B48800637823700C232377032070BD4B7900EB7E
:10B49800431393F8C92382F0010283F8C9234B7937
:10B4A80000210A4600F0B9FC0A23ACE74979FEF707
:10B4B80021FC012803D1637823700D23A3E7022818
:10B4C80001D109239FE7032810D19BE78B7B013328
:10B4D800DBB2022B8B7301D8012394E708238B740A
:10B4E8004B7802200B7070BD002070BD002070BD2D
:10B4F800A80C002070B594B0022305460C468DF8C0
:10B508004F30FEF7EDFB18B12846FEF7ECFB28B9E3
:10B5180023781BB1032B01D00323237023780B2B33
:10B5280000F29181DFE813F00C001F0026006D0186
:10B538008F01580040014C01590131018F015E0112
:10B548002846FEF7CDFB002800F07D8101232370FB
:10B55800C820FDF743FD2846FEF7BDFBD4F8803030
:10B56800DB6898476FE1D5F81433012B40F06B8105
:10B57800022367E1D4F880309B6898470021284669
:10B5880000F0B4F980216071284600F0AFF920710D
:10B598002846FEF79AFB0523C0B22370D4F8803002
:10B5A80084F821009B699847A079217994F8202094
:10B5B80094F82130019000262846009600F048F9BA
:10B5C800A0796179019094F8202094F821300096B0
:10B5D800284600F03DF936E1A378092B00F23381C3
:10B5E800DFE813F00A002800380060006B007F00D5
:10B5F8009800B100C9002B0128462146082200F016
:10B608001DFD0646002840F01E8194F82930617916
:10B61800A3710122A2700090019332463346284656
:10B6280000F043F9A3792179019300962846324620
:10B63800334634E028462146122200F0FFFC002859
:10B6480040F00181D4F8803004F12200DB6998478A
:10B65800022330E028462146012200F045FD064637
:10B66800002840F0F0800220FDF7B8FC012384F8A0
:10B678002030D4F880301B6A98470323A3702179BF
:10B6880094F82020009633462846019600F00DF9DC
:10B69800617994F82020009601962846334600F0F8
:10B6A80004F9D0E028462146092200F019FE0028B6
:10B6B80040F0C9800423A370C5E0E28E28462146E5
:10B6C80000F00EFE002840F0BE80D4F8803004F16F
:10B6D80034005B6A04F13E0104F1500298470523E7
:10B6E800E9E794F8302072B1FF23009328462146F9
:10B6F80003AB00F07BFC002840F0A580D4F8803034
:10B7080003A89B6A03E0D4F8803050489B6A9847A6
:10B718000623D0E794F8312072B1FF23009328461E
:10B72800214603AB00F062FC002840F08C80D4F87E
:10B73800803003A8DB6A03E0D4F880304348DB6A32
:10B7480098470723B7E794F832206AB1FF2300939C
:10B758002846214603AB00F049FC002873D1D4F8F1
:10B76800803003A81B6B03E0D4F8803037481B6B8C
:10B77800984708239FE794F839202846214600F087
:10B78800C0FC00285FD1092395E7D4F880309B6B73
:10B798009847012857D1E36F28461B6821469847E8
:10B7A800002850D106234DE0E36F28469B682146C8
:10B7B80098478DF84F009DF84F3043B9072341E073
:10B7C800E36F2846DB68214698478DF84F009DF8BF
:10B7D8004F102046FFF79FFD35E028462146FFF72A
:10B7E800B0FD30E021462846FFF75BFDD4F88030F5
:10B7F8005B689847E36F04F120015B682846984727
:10B8080021E0D4F880301B69984721462846FFF785
:10B8180048FDD4F880305B689847E36F04F1200155
:10B828005B6828469847284600F085F8002323706F
:10B8380028460121FEF71CFA05E0D4F880305B6B3E
:10B8480098470923237014B070BD00BFE5A405080C
:10B85800F8B501F5327430F8146001F1150400EB05
:10B86800441406F07F0784F810219DF8182084F806
:10B87800117184F81521BDF81C2084F81331A4F83F
:10B888001621C6F3C01600EB411204F5887584F83A
:10B898001261002482F8C84382F8C9430BB9012316
:10B8A8002B71FEF791F80020F8BD70B5BDF8144073
:10B8B8001AB100EB411585F8B02301F1150200EB30
:10B8C8004215B5F81661A64205F5887501D004B190
:10B8D800EC8000EB421292F813419C4202D00BB16B
:10B8E80082F81331FEF770F8002070BD10B50246DB
:10B8F8000023B2F99045002C08DB03F532726FEA99
:10B9080041416FEA514120F8121006E00133DBB2E1
:10B918000232082BEDD14FF6FF73D8B210BD0729BC
:10B9280007D801F5327130F8113023F4004320F8BC
:10B938001130002070470023A0F89435A0F8963500
:10B94800A0F89835A0F89A35A0F89C35A0F89E354F
:10B9580018467047F8B5314D95F8423006460F46FF
:10B96800052B58D8DFE803F00357571309272B6D29
:10B978001B689847042385F842303046FDF75DFF81
:10B98800012848D1254B032283F8422043E095F84B
:10B99800462095F84030214900F0A3FA204B0122B7
:10B9A8001A703046052385F84230FEF79FF980B2B9
:10B9B800A5F84C002FE0FEF799F9B5F84C30174C74
:10B9C8009BB2C01AB5F84A30984221D294F8401078
:10B9D8003046FEF78FF901280AD1114B1A78012A4F
:10B9E80019D100221A70236D20465B68984712E02F
:10B9F80094F840103046FEF77DF904280BD194F8EE
:10BA0800482094F840303046394600F095FB10B98C
:10BA1800032384F842300020F8BD00BF888E002040
:10BA2800AA0C0020384B93F8453073B50446042B14
:10BA380066D8DFE803F003320340530000F588734B
:10BA480000930923019301224FF4045300F0B4FA40
:10BA5800002855D12D4B94F8102194F813111A7021
:10BA680094F811215A7094F8122102EB01225A809D
:10BA780094F8142194F818111A7194F815215A7130
:10BA880094F816219A7194F8172102EB01221A8171
:10BA98001D4B012083F8450035E000F588730093BD
:10BAA8001A4B1B89012201934FF4085300F084FAC2
:10BAB80030BB03220EE0212300220B750A234B75AD
:10BAC800CA820A834A83134600F06CF908B1032836
:10BAD80016D104220C4B83F8452011E021230022C3
:10BAE8000B7501250B234B75CD820A834A831346B8
:10BAF800164600F057F928B9034B83F8456002E071
:10BB0800012000E028467CBD888E0020DC8E0020C5
:10BB180038B5114D95F84010044649B1FEF756F86E
:10BB280095F840102046FFF7FAFE002385F84030CC
:10BB3800094D95F8411051B12046FEF747F895F8A0
:10BB480041102046FFF7EBFE002385F84130034BF8
:10BB580000221A7038BD00BF888E0020AA0C002071
:10BB68002DE9F347344B062283F8422091F844200C
:10BB7800012A07460C4658D191F84520012A04BFEE
:10BB88002E4A1A65002283F8422083F8452091F84E
:10BB9800522083F84820B1F85420A3F8462091F8A1
:10BBA8005620092AA3F84A2003D8234B0A22A3F8CF
:10BBB8004A2094F842A0204DBAF1020F28BF4FF056
:10BBC800020A26464FF000084FF0030927E096F8CE
:10BBD80052100B0608D5384685F84410FFF786FE44
:10BBE800014685F8400009E085F8431096F85210A0
:10BBF8003846FFF77BFE014685F84100B5F8460058
:10BC080094F82020019094F82130CDF8009038461F
:10BC1800FFF71EFE08F101085FFA88F80836D045DC
:10BC2800D5D1074B0020187004E0D1F880301B6C88
:10BC380098470120BDE8FC87888E00203402002048
:10BC4800AA0C002030B543EA02229DF80C40CA82B3
:10BC580021250023049A0D750B83092523464D756C
:10BC68004C83BDE8304000F09DB800BF70474A4A99
:10BC780000232DE9F047137053709370D370054675
:10BC88001A46E918013389780139C9B2022998BFDF
:10BC98000122062BF5D1012A7CD03F4991F802C038
:10BCA8000A784B782846022601F10A098778BFB13D
:10BCB8008C1801322771D2B2002406E0013409EB56
:10BCC800040A1AF801ACBA4503D05FFA84F8E045D3
:10BCD800F4D3E04504D1CC18877801332774DBB25C
:10BCE8000136F6B20130082EE0D12B4C012B227020
:10BCF800637041D1207CE070FDF757FA2B78102B48
:10BD08001BD022460AD8022B1BD003D89BB1012B8B
:10BD18001DD112E0042B16D0052B0AE0402B12D0BF
:10BD280004D8142B11D0202B11D10AE0412B0CD0B0
:10BD3800502B0CD109E0A37509E0174B02229A7524
:10BD480005E0012302E0032300E004239375124A6F
:10BD5800937DD178114A012B05D803EB4103D05CC0
:10BD6800FDF718FA0AE0032000FB013102EB81021B
:10BD7800D2F8C030984701E00023E370064A1378F0
:10BD880002F10A01937000230432985C585401337D
:10BD9800062BFAD1BDE8F087AB0C0020D09A040836
:10BDA800FDF7F6B9C878012810B504D002284FF07D
:10BDB800010319D108E00C788B814C7008240C70B1
:10BDC8008A600877022308E00A7F0D2A03D1002041
:10BDD800CB70087710BD0B2A01D1CB7010BD0C2A8F
:10BDE80004D1CB70032010BD184610BD184610BDF5
:10BDF80000EB421310B5002483F8B24300EB421362
:10BE08000324C3F8BC130821C3F8C01383F8B8434C
:10BE18001146FDF780FFC0B210BD38B500EB4314E2
:10BE2800002584F8B2535C010519C5F8BC1300EB72
:10BE38004311C1F8C02312B9012285F8C923041996
:10BE480000EB431294F8C913002914BF0221002102
:10BE580082F8B8131946FDF75EFF002038BD38B5E3
:10BE680000EB4314012584F8B2530225C4F8BC132F
:10BE780084F8B853C4F8C0231946FDF74CFF0020D6
:10BE880038BD38B500EB4315002485F8B24300EB04
:10BE98004315C5F8C02395F8C923C5F8BC13A242B9
:10BEA80014BF0222224685F8B8231946FDF733FF4E
:10BEB800204638BD38B500EB43140125C4F8C0232B
:10BEC80094F8C823C4F8BC13002A14BF0222002225
:10BED80084F8B25384F8B8231946FDF71CFF0020F4
:10BEE80038BDF8B504461F460E46154602201A46C8
:10BEF8000E49FDF757F904EB4713012283F8B223E3
:10BF080093F8C823C3F8BC63002A14BF0221002198
:10BF180082F0010283F8B813C3F8C05383F8C8232A
:10BF280020463946FDF7F7FE0020F8BDE9A40508CC
:10BF380038B500EB4315002485F8B24300EB4315F0
:10BF4800C5F8C02395F8C823C5F8BC13A24214BF8E
:10BF58000221214682F0010285F8B81385F8C8232A
:10BF68001946FDF7D8FE204638BD38B500EB431416
:10BF7800012584F8B2532546C4F8BC13C4F8C0237D
:10BF8800002485F8B8431946FDF7C5FE204638BD9C
:10BF980038B500EB4315002485F8B24300EB431590
:10BFA800C5F8BC13C5F8C02385F8B8431946FDF792
:10BFB800B2FE204638BD00BF10B562F07F020A7598
:10BFC8000622BDF80C404A75CB8240F2094203F4C0
:10BFD8007F43B3F5407F0CBF13460023029A0B83BF
:10BFE80023464C83BDE81040FFF7DCBE73B5BDF8AF
:10BFF80018601D4642F4407300F588728DE84400CD
:10C0080000220446FFF7D8FFB8B994F81131032B82
:10C0180013D194F81031023B9E42A8BF1E46B6B217
:10C02800034606E0E218023392F8122105F8012BC4
:10C038009BB2B342F6D300232B707CBD73B500F5D9
:10C04800887316468DE8480000224FF48073044632
:10C058000D46FFF7B1FF002845D194F8103185F857
:10C06800223094F8113185F8233094F8132194F88C
:10C07800123103EB0223AB8494F8143185F826308F
:10C0880094F8153185F8273094F8163185F828305A
:10C0980094F81731082E85F8293024D994F81921F5
:10C0A80094F8183103EB02236B8594F81B2194F85C
:10C0B8001A3103EB0223AB8594F81D2194F81C3147
:10C0C80003EB0223EB8594F81E3185F8303094F8A1
:10C0D8001F3185F8313094F8203185F8323094F8E2
:10C0E800213185F833307CBD10B500230524CA8280
:10C0F8001A460B754C750B834B83BDE81040FFF750
:10C1080051BE10B500230924CA821A460B754C7516
:10C118000B834B83BDE81040FFF744BE10B50A837C
:10C12800012400220C75CB820B2413464C754A83DC
:10C13800BDE81040FFF736BE30B54FEA431302247E
:10C148000C75C31801244C75002412F0800F0A8363
:10C15800CC824C8314BF83F8C84383F8C9430022B8
:10C1680025461346BDE83040FFF71CBE2DE9F04FC9
:10C1780093461A7802705A7889B042709A78069174
:10C18800D97802EB012242801A79027159794171FA
:10C1980099798171D979C171197A0172BDF84810FC
:10C1A800092940F29480022A00F293804B4A09211F
:10C1B80092F800C0548881E01A789B1889185A7838
:10C1C800042A89B27AD19E7893F803A0069F09259C
:10C1D8004FFA86F8BAF1020F05FB08726ED81D787F
:10C1E8001F7900955D7901959D790295DD79039513
:10C1F8001D7A022F049504D9384B83F800C05C805F
:10C2080067E04FEA48050595CDF81C800025814672
:10C2180050E018781B1809185878052889B249D1B0
:10C228000798844511D000989670107004205070BB
:10C23800019882F803A050710298177190710398C1
:10C24800D0710498B446107216E0187993F80580F6
:10C2580000EB0820844230DC0098967010700420AF
:10C268005070019882F803A050710298177190716C
:10C278000398D07104981072059893F8008040FADA
:10C2880085F40BEBC4000BF834805C7844709C7820
:10C298008470DC78C47093F805801C7904EB08245A
:10C2A80084809C7984715C791879013500EB0424C9
:10C2B800A4B2EDB268B2B842ABDB484642888A42C3
:10C2C8003FF67AAF054B00205880187002E0002036
:10C2D80000E0032009B0BDE8F08F00BFC20C0020C9
:10C2E800F7B54FF4007300F58877019215460022E0
:10C2F80006460C460097FFF75FFE034633B113E08E
:10C30800F11891F810119954013300E0074A99B2D5
:10C31800A942F5D304F1340004F13E0104F15002BE
:10C328003B460095FFF722FFFEBD00BFEE8E0020C2
:10C3380003780A88D3180B800378C018704700BFA9
:10C34800036823F0010303600023036043608360F4
:10C35800C3600361212343612C4B98421CD02C4BB2
:10C36800984220D02B4B984225D02B4B98422AD06C
:10C378002A4B98422FD02A4B984233D0294B9842C7
:10C3880037D0294B984204D14FF03D5243F8AC2C9A
:10C398007047264B984203D13D2243F8082C70473A
:10C3A800234B984204D14FF4746243F8202C704711
:10C3B800204B984204D14FF4741243F8382C70473C
:10C3C8001D4B984204D14FF0746243F8502C7047CB
:10C3D8001A4B984203D11A4A43F8642C7047194BF8
:10C3E800984203D1184A43F87C2C7047174B98425F
:10C3F80003D1174A43F8942C7047164B984204BF50
:10C408004FF03D5243F8AC2C704700BF106002401B
:10C41800286002404060024058600240706002405C
:10C4280088600240A0600240B86002401064024088
:10C43800286402404064024058640240706402402C
:10C448003D00002088640240400F0020A0640240A4
:10C4580000003D20B86402400268134B10B5134039
:10C46800CC680A6822434C6922438C692243CC6910
:10C4780022430C6A22434C6A22438C6A22434C6B47
:10C4880022438C6B22431343036042690C6BCB6AD3
:10C4980022F007022343134343610B6943604B684F
:10C4A80083608B68C36010BD3F801CF0002303606D
:10C4B80043608360C360036143618361C361036256
:10C4C80043628362C36203634363836370470368A1
:10C4D80011B143F0010301E023F001030360704749
:10C4E800036811B143F4004301E023F400430360FF
:10C4F8007047036811B143F0200301E023F02003E3
:10C508000360704741607047406880B270470368B5
:10C5180012B143F4002301E023F400230360016116
:10C528007047036811B143F4802301E023F48023AA
:10C53800036070470AB101617047C16070470068C5
:10C54800C0F3C0407047006800F0010070474069C0
:10C5580000F0380070470A4A0A4B10B50A4CA0424E
:10C5680088BF13468A004CBF5B681B6821F0F02126
:10C5780021F0821119420CBF0020012010BD00BF1C
:10C5880000640240006002400F64024010B5084B8E
:10C59800084A094CA04288BF134611F0005F21F0F9
:10C5A800F02121F0821114BFD960996010BD00BF3D
:10C5B80000600240006402400F6402400B0607D589
:10C5C800436912B143F0800301E023F08003436123
:10C5D800802909D001F01E01036812B119430160D6
:10C5E800704723EA010101607047124B124A10B5E7
:10C5F800124CA0428CBF14461C4621F0F02323F0B5
:10C60800C3132BB1026802F01E0202EAD12202E033
:10C61800426902F0800288004CBF6368236821F0F9
:10C62800F02121F08210184002D0101C18BF012000
:10C6380010BD00BF00600240006402400F64024069
:10C6480010B5084B084A094CA04288BF134611F0A0
:10C65800005F21F0F02121F0821114BFD9609960A8
:10C6680010BD00BF00600240006402400F64024039
:10C67800044B00221A605A609A60DA60024A5A61D2
:10C68800704700BF003C0140FFFF7F00837910B571
:10C69800002B29D01A4B01681C68CA4314401C603F
:10C6A8005C6822405A60027902F1804202F59E32AB
:10C6B80014682143116002689C68D1430C409C6057
:10C6C800DC682140D9604179102906D19968114365
:10C6D8009960D9680A43DA6010BD01F1804303F517
:10C6E8009E3319680A4308E00379016803F180431F
:10C6F80003F59E331A6822EA01021A6010BD00BFD2
:10C70800003C014000230C220360037142718371D5
:10C718007047024B1A6902431A617047003C014096
:10C72800034B5B6918420CBF00200120704700BF13
:10C73800003C0140014B5861704700BF003C01407C
:10C74800054B1A685B69034004D010420CBF0020F7
:10C758000120704718467047003C0140014B586162
:10C76800704700BF003C01404FF0204318B943F226
:10C77800DB021A6003E043F2D20243F820204FF0B4
:10C788002042411C6FF0704342F8213002F582725A
:10C7980042F82030704770B584684568C368C16A3C
:10C7A800026825431D4303691D4343691D4383698B
:10C7B8001D43C3691D43036A1D43436A1D43836ABE
:10C7C8001D43036B0D431D434FF02043082C43F8D2
:10C7D800225005D153F8224044F0400443F8224047
:10C7E800436B9E691D6835435E6845EA06159E6879
:10C7F80045EA0625DE6845EA06451E695B6945EA9D
:10C808000655541C45EA03654FF02043B1F5804FA7
:10C8180043F8245010D1836B98691968014358680C
:10C8280041EA0011986841EA002118695B6941EA08
:10C83800005141EA036101E06FF07041014B43F898
:10C84800221070BD040100A0022242604FF4805201
:10C858004262416B4FF4005210B5826200230F22EE
:10C86800FF2403608360C360036143618361C36124
:10C878000362C36203630A604A608C60CA600A612B
:10C888004A618B61816B0A604A608C60CA600A6188
:10C898004A618B6110BD4FF0204321B153F820202D
:10C8A80042F0010203E053F82010024A0A4043F81C
:10C8B80020207047FEFF0F0010280CBF064B074BC7
:10C8C8004FF040024FF0180119605A604FF0FC32E7
:10C8D8009A60DA60704700BF600000A0800000A086
:10C8E80030B5836844681C43C36844F008041C439B
:10C8F80003691C43436944EA4324836944EA433493
:10C90800C36999685A68090441EA02211A68DB6810
:10C91800114341EA0361036A9A685D68120442EAB6
:10C9280005221D68DB682A4342EA03620368102B6C
:10C938000CBF034B034B1C609960DA6030BD00BF2D
:10C94800600000A0800000A010230360C2690023DB
:10C9580043608360C360036143618361FC231360A8
:10C9680053609360D360026A136053609360D3602E
:10C97800704741B110280CBF074B084B1A6842F0AA
:10C9880004021A60704710280CBF034A034A044B7C
:10C9980011680B4013607047600000A0800000A081
:10C9A800FBFF0F0041B110280CBF084B084B1A6859
:10C9B80042F040021A60704710280CBF034A044A2C
:10C9C800044B11680B401360704700BF600000A063
:10C9D800800000A0BFFF0F00102802D1024B586949
:10C9E8007047024B58697047600000A0800000A0A3
:10C9F800054B18221A6000225A604FF0FC329A60E8
:10CA0800DA601A61704700BFA00000A0026843689E
:10CA180042F0100242EA4322836842EA4332144B4E
:10CA280010B51A60C26891685468090441EA042183
:10CA38001468D268214341EA02629A6002699168E7
:10CA48005468090441EA04211468D268214341EA80
:10CA58000262DA60426991685068090441EA00217B
:10CA68001068D268014341EA02621A6110BD00BF32
:10CA7800A00000A0C2680023036043608360FC2319
:10CA8800136053609360D3600269136053609360CE
:10CA9800D3604269136053609360D3607047054B5D
:10CAA80018B11A6842F0040202E01968024A0A4002
:10CAB8001A607047A00000A0FBFF0F0062B11028A9
:10CAC80001D10E4B03E0B0F5807F03D10C4B5A68BF
:10CAD800114311E00B4BFAE7102804D1074B5A68B1
:10CAE80022EA010108E0B0F5807F0CBF044B054B3A
:10CAF8005A686FEA0101114059607047600000A050
:10CB0800800000A0A00000A0102801D1064B04E07E
:10CB1800B0F5807F0CBF054B054B5B680B420CBF23
:10CB280000200120704700BF600000A0800000A026
:10CB3800A00000A0102804D1074B5A6822EA01017E
:10CB480008E0B0F5807F0CBF044B054B5A686FEACC
:10CB58000101114059607047600000A0800000A0EA
:10CB6800A00000A0102801D1084B04E0B0F5807F98
:10CB78000CBF074B074B5B6813EA010004D013EAAC
:10CB8800D1010CBF00200120704700BF600000A049
:10CB9800800000A0A00000A0102804D1084B5A680B
:10CBA80022EAD10109E0B0F5807F0CBF054B064BA6
:10CBB8005A684FEAD10122EA01015960704700BF63
:10CBC800600000A0800000A0A00000A008B52C4BC9
:10CBD800984205D10120014600F048FC012048E0B8
:10CBE800284B984205D10220012100F03FFC022089
:10CBF8003FE0254B984205D10420012100F036FC86
:10CC0800042036E0214B984205D10820012100F08C
:10CC18002DFC08202DE01E4B984205D11020012143
:10CC280000F024FC102024E01A4B984205D1202063
:10CC3800012100F01BFC20201BE0174B984205D176
:10CC48004020012100F012FC402012E0134B9842D2
:10CC580005D18020012100F009FC802009E0104B5B
:10CC680098420BD14FF48070012100F0FFFB4FF484
:10CC780080700021BDE8084000F0F8BB08BD00BF87
:10CC8800000002400004024000080240000C02407C
:10CC9800001002400014024000180240001C02402C
:10CCA800002002402DE9F0470023D1F800801A4601
:10CCB8004FF0010C03270CFA02F404EA0805A54218
:10CCC8002ED1066817FA03F4E443264006600E796D
:10CCD800D0F8009006FA03FA013E4AEA0909012E43
:10CCE800C0F8009014D8866891F8059026408660B0
:10CCF800866809FA03F949EA06068660466826EA5C
:10CD0800050545608D7946689540ADB23543456067
:10CD1800C5682C40C460CC79C5689C402C43C4606D
:10CD280001320233102AC6D1BDE8F0874FF6FF73EF
:10CD380003600023037143718371C371704782B02C
:10CD48004FF480330193019B0B430193019BC36113
:10CD5800C161019BC361C3690193C369019302B0B7
:10CD68007047036919420CBF002001207047006911
:10CD780080B27047436919420CBF002001207047F8
:10CD8800406980B2704701837047418370470AB198
:10CD980001837047418370474161704743694B4045
:10CDA8004361704701F00703C908083130B59B009B
:10CDB80050F821500F249C4025EA040440F82140F3
:10CDC80050F8214012FA03F31C4340F8214030BDCB
:10CDD80008B5134B984207D14FF40010012100F019
:10CDE80069FB4FF4001014E00E4B984207D14FF442
:10CDF8008000012100F05EFB4FF4800009E00A4B3F
:10CE080098420BD14FF40000012100F053FB4FF47E
:10CE180000000021BDE8084000F04CBB08BD00BF81
:10CE28000054004000580040005C00407FB50446B4
:10CE3800868868460D4600F06DFA02992C482B68E2
:10CE480026F03F063604B1FBF0F0360C80B20643FC
:10CE5800A680228822F001021204120C2280254AA0
:10CE680093420AD85B00B1FBF3F301309BB280B266
:10CE78002084032B98BF042321E0EE884BF6FF7231
:10CE8800964205D103225343B1FBF3F39BB206E06C
:10CE980019225343B1FBF3F39BB243F480431A05C1
:10CEA8004FF4967208BF43F0010350434FF47A726F
:10CEB80090FBF2F0013080B243F400432084A38356
:10CEC80023886989AA889BB243F0010323802388B9
:10CED80023F4816323F002031B040A431B0C13434E
:10CEE8009BB223802A89AB8913439BB223817FBDE0
:10CEF80040420F00A086010041F2883303600023FE
:10CF080083804BF6FF72038143814FF48043C280D4
:10CF180083817047038819B19BB243F0010303E092
:10CF280023F001031B041B0C03807047038819B10D
:10CF38009BB243F4807303E023F480731B041B0C3F
:10CF480003807047038819B19BB243F4007303E070
:10CF580023F400731B041B0C0380704712B141F0CB
:10CF6800010101E001F0FE0101827047038819B157
:10CF78009BB243F4806303E023F480631B041B0C1F
:10CF88000380704783899BB201F0FE0123F0FE0302
:10CF98000B4383817047838919B19BB243F0010326
:10CFA80003E023F001031B041B0C838170470388F3
:10CFB80019B19BB243F0400303E023F040031B0484
:10CFC8001B0C03807047038829B16FEA43436FEA5B
:10CFD80053439BB201E05B045B0C038070470388FA
:10CFE80019B99BB243F0800303E023F080031B04CC
:10CFF8001B0C03807047B1F5804F838B04D023F45A
:10D0080080431B041B0C02E09BB243F480438383E0
:10D018007047B1F5006F038803D19BB243F40063F6
:10D0280003E023F400631B041B0C03807047B1F575
:10D03800005F038803D19BB243F4005303E023F459
:10D0480000531B041B0C03807047038819B19BB263
:10D0580043F0100303E023F010031B041B0C0380B0
:10D06800704701827047008AC0B27047038819B1BF
:10D078009BB243F4805303E023F480531B041B0C3E
:10D0880003807047B1F5006F038803D19BB243F466
:10D09800006303E023F400631B041B0C0380704748
:10D0A800038819B19BB243F0200303E023F0200367
:10D0B8001B041B0C03807047008BC0F307207047CC
:10D0C800838819B19BB243F4006303E023F400633F
:10D0D8001B041B0C83807047838819B19BB243F4EF
:10D0E800805303E023F480531B041B0C8380704798
:10D0F80082B0002301930190019BCB180193019BFF
:10D10800188880B202B0704783889BB20AB119436D
:10D1180001E023EA010181807047838A008B9BB27A
:10D1280043EA0040084020F07F40431A584240EB51
:10D1380003007047838A008B9BB243EA004020F0CB
:10D148007F40704782B00023009301930B0F01903A
:10D158000093009B21F07F4113B1019B143302E03F
:10D16800019B090C18330193019B1B6819420CBFE2
:10D178000020012002B07047C94389B281827047FC
:10D188008388808A80B208409BB206D001F0E061B3
:10D1980013EA11410CBF002001207047C94389B22E
:10D1A800818270470A4B1A6842F001021A60002215
:10D1B8009A60196821F0847121F480311960054959
:10D1C8005960196821F480211960DA60704700BF3E
:10D1D8000038024010300024024B00221A701870E8
:10D1E800704700BF02380240034B1A6822F0F80269
:10D1F80042EAC0021A60704700380240014B1860CA
:10D20800704700BF00004742064B002201281A70F1
:10D218001A7002D0042804D101E018707047052262
:10D228001A70704770380240014B1860704700BF91
:10D23800800E4742014341EA821200995B08013B94
:10D2480042EA016141EA0341014B5960704700BF5E
:10D2580000380240014B1860704700BF6000474229
:10D268008001034B40EA0171C3F88410704700BF86
:10D2780000380240014B1860704700BF6800474201
:10D28800014B1860704700BF4C004742034B9A6837
:10D2980022F0EC6202430A439A6070470038024069
:10D2A800034B9A6822F0784202430A439A60704717
:10D2B80000380240034B9A6822F0030202439A6046
:10D2C800704700BF00380240024B986800F00C001D
:10D2D800704700BF00380240034B9A6822F0F00202
:10D2E80002439A60704700BF00380240034B9A68B7
:10D2F80022F4E05202439A60704700BF00380240AF
:10D30800034B9A6822F4604242EAC0029A6070476E
:10D31800003802401E4B9A6802F00C02042A10B52D
:10D3280003D0082A03D01B4B18E01B4B16E05968A2
:10D338005A6811F4800F596814BF174B154B02F047
:10D348003F02B3FBF2F3124A5268C2F30142C1F33F
:10D35800881101324B435200B3FBF2F30C490360CE
:10D368008B680E4A0468C3F30313D35C34FA03F3DF
:10D3780043608C68C4F38224145D33FA04F4846037
:10D388008968C1F34231525CD340C36010BD00BF0D
:10D39800003802400024F40000127A003C02002009
:10D3A80000F44073B3F5407F084B08D1996820F02A
:10D3B800704221F4F81122F440720A439A601A6FFD
:10D3C800000542EA10501867704700BF0038024055
:10D3D800014B1860704700BF3C0E4742014B186074
:10D3E800704700BF400E4742014B1860704700BFAE
:10D3F8005C014742044B1A6B09B1104301E022EA71
:10D4080000001863704700BF00380240044B5A6B95
:10D4180009B1104301E022EA00005863704700BFD9
:10D4280000380240044B9A6B09B1104301E022EA2C
:10D4380000009863704700BF00380240044B1A6C24
:10D4480009B1104301E022EA00001864704700BFE8
:10D4580000380240044B5A6C09B1104301E022EA3B
:10D4680000005864704700BF00380240044B1A6936
:10D4780009B1104301E022EA00001861704700BFBB
:10D4880000380240044B5A6909B1104301E022EA0E
:10D4980000005861704700BF00380240044B9A6989
:10D4A80009B1104301E022EA00009861704700BF0B
:10D4B80000380240044B1A6A09B1104301E022EA1D
:10D4C80000001862704700BF00380240044B5A6AD7
:10D4D80009B1104301E022EA00005862704700BF1A
:10D4E80000380240044B1A6D09B1104301E022EAEA
:10D4F80000001865704700BF00380240044B5A6DA1
:10D5080009B1104301E022EA00005865704700BFE6
:10D5180000380240044B9A6D09B1104301E022EA39
:10D5280000009865704700BF00380240044B1A6E2F
:10D5380009B1104301E022EA00001866704700BFF5
:10D5480000380240044B5A6E09B1104301E022EA48
:10D5580000005866704700BF00380240044B1A7834
:10D5680009B1104301E022EA00001870704700BFBB
:10D578000D3802404309012B074A01D1136803E023
:10D58800022B0CBF136F536F00F01F0033FA00F02B
:10D5980000F00100704700BF0038024007B50023C3
:10D5A80001933120FFF7E6FF019B01330193019BB3
:10D5B800B3F5A06F01D00028F3D03120FFF7DAFFD0
:10D5C800003018BF01200EBD024B5A6F42F0807226
:10D5D8005A67704700380240034BDB6818420CBF9B
:10D5E80000200120704700BF00380240014B18702E
:10D5F800704700BF0E38024008B5154B98420BD152
:10D6080001214FF48050FFF761FF4FF48050002153
:10D61800BDE80840FFF75ABF0E4B984207D14FF4B8
:10D6280080400121FFF746FF4FF4804009E00A4B94
:10D6380098420BD14FF400400121FFF73BFF4FF414
:10D6480000400021BDE80840FFF734BF08BD00BF17
:10D658000030014000380040003C00400B88028840
:10D6680010B54C8823438C882343CC8823430C89EA
:10D6780023434C8923438C892343CC8902F44152A8
:10D68800234313439BB20380838B23F400631B045F
:10D698001B0C83830B8A038210BD838B23F47B636B
:10D6A80023F00F031B041B0C8383022303848B6862
:10D6B800F0B5858B022BADB238D0294A8E88946894
:10D6C800002E14BF02260126240203D5946824F4F0
:10D6D80000049460D2F88440D2F884705268DFF86D
:10D6E80084C002F03F02BCFBF2F2C4F38814544336
:10D6F800C7F30272B4FBF2F4CA88B2F5007F4FF0A8
:10D708000A0201D1240A02E07601B4FBF6F462436E
:10D71800B2FBF3F305330A229BB2B3FBF2F303F037
:10D7280001021202C3F34F0392B200E000229C1ED2
:10D73800A4B2FE2C28BF0022CC8828BF02231343A2
:10D7480023439BB203840B884A882B4343F400632A
:10D7580013438A8813438A8913439BB28383F0BD9A
:10D768000038024000127A0000230380438083803F
:10D77800C380038143818381C38107230382704768
:10D7880000230222038043808380C38082608381D8
:10D798007047038819B19BB243F0400303E023F0BC
:10D7A80040031B041B0C03807047838B19B19BB289
:10D7B80043F4806303E023F480631B041B0C83831E
:10D7C8007047038823F400631B041B0C0380038841
:10D7D8009BB20B4303807047B1F5804F038803D198
:10D7E8009BB243F4804303E023F480431B041B0CE7
:10D7F800038070474FF6FF639942038803D09BB2BA
:10D8080043F4807303E023F480731B041B0C038030
:10D818007047838819B19BB243F0040303E023F0F7
:10D8280004031B041B0C83807047838819B19BB2C7
:10D8380043F0100303E023F010031B041B0C838048
:10D848007047838B23F47B6323F00F031B041B0CAB
:10D858008383022303840B88828BB3F5007F10B582
:10D8680092B205D0002B0CBF4FF48073002301E067
:10D878004FF480734C8822438C88898942F4006273
:10D8880022430A4392B21343838310BD808980B236
:10D89800704781817047038819B19BB243F40053E4
:10D8A80003E023F400531B041B0C03807047038818
:10D8B8009BB243F4805303807047012902D0008B48
:10D8C80080B27047808A80B27047008A80B2704701
:10D8D80083889BB20AB1194301E023EA01018180E0
:10D8E8007047090901238B409BB21AB1828892B212
:10D8F800134303E0828892B222EA030383807047CD
:10D90800038919420CBF002001207047C94389B21E
:10D918000181704710B584880089012301F00F0246
:10D9280080B213FA02F21040A4B205D009098B4064
:10D938001C420CBF0020012010BD01F00F01012383
:10D948008B40DB439BB20381704700BF08B50121C0
:10D958004FF48040FFF7BAFD4FF480400021BDE846
:10D968000840FFF7B3BD014B18607047003801400D
:10D9780001F0030289080A4B023130B5920053F8CE
:10D9880021500F24944025EA040443F8214053F819
:10D99800214010FA02F2144343F8214030BD00BF81
:10D9A80000380140014B1860704700BFDC00274277
:10D9B800014B1860704700BF00042742024B186AE9
:10D9C800C0F30020704700BF0038014030B5048C18
:10D9D80024F001042404240C0484058B048CADB2C7
:10D9E800A4B225F0F305154324F00A0445EA03150B
:10D9F80044F00104ADB20C430583048430BD30B556
:10DA0800048C24F010042404240C0484048B058C56
:10DA180024F44074ADB22405240D25F0A00544EA91
:10DA2800022445F0100544EA033445EA0115A4B27E
:10DA3800ADB20483058430BD08B5474B984205D183
:10DA480001200146FFF742FD01203DE0B0F1804F83
:10DA580005D101200146FFF72DFD012076E03F4B5F
:10DA6800984205D102200121FFF724FD02206DE034
:10DA78003B4B984205D104200121FFF71BFD0420F0
:10DA880064E0384B984205D108200121FFF712FDC8
:10DA980008205BE0344B984205D110200121FFF7A4
:10DAA80009FD102052E0314B984205D12020012178
:10DAB800FFF700FD202049E02D4B984209D10220B4
:10DAC8000121FFF703FD02200021BDE80840FFF710
:10DAD800FDBC284B984207D14FF480300121FFF755
:10DAE800F5FC4FF48030EFE7234B984207D14FF411
:10DAF80000300121FFF7EAFC4FF40030E4E71F4B48
:10DB0800984207D14FF480200121FFF7DFFC4FF442
:10DB18008020D9E71A4B984205D140200121FFF710
:10DB2800C9FC402012E0174B984205D18020012102
:10DB3800FFF7C0FC802009E0134B98420BD14FF44B
:10DB480080700121FFF7B6FC4FF480700021BDE81A
:10DB58000840FFF7AFBC08BD0000014000040040CA
:10DB680000080040000C0040001000400014004075
:10DB780000040140004001400044014000480140C9
:10DB880000180040001C0040002000401C4A038888
:10DB980090429BB212D002F5806290420ED0B0F152
:10DBA800804F0BD0A2F58032904207D002F58062F8
:10DBB800904203D002F58062904203D14A8823F054
:10DBC800700313430F4A904208D002F580629042D6
:10DBD80004D023F440730A899BB2134303804B6833
:10DBE800C3620B880385064B984203D003F5806314
:10DBF800984201D18B7A038601238382704700BF44
:10DC080000000140001000404FF0FF334360002344
:10DC18000380038143808372704701858282704745
:10DC2800038823F070031B041B0C0B43038070470D
:10DC380041627047C1627047406A7047008D80B288
:10DC48007047038819B19BB243F0020303E023F045
:10DC580002031B041B0C03807047038819B19BB295
:10DC680043F0040303E023F004031B041B0C0380AC
:10DC78007047038819B19BB243F0800303E023F097
:10DC880080031B041B0C03807047038823F00803E0
:10DC98001B041B0C038003889BB20B430380704753
:10DCA800038823F440731B041B0C038003889BB276
:10DCB8000B4303807047038819B19BB243F00103FB
:10DCC80003E023F001031B041B0C03807047038C43
:10DCD80023F001031B041B0C038470B5038C848898
:10DCE800028B0D884E8822F073021204120C2A430C
:10DCF8008D8923F002031B0435431B0CADB22B4363
:10DD08000E4DA842A4B203D005F58065A8420ED1F5
:10DD1800CD894E8A23F008032B438D8823F0040312
:10DD28002B430D8A354324F44074ADB22C438480D0
:10DD380002838A684263038470BD00BF000001400B
:10DD4800038C23F010031B041B0C0384038C8288B0
:10DD580030B5048B0D8824F4E6442404240C23F005
:10DD6800200344EA05241B048D891B0C43EA051390
:10DD78004D8843EA0513134DA84292B2A4B29BB250
:10DD880003D005F58065A84215D1CD8923F080031D
:10DD98009BB243EA05134FF6BF751D408B8845EAD1
:10DDA80003130D8A22F4406242EA85024D8A42EA50
:10DDB80085029BB292B282808A680483826303845C
:10DDC80030BD00BF00000140038C23F480731B04A6
:10DDD8001B0C0384038C828830B5848B0D8824F057
:10DDE80073042404240C23F400731B042C438D892E
:10DDF8001B0C43EA05234D8843EA0523124DA8422C
:10DE080092B29BB203D005F58065A84215D1CD89A1
:10DE180023F400639BB243EA05234FF6FF351D4008
:10DE28008B8845EA03230D8A22F4405242EA051200
:10DE38004D8A42EA05129BB292B282808A68848334
:10DE4800C263038430BD00BF00000140038C23F48B
:10DE580080531B041B0C0384038C30B58488828B8D
:10DE68000D8822F4E6421204120C23F4005342EA0D
:10DE780005221B048D891B0C43EA05334D8843EAB0
:10DE880005330B4DA842A4B292B29BB203D005F55C
:10DE98008065A84205D10D8A24F4804444EA85149B
:10DEA800A4B2848082838A680264038430BD00BF80
:10DEB80000000140002303804380838083608381C6
:10DEC800C38103824382704730B5058C0124ADB20B
:10DED8008C4025EA040400F11803048409B10829D8
:10DEE80007D149084FF68F70CC582040C850C85801
:10DEF8000AE00439C1F34E0148F6FF70CC582040BF
:10DF0800C8501202C85892B20243CA5030BD416389
:10DF1800704781637047C163704701647047038B22
:10DF280023F070031B041B0C0B4303837047038B04
:10DF380023F4E0431B041B0C43EA01239BB2038335
:10DF48007047838B23F070031B041B0C0B438383E4
:10DF58007047838B23F4E0431B041B0C43EA012323
:10DF68009BB283837047038B23F008031B041B0CAD
:10DF78000B4303837047038B23F400631B041B0CC0
:10DF880043EA01239BB203837047838B23F0080382
:10DF98001B041B0C0B4383837047838B23F40063A0
:10DFA8001B041B0C43EA01239BB283837047038B3A
:10DFB80023F004031B041B0C0B4303837047038BE0
:10DFC80023F480631B041B0C43EA01239BB20383E5
:10DFD8007047838B23F004031B041B0C0B438383C0
:10DFE8007047838B23F480631B041B0C43EA0123D3
:10DFF8009BB283837047038B23F080031B041B0CA5
:10E008000B4303837047038B09025B0441EA5343C4
:10E018009BB203837047838B23F080031B041B0C84
:10E028000B4383837047838B09025B0441EA5343A4
:10E038009BB283837047038C23F002031B041B0CE1
:10E048000B4303847047038C23F008031B041B0C49
:10E058000B4303847047038C23F020031B041B0C21
:10E0680043EA01139BB203847047038C23F08003B7
:10E078001B041B0C43EA01139BB203847047038CF7
:10E0880023F400731B041B0C43EA01239BB2038493
:10E098007047038C23F400631B041B0C43EA012321
:10E0A8009BB203847047038C23F400531B041B0C9E
:10E0B80043EA01339BB20384704710B5048C0123F3
:10E0C8008B40A4B224EA03030384038C12FA01F1FF
:10E0D8000B439BB2038410BD10B5048C04238B4002
:10E0E800A4B224EA03030384038C12FA01F10B435C
:10E0F8009BB2038410BD00230122038043808280E9
:10E10800C38003817047406B7047806B7047C06B5A
:10E118007047006C7047038B23F00C031B041B0C27
:10E128000383038B9BB20B4303837047038B23F456
:10E1380040631B041B0C0383038B9BB243EA01233C
:10E148009BB203837047F8B50C464988A288B4F897
:10E1580000E02389054600290CBF02270027012A71
:10E1680014BF01260226BEF1000F10D1FFF72EFCC6
:10E178002846E188FFF7CFFF2846394632462389EB
:10E18800FFF73DFCE1882846BDE8F840CEE7FFF7F9
:10E1980036FC2846E188FFF7C9FF2846394632464B
:10E1A8002389FFF713FCE1882846BDE8F840B2E769
:10E1B800838B23F00C031B041B0C8383838B9BB280
:10E1C8000B4383837047838B23F440631B041B0C2E
:10E1D8008383838B9BB243EA01239BB2838370477B
:10E1E800F8B50D460B88AA88498804463BB92B899F
:10E1F800FFF7ECFBE9882046BDE8F8408BE7042BE5
:10E2080007D12B89FFF7FBFBE9882046BDE8F840DA
:10E218008CE7082BB5F808C0078C1DD127F4807748
:10E228003F043F0C0784868B038CB6B29BB226F062
:10E23800F30623F4206346EA0C1C43EA01211FFA83
:10E248008CFC89B24CEA020241F480718283018419
:10E25800E988BDE8F840ABE727F480573F043F0C56
:10E268000784868B038C26F4407623F40053360506
:10E278005B04360D5B0C46EA022243EA013342EAAC
:10E288000C329BB2E98892B243F4805382830384B0
:10E29800BDE8F84097E74A880B8813438A881343F8
:10E2A800CA8813430A8913434A8913438A89134343
:10E2B8009BB2A0F8443070470023038043808380DA
:10E2C800C3800381438183817047B0F8443029B10A
:10E2D8006FEA43436FEA53439BB201E05B045B0C74
:10E2E800A0F844307047838819B19BB243F0040307
:10E2F80003E023F004031B041B0C8380704783880E
:10E3080019B19BB243F0010303E023F001031B049E
:10E318001B0C8380704783899BB20AB1194301E0C3
:10E3280023EA01018181704781827047038A19427B
:10E338000CBF002001207047C94389B20182704791
:10E34800038A828911EA030092B203D011420CBFFA
:10E35800002001207047C94389B2018270470A43EF
:10E36800A0F84820704783899BB20AB1194301E09D
:10E3780023EA010181817047838819B19BB243F078
:10E38800080303E023F008031B041B0C8380704779
:10E39800038923F007031B041B0C038170470389BF
:10E3A80023F070031B041B0C0B43038103899BB2EE
:10E3B80043F007030381704738B50D461146012223
:10E3C800602D044602D1FFF71AFB01E0FFF7FEFAC1
:10E3D800238923F070031B041B0C1D43258123890B
:10E3E8009BB243F00703238138BD038923F07003F0
:10E3F8001B041B0C0B4303817047838823F07003B5
:10E408001B041B0C838083889BB20B43838070475B
:10E41800038923F007031B041B0C038103899BB2A8
:10E428000B4303817047038923F080031B041B0CF3
:10E43800038103899BB20B430381704710B504899C
:10E44800E4B20C43144344EA0324A4B2048110BD8B
:10E4580010B50446FFF7F2FF23899BB243F48043CB
:10E46800238110BD10B50446FFF7E8FF238923F088
:10E4780077031B041B0C43F07703238110BD70B591
:10E488000489068B058C26F44076ADB226F0030687
:10E4980024F00704360425F022052404360C15431D
:10E4A800240C46F4807645EA0315214346F001061C
:10E4B800ADB201810683058470BD838819B19BB212
:10E4C80043F0800303E023F080031B041B0C8380CC
:10E4D8007047A0F85010704708B5234B984205D1F3
:10E4E80010200121FEF7F2FF102037E01F4B984261
:10E4F80007D14FF400300121FEF7DCFF4FF4003064
:10E5080009E01B4B98420BD14FF480200121FEF704
:10E51800D1FF4FF480200021BDE80840FEF7CABFB4
:10E52800144B984207D14FF400200121FEF7C2FF97
:10E538004FF40020EFE7104B984207D14FF48010BA
:10E548000121FEF7B7FF4FF48010E4E70B4B984228
:10E5580009D120200121FEF7B9FF20200021BDE8C4
:10E568000840FEF7B3BF08BD00100140004400405A
:10E5780000480040004C004000500040001401409A
:10E58800038ACA889BB223F4405330B513430D461F
:10E59800038283890989AA8823F4B0530A436989C5
:10E5A80023F00C031B040A431B0C92B21343838110
:10E5B800838AAA899BB223F44073134385B083826C
:10E5C80004466846FEF7A6FE1A4B9C4203D003F5A4
:10E5D80080639C4201D1039B00E0029BA28912B296
:10E5E800002A4FF019012A6801FB03F101DA5200F1
:10E5F80000E092006423B1FBF2F1B1FBF3F21201E7
:10E60800100903FB1011A08900B2002806DAC9001E
:10E618003231B1FBF3F303F0070305E009013231AE
:10E62800B1FBF3F303F00F031A4392B2228105B052
:10E6380030BD00BF001001404FF4165303600C2298
:10E6480000238380C38003814281838170470B88C4
:10E65800028A10B54C8823438C88C988234392B218
:10E668000B4322F470629BB21343038210BD002354
:10E67800038043808380C3807047838919B19BB22C
:10E6880043F4005303E023F400531B041B0C838161
:10E698007047038B03F47F430383038B9BB20B43C5
:10E6A80003837047838929B16FEA43436FEA534371
:10E6B8009BB201E05B045B0C83817047838A19B1CC
:10E6C8009BB243F4006303E023F400631B041B0CB8
:10E6D80083827047C905C90D818070478088C0054D
:10E6E800C00D7047038A23F00F031B041B0C038221
:10E6F800038A9BB20B4303827047838919B19BB28B
:10E7080043F0020303E023F002031B041B0C838184
:10E718007047838923F400631B041B0C838183895E
:10E728009BB20B4383817047038A23F020031B04A9
:10E738001B0C0382038A9BB20B4303827047038A34
:10E7480019B19BB243F4804303E023F480431B04D4
:10E758001B0C0382704783899BB243F001038381BA
:10E768007047838A19B19BB243F0080303E023F092
:10E7780008031B041B0C83827047038BDBB20383E3
:10E78800038B9BB243EA012303837047838A19B141
:10E798009BB243F0200303E023F020031B041B0C6F
:10E7A80083827047838A19B19BB243F0100303E058
:10E7B80023F010031B041B0C83827047838A23F009
:10E7C80004031B041B0C8382838A9BB20B43838242
:10E7D8007047838A19B19BB243F0020303E023F028
:10E7E80002031B041B0C83827047838A9BB20AB105
:10E7F800194301E023EA010181827047C1F3421302
:10E8080010B501F01F01012414FA01F1A34201D14E
:10E818000C3004E0022B01D1103000E01430036802
:10E828000AB1194301E023EA0101016010BD038820
:10E8380019420CBF002001207047C94389B20180EA
:10E848007047012210B501F01F03C1F342149A402A
:10E85800012C01D1838903E0022C0CBF038A838A2F
:10E868009BB21340028892B243B1090A012313FAFA
:10E8780001F111420CBF0020012010BD184610BD47
:10E88800090A01238B40DB439BB20380704700BF1A
:10E8980081F0004102E000BF83F0004330B54FEA49
:10E8A80041044FEA430594EA050F08BF90EA020FB6
:10E8B8001FBF54EA000C55EA020C7FEA645C7FEA49
:10E8C800655C00F0E2804FEA5454D4EB5555B8BF6C
:10E8D8006D420CDD2C4480EA020281EA030382EADD
:10E8E800000083EA010180EA020281EA0303362D6F
:10E8F80088BF30BD11F0004F4FEA01314FF4801C42
:10E908004CEA113102D0404261EB410113F0004F53
:10E918004FEA03334CEA133302D0524263EB43030A
:10E9280094EA050F00F0A780A4F10104D5F1200EA8
:10E938000DDB02FA0EFC22FA05F2801841F1000103
:10E9480003FA0EF2801843FA05F359410EE0A5F1D7
:10E9580020050EF1200E012A03FA0EFC28BF4CF008
:10E96800020C43FA05F3C01851EBE37101F00045BE
:10E9780007D54FF0000EDCF1000C7EEB00006EEBCB
:10E988000101B1F5801F1BD3B1F5001F0CD3490855
:10E998005FEA30004FEA3C0C04F101044FEA4452AC
:10E9A80012F5800F80F09A80BCF1004F08BF5FEA33
:10E9B800500C50F1000041EB045141EA050130BD13
:10E9C8005FEA4C0C404141EB010111F4801FA4F1B6
:10E9D8000104E9D191F0000F04BF01460020B1FA0B
:10E9E80081F308BF2033A3F10B03B3F120020CDA43
:10E9F8000C3208DD02F1140CC2F10C0201FA0CF021
:10EA080021FA02F10CE002F11402D8BFC2F1200C85
:10EA180001FA02F120FA0CFCDCBF41EA0C0190403B
:10EA2800E41AA2BF01EB0451294330BD6FEA040484
:10EA38001F3C1CDA0C340EDC04F11404C4F120026F
:10EA480020FA04F001FA02F340EA030021FA04F381
:10EA580045EA030130BDC4F10C04C4F1200220FAD8
:10EA680002F001FA04F340EA0300294630BD21FA16
:10EA780004F0294630BD94F0000F83F4801306BFDC
:10EA880081F480110134013D4EE77FEA645C18BFD0
:10EA98007FEA655C29D094EA050F08BF90EA020F67
:10EAA80005D054EA000C04BF1946104630BD91EA5F
:10EAB800030F1EBF0021002030BD5FEA545C05D162
:10EAC8004000494128BF41F0004130BD14F58004A1
:10EAD8003CBF01F5801130BD01F0004545F0FE4115
:10EAE80041F470014FF0000030BD7FEA645C1ABF4A
:10EAF800194610467FEA655C1CBF0B46024650EA81
:10EB0800013406BF52EA033591EA030F41F40021AC
:10EB180030BD00BF90F0000F04BF0021704730B532
:10EB28004FF4806404F132044FF000054FF0000107
:10EB380050E700BF90F0000F04BF0021704730B5C8
:10EB48004FF4806404F1320410F0004548BF40429D
:10EB58004FF000013EE700BF42004FEAE2014FEAF2
:10EB680031014FEA02701FBF12F07F4393F07F4FCD
:10EB780081F06051704792F0000F14BF93F07F4FFF
:10EB8800704730B54FF4607401F0004521F0004142
:10EB980020E700BF50EA010208BF704730B54FF0C8
:10EBA80000050AE050EA010208BF704730B511F0CD
:10EBB800004502D5404261EB41014FF4806404F105
:10EBC80032045FEA915C3FF4DCAE4FF003025FEA87
:10EBD800DC0C18BF03325FEADC0C18BF033202EB0F
:10EBE800DC02C2F1200300FA03FC20FA02F001FA69
:10EBF80003FE40EA0E0021FA02F11444C1E600BF08
:10EC080070B54FF0FF0C4CF4E06C1CEA11541DBFBA
:10EC18001CEA135594EA0C0F95EA0C0F00F0DEF885
:10EC28002C4481EA030621EA4C5123EA4C5350EA6A
:10EC3800013518BF52EA033541F4801143F48013BB
:10EC480038D0A0FB02CE4FF00005E1FB02E506F04C
:10EC58000042E0FB03E54FF00006E1FB03569CF0A1
:10EC6800000F18BF4EF0010EA4F1FF04B6F5007FA7
:10EC780064F5407404D25FEA4E0E6D4146EB060619
:10EC880042EAC62141EA55514FEAC52040EA5E50A2
:10EC98004FEACE2EB4F1FD0C88BFBCF5E06F1ED84C
:10ECA800BEF1004F08BF5FEA500E50F1000041EB83
:10ECB800045170BD06F0004646EA010140EA020030
:10ECC80081EA0301B4EB5C04C2BFD4EB0C0541EA52
:10ECD800045170BD41F480114FF0000E013C00F367
:10ECE800AB8014F1360FDEBF002001F0004170BD8B
:10ECF800C4F10004203C35DA0C341BDC04F11404A4
:10ED0800C4F1200500FA05F320FA04F001FA05F22F
:10ED180040EA020001F0004221F0004110EBD370FC
:10ED280021FA04F642EB06015EEA430E08BF20EA28
:10ED3800D37070BDC4F10C04C4F1200500FA04F3CB
:10ED480020FA05F001FA04F240EA020001F000415D
:10ED580010EBD37041F100015EEA430E08BF20EAD0
:10ED6800D37070BDC4F1200500FA05F24EEA020E18
:10ED780020FA04F301FA05F243EA020321FA04F047
:10ED880001F0004121FA04F220EA020000EBD370FE
:10ED98005EEA430E08BF20EAD37070BD94F0000FFE
:10EDA8000FD101F00046400041EB010111F4801F32
:10EDB80008BF013CF7D041EA060195F0000F18BFE3
:10EDC800704703F00046520043EB030313F4801F1F
:10EDD80008BF013DF7D043EA0603704794EA0C0FD9
:10EDE8000CEA135518BF95EA0C0F0CD050EA4106EF
:10EDF80018BF52EA4306D1D181EA030101F000416C
:10EE08004FF0000070BD50EA410606BF1046194693
:10EE180052EA430619D094EA0C0F02D150EA01369F
:10EE280013D195EA0C0F05D152EA03361CBF1046E0
:10EE380019460AD181EA030101F0004141F0FE417F
:10EE480041F470014FF0000070BD41F0FE4141F403
:10EE5800780170BD70B54FF0FF0C4CF4E06C1CEA03
:10EE680011541DBF1CEA135594EA0C0F95EA0C0FB8
:10EE780000F0A7F8A4EB050481EA030E52EA033573
:10EE88004FEA013100F088804FEA03334FF0805594
:10EE980045EA131343EA12634FEA022245EA1115C1
:10EEA80045EA10654FEA00260EF000419D4208BF72
:10EEB800964244F1FD0404F5407402D25B084FEA1F
:10EEC8003202B61A65EB03055B084FEA32024FF4CB
:10EED80080104FF4002CB6EB020E75EB030E22BF28
:10EEE800B61A754640EA0C005B084FEA3202B6EBE8
:10EEF800020E75EB030E22BFB61A754640EA5C0097
:10EF08005B084FEA3202B6EB020E75EB030E22BF26
:10EF1800B61A754640EA9C005B084FEA3202B6EB27
:10EF2800020E75EB030E22BFB61A754640EADC00E6
:10EF380055EA060E18D04FEA051545EA16754FEA48
:10EF480006164FEAC30343EA52734FEAC2025FEA66
:10EF58001C1CC0D111F4801F0BD141EA00014FF0F5
:10EF680000004FF0004CB6E711F4801F04BF0143C6
:10EF78000020B4F1FD0C88BFBCF5E06F3FF6AFAEE2
:10EF8800B5EB030C04BFB6EB020C5FEA500C50F172
:10EF9800000041EB045170BD0EF0004E4EEA1131F5
:10EFA80014EB5C04C2BFD4EB0C0541EA045170BDFC
:10EFB80041F480114FF0000E013C90E645EA060E40
:10EFC8008DE60CEA135594EA0C0F08BF95EA0C0F6E
:10EFD8003FF43BAF94EA0C0F0AD150EA01347FF4B6
:10EFE80034AF95EA0C0F7FF425AF104619462CE78D
:10EFF80095EA0C0F06D152EA03353FF4FDAE1046F0
:10F00800194622E750EA410618BF52EA43067FF440
:10F01800C5AE50EA41047FF40DAF52EA43057FF4D0
:10F02800EBAE12E74FF0FF3C06E000BF4FF0010CDB
:10F0380002E000BF4FF0010C4DF804CD4FEA410C3F
:10F048007FEA6C5C4FEA430C18BF7FEA6C5C1BD00C
:10F0580001B050EA410C0CBF52EA430C91EA030F8D
:10F0680002BF90EA020F0020704710F1000F91EAEA
:10F07800030F58BF994208BF90422CBFD8176FEAB8
:10F08800E37040F0010070474FEA410C7FEA6C5C86
:10F0980002D150EA013C07D14FEA430C7FEA6C5C8D
:10F0A800D6D152EA033CD3D05DF8040B704700BFB9
:10F0B8008446104662468C461946634600E000BF07
:10F0C80001B5FFF7B7FF002848BF10F1000F01BDD9
:10F0D8004DF808EDFFF7F4FF0CBF012000205DF8A4
:10F0E80008FB00BF4DF808EDFFF7EAFF34BF012029
:10F0F80000205DF808FB00BF4DF808EDFFF7E0FFC2
:10F1080094BF012000205DF808FB00BF4DF808ED12
:10F11800FFF7CEFF94BF012000205DF808FB00BF79
:10F128004DF808EDFFF7C4FF34BF012000205DF85B
:10F1380008FB00BF4FEA410212F5001215D211D5A3
:10F148006FF47873B3EB625212D94FEAC12343F0DC
:10F15800004343EA505311F0004F23FA02F018BF5E
:10F16800404270474FF00000704750EA013005D127
:10F1780011F0004008BF6FF0004070474FF00000EA
:10F18800704700BF4A0011D212F5001211D20DD5F6
:10F198006FF47873B3EB62520ED44FEAC12343F095
:10F1A800004343EA505323FA02F070474FF000003F
:10F1B800704750EA013002D14FF0FF3070474FF0EE
:10F1C800000070474FEA4102B2F1E04324BFB3F5B3
:10F1D800001CDCF1FE5C0DD901F0004C4FEAC002C6
:10F1E8004CEA5070B2F1004F40EB830008BF20F0AA
:10F1F8000100704711F0804F21D113F13872BCBF64
:10F2080001F00040704741F480114FEA5252C2F1B8
:10F218001802C2F1200C10FA0CF320FA02F018BF01
:10F2280040F001004FEAC1234FEAD32303FA0CFC54
:10F2380040EA0C0023FA02F34FEA4303CCE77FEAE3
:10F24800625307D150EA01331EBF4FF0FE4040F42D
:10F258004000704701F0004040F0FE4040F40000DC
:10F26800704700BF4BB942B9002908BF002802D037
:10F278004FF0FF31084600F037B882B0EC462DE970
:10F28800005000F01BF8DDF804E002B00CBC704739
:10F29800F8B5144606460F461D4600F027F804FB4D
:10F2A80001F300FB0535A4FB0023EB18069CB21AFA
:10F2B80067EB0303C4E90023F8BD00BFF8B51446A3
:10F2C80006460F461D4600F075F900FB05F5A0FB44
:10F2D800042304FB0155EB18069CB21A67EB0303E1
:10F2E800C4E90023F8BD00BF704700BF00292DE91D
:10F2F800F0071D46C0F29E800024002DC0F29580C4
:10F3080007460D4616469C46002B3ED18A4254D9E4
:10F31800B2FA82F343B1C3F1200620FA06F501FAE6
:10F3280003F19A4029439840160CB1FBF6F597B2C1
:10F3380006FB15114FEA104C07FB05F34CEA014197
:10F348008B4209D9891805F1FF3C80F015818B4261
:10F3580040F21281023D8918C3EB010CBCFBF6F3A5
:10F3680006FB13C180B207FB03F740EA014087425E
:10F3780007D9591E821880F00581974240F2028110
:10F38800023B43EA0542002303E08B420AD90023EB
:10F398001A461046194614B1404261EB4101BDE8D6
:10F3A800F0077047B3FA83F3002B40F087808C4551
:10F3B80001D38242ECD80122EBE712B90123B3FB57
:10F3C800F2F2B2FA82F6002E3AD1891A150C1FFA17
:10F3D80082FC0123B1FBF5F705FB17114FEA104832
:10F3E8000CFB07F648EA01418E4207D9891807F154
:10F3F800FF3802D28E4200F2DA804746891BB1FB01
:10F40800F5F605FB161180B20CFB06FC40EA01403C
:10F41800844507D9711E821880F0B080944540F267
:10F42800AD80023E46EA0742B3E7E443524263EB4B
:10F43800430365E7404261EB41014FF0FF345CE76D
:10F44800B240C6F1200521FA05F320FA05F701FAC2
:10F4580006F9150CB3FBF5F847EA09091FFA82FC0F
:10F4680005FB18374FEA19410CFB08F341EA074737
:10F47800B040BB420AD9BF1808F1FF3180F095802F
:10F48800BB4240F29280A8F10208BF18FE1AB6FBF0
:10F49800F5F305FB13611FFA89F90CFB03F649EA3A
:10F4A80001418E4206D95F1E891878D28E4276D9DC
:10F4B800023B8918891B43EA08438BE7C3F12007FD
:10F4C80026FA07F80CFA03F248EA020C21FA07F1C7
:10F4D80005FA03FA4FEA1C4920FA07F5B1FBF9F8D7
:10F4E80045EA0A0509FB18172A0C1FFA8CFA0AFBC9
:10F4F80008F142EA0747B94206FA03F609D917EBB9
:10F508000C0708F1FF324ED2B9424CD9A8F10208D3
:10F5180067447F1AB7FBF9F209FB1271ADB20AFB17
:10F5280002FA45EA01418A4507D9551E11EB0C013B
:10F5380037D28A4535D9023A614442EA08424FEA4D
:10F54800124C1FFA86F808FB0CF7360C95B208FB2C
:10F5580005F806FB057505EB184506FB0CFCAF42E4
:10F5680088BF0CF5803CCAEB01010CEB1546B14293
:10F5780012D309D000230CE76546EDE60E4646EAAD
:10F58800074206E70B46FCE61FFA88F800FA03F381
:10F5980008EB0545AB42EDD2013A0023F9E63B46BC
:10F5A80088E72A46C9E79046B3E788466EE7023FF0
:10F5B800891823E72DE9F00F144605460E46002B5F
:10F5C8003FD18A424AD9B2FA82F343B1C3F120004B
:10F5D80025FA00F201FA03F69C4016439D40210CDF
:10F5E800B6FBF1F22F0CA0B201FB126C00FB02F388
:10F5F80047EA0C46B34208D9571E361980F0FF80F7
:10F60800B34240F2FC80023A3619F61AB6FBF1F31F
:10F6180001FB1361ADB200FB03F045EA01418842EA
:10F6280007D95E1E091980F0EC80884240F2E98013
:10F63800023B43EA0242002310461946BDE8F00F98
:10F6480070478B4243D8B3FA83F4002C42D18B42E3
:10F65800234601D382423BD80122EDE712B90123A8
:10F66800B3FBF2F4B4FA84F2002A40F08A80091B52
:10F67800260CA7B20123B1FBF6F006FB10114FEAE6
:10F68800154C07FB00F24CEA01418A4207D90919D7
:10F6980000F1FF3C02D28A4200F2D3806046C2EBFE
:10F6A800010CBCFBF6F206FB12C1ADB207FB02F778
:10F6B80045EA0145AF4207D9511E2C1980F0A380B5
:10F6C800A74240F2A080023A42EA0042B4E700238F
:10F6D8001A46B1E7C4F1200722FA07F603FA04F341
:10F6E800334321FA07FA4FEA134C01FA04FB20FAD4
:10F6F80007F141EA0B0BBAFBFCF70CFB17A61FFA44
:10F7080083F84FEA1B4508FB07F945EA0645A94572
:10F7180002FA04FA04D97A1EED18C0F08880174658
:10F72800C9EB0505B5FBFCF60CFB16521FFA8BFB63
:10F7380008FB06F84BEA0241884503D9721EC9182E
:10F7480070D3164646EA0742170C1FFA8AFC0CFBD0
:10F7580007F695B24FEA1A430CFB05FC03FB056557
:10F7680005EB1C4503FB07F3AE4288BF03F5803366
:10F77800C8EB010103EB1543994250D347D000234E
:10F788005AE79440C2F12008260C20FA08F721FA1B
:10F7980008F501FA02F9B5FBF6F847EA090906FB8C
:10F7A8001855A7B24FEA194C4CEA054C07FB08F369
:10F7B800634500FA02F509D91CEB040C08F1FF3285
:10F7C8003DD263453BD9A8F10208A444C3EB0C021F
:10F7D800B2FBF6F306FB13201FFA89F907FB03F2C5
:10F7E80049EA00418A4206D9581E091925D28A4297
:10F7F80023D9023B0919891A43EA08433BE73A46E9
:10F8080003E7334615E70A4642EA004214E71FFABF
:10F818008CF100FA04F001EB0545A842AFD2013A99
:10F82800002309E788458CD9023EC9188AE7A9450B
:10F838007FF675AF023FED1872E70346DBE79046A7
:10F84800C4E7023809192AE7002103E00A4B5B588C
:10F858004350043109480A4B42189A42F6D3094AE0
:10F8680002E0002342F8043B074B9A42F9D3F9F728
:10F878007DF900F00DF870470CAA0508000000207B
:10F888000C0B0020100B0020F4900020FEE7000075
:10F89800844B854A2DE9F3414FF4FA661E60834B89
:10F8A800DFF874821A60824A824B1A60824B42F2F5
:10F8B80010721A60814B64241C60814B4FF0FF3238
:10F8C8001A60804B00251D70012788F80070F7F733
:10F8D8003DFDF6F76FFD2046F7F7D2F9F6F790FDF4
:10F8E8002046F7F7CDF9F7F717FDF7F765FBF7F7B8
:10F8F800DDF92046F7F7C4F9F9F720FA2046F7F7BB
:10F90800BFF94FF4FA50F7F727F92046F7F7B8F997
:10F91800F6F7A8FC2046F7F7B3F92846F7F7F0F909
:10F928006948F7F7ADF9F4F703F82046F7F7A8F9AF
:10F93800664B03F1100229468DE8240028465A68D0
:10F948001B68F4F7FBF93046F7F79AF92846F4F7FD
:10F9580075FC4FF6FF70F4F787FC322003215C4AF0
:10F968002B46F4F799FD96208C215A4A2B46F4F73A
:10F9780093FD9620584AA0212B46F4F78DFDB4211B
:10F98800564A2B469620F4F787FD3046F7F778F964
:10F99800DC21534A2B462846F4F77EFD5148F7F7F9
:10F9A8006FF92046F7F76CF9F6F724FA2046F7F7CF
:10F9B80067F99FED4D0AF7F7BBF92046F7F760F9AD
:10F9C8004A4B4B4A009339464A4B4B48FBF782FC5B
:10F9D8002046F7F755F9F5F729F82046F7F750F9D3
:10F9E8001420F5F777FF2846F5F7C7FF2046F7F705
:10F9F80047F9F6F749F92046F7F742F9F6F7D2FC46
:10FA08002046F7F73DF9F6F745FA08B188F80050AF
:10FA1800F6F74CFA08B1F9F76FF8384B00241C7068
:10FA2800F1F722FCF4F7B8FF08B9354802E0354B86
:10FA380035481C70F1F72FFC344E354DF5F720FC96
:10FA4800F8F71BF8F8F74EF8F7F752FEF7F786FDC8
:10FA58003746F6F741FA337833B1012B02D1F7F77D
:10FA6800D9FA01E0F7F7FEFA00243C70F7F73CFCFE
:10FA7800F3F7E0F9F8F79EFF2A8812B2012AE8D1D5
:10FA880024484FF40051FDF782F9F8F78BF8F7F79F
:10FA9800D5FB20484FF400512246FDF778F92C8019
:10FAA800D7E700BF64400020E067350088400020A9
:10FAB80080C3C901384100208C4000204C40002000
:10FAC800844000208C4D002000127A00B07B010891
:10FAD800AFA20508C9A20508D5A20508E1A2050834
:10FAE800EAA20508002D31010000FA44C4010020F3
:10FAF8009840002024020020983A00206C40002002
:10FB0800BC0D0020943A0020A80F0020904000204F
:10FB1800FC0B002000080240080D002010B4314CF6
:10FB28000180B1F5807F44608270C37052D00DD9D6
:10FB3800B1F5806F39D017D9B1F5006F2ED0B1F576
:10FB4800805F24D0FF2040B210BC704720293AD0F3
:10FB580014D9402930D08029F4D123494FF02012FC
:10FB6800C26081600020EEE7B1F5007FEAD11F4B4B
:10FB78004FF00811C16083600020E4E71029E1D14B
:10FB88001B494FF00122C26081600020DBE7194B5E
:10FB98004FF00111C16083600020D4E7164A4FF08E
:10FBA8000213C36082600020CDE714494FF00412AD
:10FBB800C26081600020C6E7114B4FF04011C16060
:10FBC80083600020BFE70F4A4FF08013C360826054
:10FBD8000020B8E70C4A4FF01013C3608260002081
:10FBE800B1E700BFC8A1040806920508D691050828
:10FBF800C6930508C8910508CA910508CE9105085D
:10FC080046920508C6920508E69105082DE9F00F09
:10FC1800B2B02E9030932E9B00882E9C5B68309F4C
:10FC2800A4682D90451E03EB4506BF082093289431
:10FC38002C952F911F921E96319700F03A814FEA2A
:10FC4800900A4FEACA0B00F003002F99299003F19C
:10FC5800080504EB0B00CDF884A0CDF8A8B01995E1
:10FC68001A921B97189617912B90179A189E13881B
:10FC78003380B2F802C0A6F802C09488B480D7884E
:10FC8800F78008361896219F199E0832179256F861
:10FC9800041C56F8082C4FF0000A4FF0000B002FF8
:10FCA80000F06982CDE904ABCDE906ABCDE902AB42
:10FCB800CDE900AB289CBC46029BDDF80C9025687A
:10FCC800C2FBC5394FF0000848EA030ACB46CDE924
:10FCD80002AB049BDDF814B0C1FBC53BCDF824B0E2
:10FCE800CDF82080DDE908ABC1EA02004AEA030A40
:10FCF800CDE904AB069BDDF81CB03268C0FBD53BF0
:10FD0800CDF82CB0CDF82880DDE90AABC2EA0107AE
:10FD18004AEA030ACDE906AB9DE80108C7FBD50B03
:10FD2800CDF834B0CDF83080DDE90CAB4AEA000AF2
:10FD380063680298CDE900AB0834DDF80CB0C1FB6C
:10FD4800C30BCDF83CB0CDF83880DDE90EAB4AEAFC
:10FD5800000ACDE902AB71680498DDF814B0C2FB63
:10FD6800C30BCDF844B0CDF84080DDE910AB4AEACA
:10FD7800000ACDE904AB0698DDF81CB0C7FBD30B2D
:10FD8800CDF84CB0CDF84880DDE912ABC1EA0205E8
:10FD98004AEA000ACDE906AB9DE80108C5FBD30B8A
:10FDA800CDF854B0CDF85080DDE914AB08364AEAF6
:10FDB800000ABCF1010CCDE900AB7FF47DAF2A9DB0
:10FDC80019982B9B2E18299F002F35D01868039F50
:10FDD800029BC2FBC03700241D971C94DDE91C451B
:10FDE80044EA0304CDE90245049B059DC1FBC035E7
:10FDF800002723952297DDE9224544EA0304CDE94B
:10FE08000445C1EA0203079D069AC3FBD025259540
:10FE18002497DDE9244544EA02043368C3EA010172
:10FE2800CDE9064553465D46C1FBD0352795269753
:10FE3800DDE926AB4AEA030A069A029C0499039D67
:10FE4800079FD30B059AE60BC90B46EA454043EAE0
:10FE5800474441EA424604F30F0500F30F0C199B8F
:10FE6800CCEA054706F30F001A9D1B9E2F604FEA48
:10FE7800DA3A08334AEA4B4B0BF30F04C0EA044260
:10FE88006A600835711E19931A951B917FF4EDAEBF
:10FE9800319A2F9E1E991F9BDDF880B0D00037182D
:10FEA8000D182F970BEB000A1F181E951F97CDF8FA
:10FEB80080A0DDF8C0C01CF0030BCDF820B000F026
:10FEC80086802D9BDDF8BC80CDF808B05808DDF899
:10FED80080A0DDF8A0B00690CDF81080049A1E9E90
:10FEE80032F8025B069826F8025B0492BAF80270B0
:10FEF800BBF80230BAF80020BBF800401E9617FB8A
:10FF080003F112FB04F6451E4FEAE17711EB0608F0
:10FF18002B4605F0010047EBE6790AF104020BF1E4
:10FF28000401002D3BD0A8B1B2F800C0BBF80470A2
:10FF3800548848881CFB07F518EB050749EBE5765C
:10FF480014FB00F917EB090846EBE9790432043190
:10FF5800013B24D00F88B2F800C0568848888C88A6
:10FF680095881CFB07FC18EB0C0816FB00F7D088DB
:10FF7800CE8849EBEC7C15FB04F518EB07084CEB35
:10FF8800E77918EB050710FB06FC49EBE57417EB5E
:10FF98000C0844EBEC7908320831023BDAD11F9A9D
:10FFA80002994FEAD83545EA494404F30F0322F889
:10FFB800023B4F1E0AF1020A1F9202978ED1DDF80A
:10FFC80080A0DDF820B00AEB4B0ACDF880A02C9E6B
:10FFD8002E98B50840683FD0209F47EA000212F0EB
:10FFE800030F00F1080307F1080214BF00210121E3
:08FFF8009F4298BF904294BFA4
:020000040801F1
:1000000000260126314277D097E8420001600121A5
:100010006C1EA942466004EA010419D044B192E87A
:100020001200196002215C6008320833A9420FD027
:1000300092E850001C605E60966802F1080BD2687E
:100040009E600231DA601033A9420BF10802EFD151
:10005000DDF880C0ED000CEB050B4019CDF880B049
:100060002C9C14F0030343D05A085400002A00F0DB
:100070008E80209D40EA050717F0030F209F14BFD4
:1000800000250125011D3E1D012B94BF002505F013
:1000900001058F4298BFB04294BF002101210D425B
:1000A00075D039689200BF18A342016020971044B0
:1000B000C4EB03011CD0209B013933F8024B0A46E4
:1000C00020F8024B01F0010192B129B133F8021B73
:1000D000013A20F8021B0BD01C46014634F802CB33
:1000E00021F802CB5D88A31C4580881C023AF3D11D
:1000F00032B0BDE8F00F7047B7F800C0A0F800C0FC
:100100007C884480BE888680691EFE880C46BA467C
:1001100001F00101C680002C9AD089B1B2F800B07C
:10012000A3F800B051885980B2F804C0A3F804C005
:10013000B2F806B00832A3F806B00833013C87D005
:1001400016881E8051885980B2F804B0A3F804B014
:10015000B2F806C0A3F806C016891E8103F1080B89
:100160005189ABF802109389ABF80430D68910326C
:10017000023C0BF10803ABF80660E1D168E7289B6D
:10018000CDE904ABCDE906ABCDE902AB1FE61946DC
:1001900091E700BF2DE9F00F9CB006780F900F9CFF
:1001A00040880F9DA4686D681990B3FBF6FA471E4E
:1001B0004FEA5A0804EB4709AAEB480340460A9461
:1001C0000D951A97CDF86C800C911492CDF82C9067
:1001D0001193002800F0B5811746199A199CCDF8A3
:1001E00048809108CA00159104F00303A9181792DA
:1001F000169310971891760075084FEA450C002D5C
:1002000000F03B840B9FDDF8308047EA080010F0D7
:10021000030F14BF0021012108F10404381D012E31
:1002200094BF002101F00101804598BFA74294BF0F
:100230004FF000094FF0010911EA090F00F01D8489
:10024000BB46D8F8002001236F1EAB42CBF800203C
:1002500007EA03072146024614D237B12468022375
:100260000431021DAB4204600CD20C46104654F817
:10027000047B40F8047B496802335160211D021D54
:10028000AB42F2D3DDF83080DDF82CB04FEA4C05FC
:10029000664508EB05020BEB0503CCEB06001DD011
:1002A000013832F802CB014623F802CB00F00100FE
:1002B000A1B128B132F8029B013923F8029B0DD07D
:1002C00014461F4634F8029B27F8029BB2F802A09E
:1002D000A21CA3F802A0BB1C0239F1D10C9ADDF8D4
:1002E0003CC00B989CF80080710053180A9E0C9338
:1002F000159BCDF84C80451806EB48020B950E92E5
:10030000002B00F0B18300240025CDE90445CDE9A0
:10031000024507930D9913460A9AB3F804A0B2F860
:1003200006B0CDF804A0B3F806A00E881588CDF865
:1003300020B0CDF824A0DDE902AB15FB06F51AEBE1
:10034000050A4BEBE57BCDE902AB1F884888B2F884
:1003500002C0B3F80290B2F804808C88CDF81880FF
:10036000DDE904AB16FB07F61AEB060A4BEBE67B5E
:10037000DDE902671CFB00F5761910FB09F047EB7D
:10038000E5771AEB000A4BEBE07BCDE902ABDDF839
:1003900018B0DDF804C0B1F80680099D1BFB04F01D
:1003A00016EB000A47EBE07BDDE9026714FB0CF477
:1003B000361947EBE477089C14FB08F00831083243
:1003C00008331AEB000418FB05F84BEBE0750798AF
:1003D00016EB080A47EBE87B0138CDE90245CDE989
:1003E00004AB079099D1179E0E9C0A9B1899A719E8
:1003F0009A190E97169F002F73D00E9B31F8020B9F
:1004000032F8024B33F8026BDDE90289DDE904AB17
:1004100014FB00F47D1E10FB06F618EB040849EBF4
:10042000E4791AEB060A4BEBE67B2F4605F0010058
:10043000CDE90289CDE904AB002D52D0002873D05C
:1004400031F8024B32F8020B33F8025B10FB04F672
:1004500014FB05F0DDE90245DDE90489A41945EB4B
:10046000E67518EB000849EBE079013FCDE902455C
:10047000CDE9048935D0C246CB46DDE902890D4677
:1004800014460497214628461A4630F8026B31F884
:10049000027B32F802CB6D8864885B8817FB06F715
:1004A00018EB070816FB0CF649EBE7791AEB060781
:1004B00014FB05FA4BEBE67B15FB03FC8C1C931C31
:1004C0000499851C18EB0A0849EBEA7917EB0C0A2A
:1004D0004BEBEC7B8A1ECDE902890492D2D1CDE9A7
:1004E00004AB029D03990498DDF828A0059BEA0B54
:1004F000109D42EA4148129908F30F09A5F80090AF
:10050000DDF84C90C70B0AEB8908281D4A1E47EA04
:100510004346CDF8288006F30F0410906C801292A9
:100520000AD00F9C267866E6DDE904AB0D4614463A
:100530000497DDE90289A5E7149F1B9B07EB83065F
:100540001496119F002F00F0A681DDF864B0DDF84D
:100550006480DDF834C04FEA9B09CDF81C904FEA67
:10056000C90908F0030A0CEB090BCDF82090CDF86F
:1005700010A0CDF824B0DDF83CC09CF800607508F0
:100580004FEA450C002D00F07E820C990B980B9FD2
:1005900040EA010414F0030F14BF002201220C1DD5
:1005A0000430012E94BF002202F00102814298BF64
:1005B000A74294BF002301231A4200F06482BA4686
:1005C00001230F68691EAB42CAF80070024601EAB7
:1005D0000307214614D237B127680223211D021DCB
:1005E000AB4207600CD20C46104654F8047B40F82E
:1005F000047B496802335160211D021DAB42F2D3D6
:10060000DDF83090DDF82C804FEA4C05664509EBAB
:10061000050208EB0503CCEB06001DD0013832F8CB
:1006200002BB014623F802BB00F00100A1B128B1D2
:1006300032F8025B013923F8025B0DD014461F46E5
:1006400034F802AB27F802ABB2F802C0A21CA3F840
:1006500002C0BB1C0239F1D1DDF82CA0DDF830B0AE
:10066000079876000AEB060C0BEB0608CDF82CC0B9
:10067000CDF83080002800F0F0810A9ADDF834804F
:100680005788B2F800A0DDF828909488B9F8069051
:10069000B8F8062084460D9841880588B8F804000B
:1006A00017FB01F61AFB05F3B3461BEB03014FEAF8
:1006B000E67714FB00F047EBE3750F180A9B19FB74
:1006C00002F145EBE0750CF1FF3617EB010AB1467C
:1006D00006F0010008F1080203F1080345EBE17B95
:1006E000002E00F0858048B3DDF834C01E88BCF8C9
:1006F00008405888518897889D88B2F80680B3F8DA
:1007000006C016FB04F41AEB040A10FB01F14BEBD4
:10071000E4761AEB010415FB07FB46EBE17014EBE2
:100720000B011CFB08F640EBEB740832083311EBAD
:10073000060A44EBE67BB9F1010959D0CDE902ABD9
:10074000CB46B3F80080B3F808901688CDF83890FF
:1007500018FB06F6DDE902895D885488988891883F
:10076000B2F806C0DF88B2F808A015FB04F418EB55
:10077000060810FB01F149EBE67918EB040817FBBA
:100780000CF749EBE47918EB010849EBE17918EB38
:10079000070849EBE779CDE90289DDF838905D89F2
:1007A000548998899189B2F80EC0DE8919FB0AF73D
:1007B000DDE9028915FB04F418EB070810FB01F1D1
:1007C00049EBE77918EB040849EBE47916FB0CF6E2
:1007D00018EB010449EBE17510321033A01945EB19
:1007E000E671BBF1020BCDE90201AAD182468B462C
:1007F0000DF1200898E816006318049D9DB332F8A7
:1008000002CB33F8026B16FB0CF4013D1AEB040A21
:10081000294605F001004BEBE47B25B358B132F8D3
:10082000028B33F8020B10FB08F71AEB070A4BEBAD
:10083000E77B691E17D01446184634F8025B30F87F
:10084000027B52885B8817FB05F81AEB08064BEB16
:10085000E87713FB02FBA21C831C16EB0B0A47EB89
:10086000EB7B0239E7D10F9DDDF8508095F800C091
:100870000A9A119E4FEADA3343EA4B4404F30F001D
:1008800028F8020B02EB4C07711E0A97CDF8508036
:1008900011917FF470AE1A9E0F9CB508A06842D0EB
:1008A0000A9F47EA000616F0030F07F1080200F15D
:1008B000080314BF002101219F4298BF904294BFBA
:1008C0004FF0000A4FF0010A11EA0A0F7FD097E8B3
:1008D0004200016001216C1EA942466004EA010445
:1008E00019D044B192E81200196002215C6008320C
:1008F0000833A9420FD092E850001C605E609668F1
:1009000002F10804D2689E600231DA601033A94215
:1009100004F10802EFD1DDF828A0ED000AEB05098B
:100920004019CDF82890DDF868A01AF003034AD0EA
:100930005A085400002A00F0A480DDF828B040EAEC
:100940000B0515F0030F14BF002501250BF104065C
:10095000011D012B94BF002505F001058B4598BFB3
:10096000B04294BF4FF0000C4FF0010C15EA0C0F91
:1009700000F08780DBF8001092009344A3420160EE
:10098000CDF828B01044C4EB03011CD00A9B0139F8
:1009900033F8024B0A4620F8024B01F0010192B1F4
:1009A00029B133F8021B013A20F8021B0BD01C4678
:1009B000014634F802CB21F802CB5D88A31C4580A8
:1009C000881C023AF3D11CB0BDE8F00F7047B7F8AD
:1009D0000090A0F800907C884480BE888680691EC4
:1009E000FE880C46B84601F00101C680002C92D06A
:1009F00091B111881980B2F802C0A3F802C0B2F810
:100A000004A0A3F804A0B2F806900832A3F8069058
:100A10000833013C3FF47FAF11881980B2F802C05F
:100A2000A3F802C0B2F80490A3F80490B2F806A0AC
:100A3000A3F806A016891E8103F1080C5189ACF8B1
:100A400002109389ACF80430D6891032023C0CF1C4
:100A50000803ACF80660DFD15DE70D9A0A9B4FF002
:100A6000000A4FF0000BC8E600260027CDE9046716
:100A70000A9A0D99CDE90267BCE430460B9B0C9AAB
:100A80000EE4194682E730460B9B0C9AC6E500BF80
:100A900000B553EC102B42F2FB1223F00043C3F6D7
:100AA000E972934285B026DD4FF6FF72C7F6EF720A
:100AB00093420BDD51EC100B02460B46FDF7F0FEA6
:100AC00002460B4643EC102B05B000BD684600F013
:100AD000BFFB00F0030001289DED000B9DED021B04
:100AE0001AD0022810D0F8B900F0D2FE53EC102B27
:100AF00010461946E4E79FED101B00F0C9FE53ECC9
:100B0000102B10461946DBE700F0C2FE53EC102B09
:100B1000104603F10041D3E701F0F6FB53EC102B34
:100B2000104603F10041CBE7012001F0EDFB53EC4F
:100B3000102B10461946C3E700000000000000001B
:100B40002DE9F04759EC108BC9F30A56A6F57E74CF
:100B5000073C132C4D46CA46474626DC002C4FDB8B
:100B60004FF6FF76C0F20F0646FA04F606EA0905CC
:100B700055EA080517D044A3D3E9002351EC100B24
:100B8000FDF790FE00220023FEF7CEFA00284AD09F
:100B9000B9F1000F6EDB2AEA060A4FF0000853464F
:100BA000424643EC102BBDE8F087332C0CDDB4F546
:100BB000806FF8D151EC100B3A460B46FDF772FEF0
:100BC00041EC100BBDE8F087A6F58265033D4FF0C0
:100BD000FF3323FA05F515EA080FE4D02AA3D3E979
:100BE000002351EC100BFDF75DFE00220023FEF701
:100BF0009BFAC0B1B9F1000F1CDB28EA050813E02D
:100C000021A3D3E9002351EC100BFDF74BFE00228A
:100C10000023FEF789FA38B1B9F1000F1BDB4FF062
:100C20000008C24600E0CA465346424643EC102B39
:100C3000BDE8F087142C09D0C6F5866303334FF066
:100C4000010808FA03F818EB0708D6D30AF1010ADD
:100C500028EA0508E8E729F0004848EA07084FF0C5
:100C6000000AD045CBF6F07A08BFCA4618BF4FF04D
:100C70000008D9E74FF4801343FA04F409EB040A9F
:100C800089E700BFAFF300809C7500883CE4377EA5
:100C900000B553EC102B42F2FB1223F00043C3F6D5
:100CA000E972934285B027DD4FF6FF72C7F6EF7207
:100CB00093420BDD51EC100B02460B46FDF7F0FDA5
:100CC00002460B4643EC102B05B000BD684600F011
:100CD000BFFA00F0030001289DED000B9DED021B03
:100CE0001DD0022812D008BB012001F00DFB53ECEF
:100CF000102B10461946E3E700209FED111B01F071
:100D000003FB53EC102B10461946D9E7012001F0E4
:100D1000FBFA53EC102B104603F10041D0E700F032
:100D2000B7FD53EC102B10461946C9E700F0B0FD93
:100D300053EC102B104603F10041C1E7AFF30080E4
:100D4000000000000000000000F0E6B8D0B52DED76
:100D5000048BB0EE408AF0EE608A3C4C8AB000F022
:100D6000DBF994F90030B0EE409AF0EE609A01336E
:100D700035D0B0EE480AF0EE680A01F04FFD0028C9
:100D80002DD051EC180B00220023FEF7B9F930B337
:100D90002F4B24780193002308938DED028B8DED6A
:100DA000048B002C23D000270026CFF6F07751ECDF
:100DB000180B00220023CDE90667FEF78DF9002805
:100DC00025D002239C42009336D0684601F05EFD98
:100DD000002831D0089B002B27D19DED069BB0EE5B
:100DE000490AF0EE690A0AB0BDEC048BD0BD4FF69B
:100DF000FF774FF06046CCF2EF7751EC180B0022F2
:100E00000023CDE90667FEF767F90028D9D1012351
:100E1000022C009315D0684601F038FD88B10D48CA
:100E200001F036FD8DED060BD4E701F0EFFF089BD6
:100E30009DED069B0360D2E701F0E8FF22230360EB
:100E4000C8E701F0E3FF21230360E8E74C0200203C
:100E500010A5050870A7050810B52DED048BB0EEA0
:100E6000408AF0EE608A294C8AB000F02DFC94F99B
:100E70000030B0EE409AF0EE609A01332BD0B0EE25
:100E8000480AF0EE680A01F0C9FC20B351EC180BD7
:100E900000220023FEF72AF9E8B11D4B24780193C4
:100EA00001230093002308938DED048B8DED028BBD
:100EB000CCB10020002102460B46FDF7CFFF022CEB
:100EC000CDE9060115D101F0A1FF21230360089BA4
:100ED000ABB99DED069BB0EE490AF0EE690A0AB087
:100EE000BDEC048B10BD0022002343EC172B8DEDCD
:100EF000067B684601F0CAFC0028E8D1E3E701F070
:100F000085FF089B9DED069B0360E4E74C020020F3
:100F100018A5050800000000F8B5B0EE407AF0EE24
:100F2000607A53EC112B544210461D46002125F0E7
:100F30000047044353EC102B47EAD474C7F6F07112
:100F40008C4216463DD85442344323F0004242EAD4
:100F5000D4748C4235D805F1404101F5801101432C
:100F60004FD0AC1704F00204164344EAD37435D0D2
:100F7000384341D00021C7F6F0718F424FD0002195
:100F8000C7F6F0718A4237D0D21B12153C2A42DCD8
:100F9000002D7DDB53EC112B51EC170BFDF75EFFA1
:100FA00041EC100B01F030FC01F06AFA51EC100B2F
:100FB000012C68D0022C57D0002C48D141EC170BE3
:100FC00007E051EC170B53EC112BFDF76BFC41ECD8
:100FD000170BB0EE470AF0EE670AF8BD032CC7D82E
:100FE00001A151F824F000BFD30F0108D30F01086D
:100FF000111001080B100108002B25DB9FED307B41
:10100000E7E7BDE8F84001F03BBA9FED2F7BE0E752
:101010009FED2F7BDDE72AA1D1E90001C8E7BA42A5
:101020003CD0032CABD801A151F824F043100108A7
:101030003D100108111001080B1001089FED267BDF
:10104000C7E79FED277BC4E79FED277BC1E730A370
:10105000D3E90023FDF724FC1DA3D3E90023FDF70A
:101060001FFC41EC170BB4E729A3D3E90023FDF7DC
:1010700017FC02460B4616A1D1E90001FDF710FC52
:1010800041EC170BA5E701F1004141EC170BA0E77C
:101090003C32BFF67FAF0020002189E7032CABD89C
:1010A000DFE804F00B0805029FED117B91E79FED4F
:1010B000127B8EE79FED127B8BE79FED137B88E71A
:1010C000182D4454FB21F93F182D4454FB2109C02D
:1010D000182D4454FB21094000000000000000804E
:1010E0000000000000000000182D4454FB21F9BF4F
:1010F000D221337F7CD902C0D221337F7CD90240F8
:10110000182D4454FB21E9BF182D4454FB21E93F1D
:10111000075C143326A6A13C2DE9F84F55EC104B83
:10112000B5F5801F2F4622DA25F00043234368D00F
:10113000002D2046294670DB00230022C4F25033E4
:10114000FDF762FD4FF6FF730F46C7F6EF739F4240
:1011500004460D466FF0350210DD20462946224632
:101160002B46FDF79FFB41EC100BBDE8F88F4FF6C7
:10117000FF73C7F6EF7300229F42EEDC3B15A3F529
:101180007E73073B9A18D60F901927F07F47C6F554
:101190007E76FDF7D3FC073627F4700747EA06553D
:1011A00045EC104B8046894601F00AFC4046494612
:1011B00021A3D3E9002355EC104BFDF725FD20A317
:1011C000D3E9002382468B4640464946FDF71CFD85
:1011D0001DA3D3E9002306460F4620462946FDF706
:1011E00013FD02460B4630463946FDF75BFB0246CF
:1011F0000B4650465946FDF755FB41EC100BBDE838
:10120000F88F00210020CCF2503100220023FDF79E
:1012100025FE41EC100BBDE8F88F22462B46FDF76A
:101220003FFB00220023FDF719FE41EC100BBDE847
:10123000F88F00BFAFF3008000609F501344D33F8E
:10124000362BF111F3FE593D0EE526157BCBDB3F26
:101250002DE9F04F53EC102B42F2FB1223F0004427
:10126000C3F6E97294428FB01E46074640F3AA8047
:101270004DF67B13C4F202039C422ADC002E51EC93
:10128000100BDDA3D3E9002340F3CA81FDF708FB6F
:1012900042F2FB13C3F6F9739C428046894600F084
:1012A000AA80D7A3D3E90023FDF7FAFA0D46044636
:1012B0002B462246C7E9004540464946FDF7F0FA6D
:1012C000CFA3D3E90023FDF7EBFA0125C7E902011B
:1012D00081E042F2FB13C4F239139C4240F3AA802E
:1012E0004FF6FF73C7F6EF739C4278DC4FEA245A3F
:1012F000AAF5826AAAF1060A51EC100BA4EB0A5374
:1013000019461D460446FDF719FFFDF717FC8046F8
:10131000894642464B4620462946CDE90889FDF7D5
:10132000BFFA00230022C4F27013FDF76DFC0D46D6
:101330000446FDF703FFFDF701FC80468946204681
:10134000294642464B46CDE90A89FDF7A9FA002312
:101350000022C4F27013FDF757FC002204460D462C
:101360000023CDE90C45FDF7B7FE002800F07B8196
:101370004046494600220023FDF7AEFE03240AAD95
:10138000013C40B175E9020100220023FDF7A4FEF3
:10139000013C0028F6D12346022400949E4C08A864
:1013A00039465246019400F0ABFB002E054612DA96
:1013B0007A68FB6802F1004203F100437A60FB6047
:1013C000454208E00022002343EC172B87ED000B79
:1013D00080ED027B002528460FB0BDE8F08F51EC70
:1013E000100B02460B46FDF75BFA0025C7E9020128
:1013F000C7E90001EFE77AA3D3E90023FDF750FA2C
:1014000079A3D3E9002380468946FDF749FA0D46C2
:1014100004462B462246C7E9004540464946FDF7AB
:101420003FFA71A3D3E90023FDF73AFA0125C7E992
:101430000201D0E701F0E8F959EC108B6CA3D3E975
:10144000002340464946FDF7DFFB00230022C3F698
:10145000E073FDF727FAFDF771FE0546FDF76EFB19
:1014600065A3D3E90023CDE90201FDF7CDFB0246D8
:101470000B4640464946FDF713FA61A3D3E9002322
:1014800082468B46DDE90201FDF7BEFB1F2DCDE94B
:101490000401504659462BDC6A1E604B53F822303B
:1014A000A34225D0DDE90423FDF7FAF902460B46F5
:1014B000C7E90023814688464A4643465046594676
:1014C000FDF7EEF9DDE90423FDF7EAF9002E024607
:1014D0000B46C7E90223BFF67EAF08F1004301F1D6
:1014E0000041C7F800907B60B860F9606D4272E718
:1014F000DDE90423FDF7D4F988462415C8F30A531F
:10150000E31A102B8146C7E90001D5DD34A3D3E9E6
:101510000023DDE90201FDF777FB8046894642465C
:101520004B4650465946FDF7BBF9CDE90601DDE9CA
:10153000062350465946FDF7B3F942464B46FDF7A0
:10154000AFF929A3D3E9002380468946DDE90201EA
:10155000FDF75AFB42464B46FDF7A2F9CDE90401DF
:10156000DDE90423DDE90601FDF79AF98846C8F3B1
:101570000A53E41A312C8146C7E9000140F39580F3
:1015800021A3D3E90023DDE90201FDF73DFB8046FD
:10159000894642464B46DDE90601FDF781F9824660
:1015A0008B4652465B46DDE90601FDF779F9424676
:1015B0004B46FDF775F916A3D3E90023804689460B
:1015C000DDE90201FDF720FB42464B46FDF768F9D5
:1015D000CDE904015046594664E700BFAFF30080EF
:1015E0000000601A61B4D03D7370032E8A19A33BCA
:1015F00083C8C96D305FE43F00004054FB21F93FD0
:101600003163621A61B4D03D0000002E8A19A33BF9
:10161000C14920259A837B39A0A5050820A5050886
:10162000FDF740F942F2FB13C3F6F9739C42804682
:1016300089461AD01EA3D3E90023FDF733F90D46DE
:1016400004462B462246C7E9004540464946FDF779
:1016500027F917A3D3E90023FDF724F94FF0FF354D
:10166000C7E90201B7E6032495E613A3D3E90023F3
:10167000FDF718F912A3D3E9002380468946FDF748
:1016800011F90D4604462B462246C7E9004540465F
:101690004946FDF705F90AA3D3E90023FDF702F94E
:1016A0004FF0FF35C7E9020195E6DDE906AB03E738
:1016B0003163621A61B4D03D0000601A61B4D03D5C
:1016C0007370032E8A19A33B2DE9F84353EC102BBA
:1016D00000242546C7F6F074C7F6F0751C40AC42EE
:1016E0002DED028BB0EE408AF0EE608A194610466E
:1016F00000F0AB80002B7FDD1A1500F08980A2F589
:101700007E7721F07F4323F47003073FD20743F431
:10171000801366D5C20F4FF0000C02EB43037F101D
:101720004200654616204FF400116C18D60F9C42FB
:101730004FEA420202DC65181B1B8C444908013841
:1017400006EB4303F1D1202680464FF0004107E02D
:1017500043D0D40F49085200013E04EB43031BD091
:10176000AB4208EB0104F3DD04F00049B9F1004F8E
:1017700004EB01082BD0A9469442C5EB0303C4EB4C
:10178000020288BF013B4018D40F49085200013EB5
:101790004D4604EB4303E3D11A4327D146084FEAF1
:1017A0006C0101F17E511CF0010F01F5C00118BF61
:1017B00046F0004601EB0753324643EC182BB0EEDF
:1017C000480AF0EE680ABDEC028BBDE8F883B8F178
:1017D000000FD0DB05F10109CEE79442C4D91D46C4
:1017E000B7E7C20F02EB4303400093E7431C39D035
:1017F00000F001031818D1E723F000441443DED0B1
:10180000002B36D11A46C10A153A40050029FAD0F4
:1018100011F4801329D149000133CC02FBD5C3F167
:101820000105C3F1200420FA04F452192143984021
:10183000A2F57E7721F07F4323F47003073FD207A0
:1018400043F480133FF566AFCBE751EC100BFDF787
:10185000DBF902460B4651EC180BFDF723F841EC7F
:10186000180BACE70CF1010C99E7202401250023AB
:10187000D9E751EC100B0B46FDF712F802460B4668
:10188000FDF7ECFA41EC180B99E700BF00000000EF
:101890002DE9F04F5BEC10AB2DED028BB0EE418AE1
:1018A000F0EE618A2BF00044B4F1795F85B071DA13
:1018B00050465946FDF742FC002800F0FD80524694
:1018C0005B4650465946FDF79FF981A3D3E90023B3
:1018D00006460F46FDF798F97FA3D3E90023FCF7EE
:1018E000E1FF32463B46FDF78FF97DA3D3E90023A4
:1018F000FCF7D6FF32463B46FDF786F97AA3D3E9DB
:101900000023FCF7CFFF32463B46FDF77DF978A375
:10191000D3E90023FCF7C4FF32463B46FDF774F9D8
:1019200075A3D3E90023FCF7BDFF32463B46FDF724
:101930006BF98046894600230022C3F6E0733046E7
:101940003946FDF761F94246CDE900014B46304684
:101950003946FDF759F953EC182B04460D4650460D
:101960005946FDF751F902460B4620462946FCF739
:1019700097FF02460B46DDE90001FCF791FF0B469D
:1019800000210246C3F6F0710020FCF789FF41EC0C
:10199000100B83E052465B4650465946FDF734F93A
:1019A0004BA3D3E9002306460F46FDF72DF94AA3C2
:1019B000D3E90023FCF776FF32463B46FDF724F9D6
:1019C00047A3D3E90023FCF76BFF32463B46FDF704
:1019D0001BF945A3D3E90023FCF764FF32463B46DD
:1019E000FDF712F942A3D3E90023FCF759FF324671
:1019F0003B46FDF709F940A3D3E90023FCF752FF6A
:101A00003B463246FDF700F943F23233C3F6D37357
:101A10009C42804689468EDD0023C3F6E9739C42D2
:101A200041DC0021A4F5001300220020C3F6F07170
:101A300014461D46FCF734FFCDE9020100230022C5
:101A4000C3F6E07330463946FDF7DEF822462B46F2
:101A5000FCF726FF4246CDE900014B4630463946A9
:101A6000FDF7D2F853EC182B04460D465046594664
:101A7000FDF7CAF802460B4620462946FCF710FF40
:101A800002460B46DDE90001FCF70AFF02460B4661
:101A9000DDE90201FCF704FF41EC100B05B0BDECE1
:101AA000028BBDE8F08F9FED067B00258DED027B5C
:101AB0000024C3F6D275C1E79FED030BEEE700BF2C
:101AC000000000000000E73F000000000000F03FC1
:101AD000D43888BEE9FAA8BDC4B1B4BD9EEE213E9B
:101AE000AD529C804F7E923E9015CB19A001FA3EDC
:101AF0007751C1166CC1563F4C5555555555A53FAC
:101B00002DE9F04F4AF6AB25ADF51B7DD41EC2F68C
:101B1000AA2585FB0465E417A49F114E0690C4EB2B
:101B2000A50424EAE47456F827600A941F46E343A8
:101B300003EB43037C1E02EBC30314EB0608099678
:101B400002940891079321D40A9EA599351B08F1A8
:101B500001080CAE4FEA8808002401EB85090BE070
:101B6000A8A6050859F80400FCF7E8FF043401357D
:101B70004445E6E9020109D0002DF3DA04340020DF
:101B8000002101354445E6E90201F5D1099C002C0C
:101B90002CDB099C5EAE06EBC4060DF5B87ABB469D
:101BA0000096029D002DC0F254820EA9069D01EB05
:101BB000CB064FF000084FF00009002476E902231D
:101BC000F5E80201FDF720F802460B46404649467B
:101BD000FCF768FE0134BC4280468946EED1EAE952
:101BE0000289009DAA450BF1010BDAD1099E731EF3
:101BF0009B0086AC9AAD04EB8604ED180B9300961F
